:020000040800F2
:20000000F0FF00101D1E070879F8000829180508BD1E0708BD1E0708BD1E07080000000012
:2000200000000000000000000000000075F8000871F80008000000006DF800089DDB0408E9
:20004000BD1E0708BD1E0708BD1E0708BD1E0708BD1E0708BD1E07087D2E0508452E0508EC
:200060000D2E0508D52D05089D2D050859CD060849CD060839CD060829CD060815CD0608F2
:2000800001CD0608EDCC0608BD1E0708BD1E0708BD1E0708BD1E0708BD1E0708652D05088C
:2000A0003DC10408BDC104082DC10408E1C10408B1C10408A1C1040891C10408590A070848
:2000C000610A07084D0A0708550A0708BD1E0708BD1E0708ADDF0408F1DE040835DE04086C
:2000E0002D2D0508BD1E0708311101081DC104084DC104080DC1040871C10408D9CC060895
:20010000BD1E0708F5A9060881C10408BD1E070879DD0408BDDC04084D090408390904085A
:20012000C5CC0608B1CC06089DCC060889CC060875CC0608BD1E0708BD1E0708BD1E0708AE
:20014000BD1E0708BD1E0708BD1E0708F9F1000861CC06084DCC060839CC060801DC040891
:20016000410A0708490A0708BD1E0708BD1E0708BD1E0708BD1E0708BD1E0708BD1E070847
:20018000BD1E0708BD1E0708FFFFFFFFFFFFFFFFFFFFFFFFFFFFFFFFFFFFFFFFFFFFFFFFA3
:2001A000FFFFFFFFFFFFFFFFFFFFFFFFFFFFFFFFFFFFFFFFFFFFFFFFFFFFFFFFFFFFFFFF5F
:2001C000FFFFFFFFFFFFFFFFFFFFFFFFFFFFFFFFFFFFFFFFFFFFFFFFFFFFFFFFFFFFFFFF3F
:2001E000FFFFFFFFFFFFFFFFFFFFFFFFFFFFFFFFFFFFFFFFFFFFFFFFFFFFFFFFFFFFFFFF1F
:20020000FFFFFFFFFFFFFFFFFFFFFFFFFFFFFFFFFFFFFFFFFFFFFFFFFFFFFFFFFFFFFFFFFE
:020000040800F2
:2028000000C00F0800001008FFFFFFFFFFFFFFFFFFFFFFFFFFFFFFFFFFFFFFFFFFFFFFFFE1
:20282000FFFFFFFFFFFFFFFFFFFFFFFFFFFFFFFFFFFFFFFFFFFFFFFFFFFFFFFFFFFFFFFFB8
:20284000FFFFFFFFFFFFFFFFFFFFFFFFFFFFFFFFFFFFFFFFFFFFFFFFFFFFFFFFFFFFFFFF98
:20286000FFFFFFFFFFFFFFFFFFFFFFFFFFFFFFFFFFFFFFFFFFFFFFFFFFFFFFFFFFFFFFFF78
:20288000FFFFFFFFFFFFFFFFFFFFFFFFFFFFFFFFFFFFFFFFFFFFFFFFFFFFFFFFFFFFFFFF58
:020000040800F2
:20400000AEBE08000E02000000000B0014020000000000FF000A0013020000000001351097
:2040200000030101000000000000000000000076000D0001000100000014050405000000D4
:204040000000000000000504050000000000000000010504050000000040000000020504F8
:20406000050000000000000000030504050000000000000000040504050000000000000018
:20408000000505040500000000000000001E05040500000000000000001F050405000000B4
:2040A0000064005200070009020000282A00FD01000019002A1000360000000000001A0045
:2040C0002B1142370000000000000000390000380000000000000700FB010000280F00FC84
:2040E0000100000000000000000000000C00F70100002401000000000A00F901000025006D
:2041000000004500160200002802FF3802FF2002002102001301011201002601001801FF34
:204120001901001A010000000000000000000000000000000000000000000000000000004A
:2041400000000000000000160034000000DC0532000000000000000000000001040E0011DE
:2041600002000000000000010101010A0012020100FFFFFFFF3E00180003000001030204BB
:2041800005060702000000000001006400DC051A046C070019750343080E00000100000049
:2041A000001E1E1E0101000000000000000000000000001100000200000000000000FF0091
:2041C000000000000B00FF01020002272C0101150008020100151617FFFF2D2E2F00FF3A58
:2041E0003B3CFFFF0900FA0100002C02000E002A020000960058022C0103000E0020020589
:204200000003643200F40196002A0006000100E001070000010020211312381800000002A8
:20422000000001020304050607C2012E04D007E8030C000A000C020000011F030012001141
:204240000000000100123456789ABC000000001A00FE010000013200300131000002000043
:204260000000000000FF01FF001600120003000000000100000553343035000008020020F8
:20428000000B000300AE014A015E012C0164010100000001000A019A01001E0A0000022A29
:2042A000001F000500000000000001000100050000010203000000000000000000000000CD
:2042C0000000000000008017000A00050200000000000016001B02000006000000E8030012
:2042E00000000000000000000012001B000200002600020301F40132000164F600210200BE
:2043000000000000000000000000000000000000000000000000000000000000000000009D
:2043200000000000000000000000000000000000000000000000000000000000000000007D
:2043400000000000000000000000000000000000000000000000000000000000000000005D
:2043600000000000000000000000000000000000000000000000000000000000000000003D
:2043800000000000000000FFFF000000FF1E0000FF3C0000FF5A0000FF780000FF96000062
:2043A000FFB40000FFD20000FFF00000FF0E0100FF2C0100FF4A0100FF0000000000000007
:2043C00000010B020D0A03050B030D0A030A0B040D0A03080B040D0A03070B030D0A0300F5
:2043E0000000000000060A0100000203060000000336003700010020003200C800D00796A9
:20440000001400320028004C0440060005500014000F00080064000100010005000A0000A3
:2044200000F40196000F000C0016000100C4090000190028002F0001000000000000000081
:2044400000000000000000000000000000000000000000000000000000000016002302021F
:2044600000000000000000000000000000FF0000000F001E0000000005010000000000000A
:204480001200050002000201000000000000000000008200FD070000EA00EA00CD004E008B
:2044A000CE00EA00EA00EA00EA00EA00EA00EA00EA00EA00EA00EA00EA00EA00EA00EA0078
:2044C000EA004939EA00EA00EA00EA00EA00EA00EA00EA00EA00EA00EA00EA00EA00EA00A4
:2044E000EA00EA00EA00EA00EA00EA00EA00EA00EA00EA00EA00EA00EA00EA00EA00EA001C
:20450000EA00EA00EA00EA00EA002300EA00EA00CD00EA007200F5010900980864001401D1
:20452000000A010A0000FF1F0000142800002C3700008000FFFFFFFF4600010200000000E4
:2045400000000000000000000000000000000000000000000000000000000000000000005B
:20456000000000000000000000000000000000005000C4FF00FFFFFFFF0100000005180B03
:204580000C00000000001600230002000A0000000000000000000000000000001400260090
:2045A000010002032300000115005802D90300000B0014000000030100230012000100022B
:2045C00000E80364000F0A00010A001E002A000A00090030000000FA00F4010000000000EE
:2045E0000000000000020000029E077D00FA00F401000105016400C2010E00030064004BB8
:2046000000000000002D50280078002F542E007D002D500000780032324B00000028000083
:204620000000000055F401900101374B000000FA00AC0D00000000320090015E01F4010052
:20464000000A64C8009001960000050F00010F0114004B3200005A140B00004B00960000ED
:204660001400280100C8001E22002514640000000000000000000000003232329600001913
:20468000070F5A050000026464646464646401646464004B00000000002D50280078002F23
:2046A000542E007D002D500000780032324B0000002800000000000055F401900101374BD1
:2046C000000000FA00AC0D00000000320090015E01F40100000A64C8009001960000050F9F
:2046E00000010F0114004B3200005A140B00004B009600001400280100C8001E2200251440
:204700006400000000000000000000000032323296000019070F5A05000002646464646485
:20472000646401646464004B00000000002D50280078002F542E007D002D500000780032C7
:20474000324B0000002800000000000055F401900101374B000000FA00AC0D000000003271
:204760000090015E01F40100000A64C8009001960000050F00010F0114004B3200005A14D3
:204780000B00004B009600001400280100C8001E220025146400000000000000000000004B
:2047A0000032323296000019070F5A05000002646464646464640164640A00130001000892
:2047C0000045100A0001010000000000000A0000010000900100000900020100006E0A0157
:2047E000220122020000000000000000000000000000000000000000000000000000000072
:20480000000000000000000000000000000000000000000000000000000000000000000098
:20482000000000000000000000000000000000000000000000000000000000000000000078
:20484000000000000000000000000000000000000000000000000000000000000000000058
:20486000000000000000000042414E44312020200042414E44322020200042414E44332083
:2048800020200042414E44342020200042414E44352020200042414E443620202000424157
:2048A0004E44372020200042414E44382020200031323334353637383100320033003400B4
:2048C0003500360037003800000000000000000000000000000000000000000000000000FE
:2048E00000004C5630004C5631004C5632004C5633004C5634004C5635004C5636004C5643
:204900003700EA000C000400320003070707000000434343410046050064CE07CE07CE07E4
:20492000010000000000000000000000000032000307070700000043434341004605006473
:20494000CE07CE07CE070100000000000000000000000000320003070707000000434343C4
:20496000410046050064CE07CE07CE0701000000000000000000000000003200030707077D
:20498000000000434343410046050064CE07CE07CE070100000000000000000000000000DE
:2049A000320003070707000000434343410046050064CE07CE07CE07010000000000000074
:2049C000000000000000320003070707000000434343410046050064CE07CE07CE07010054
:2049E000000000000000000000000000110001020000000000000200000000000009000296
:204A0000020000000000760015000000000000000000000000000000000000000000000009
:204A2000000000000000000000000000000000000000000000000000000000000000000076
:204A4000000000000000000000000000000000000000000000000000000000000000000056
:204A600000000000000000000000000000000000000000000000000000000000070003002C
:204A800000000066002A00000000000000E803D007DC0564FF00000000E803D007DC056479
:204AA000FF00000000E803D007DC0564FF00000000E803D007DC0564FF00000000E803D030
:204AC00007DC0564FF00000000E803D007DC0564FF00000000E803D007DC0564FF0000007F
:204AE00000E803D007DC0564FF16002C000000E803D007E803D007E803D007E803D0077EE8
:204B000000290002000000000000000000000000000000000000000000000000000000006A
:204B2000000000000000000000000000000000000000000000000000000000000000000075
:204B4000000000000000000000000000000000000000000000000000000000000000000055
:204B6000000000000000000000000000000000000000000000000000000000000014001A07
:204B80000000007E05EA05B4053200E803D00700002A002B000000001E001E001E00050141
:204BA0001E011E011E011E011E011E011E011E011E011E011E011E011E011E160019020013
:204BC00000000000000000000000000000000000001200F6010200000000000100000002C7
:204BE00002000022001C0200000002011400003404000000008C0A01020100000000010089
:204C000000000000001C002800030000010102000000000000000000000000000000000049
:204C200000080004020100391807000F020000000C00F80103000101F401140008001000D1
:204C4000010000050B00190000000000280100460029020000000000000000000000000090
:204C6000000000000000000000000000000000000000000000000000000000000000000034
:204C80000000000000000000000000000000000000000000000A002C020000190019001A90
:204CA000000A02000000004A01B400D6010000C2010E01960044000000320125000200000C
:204CC0000000000000000000000000000000000000000000000000000000000000000000D4
:204CE0000000000000000000000000000000000000000000000000000000000000000000B4
:204D0000000000000000000000000000000000000000000000000000000000000000000093
:204D2000000000000000000000000000000000000000000000000000000000000000000073
:204D4000000000000000000000000000000000000000000000000000000000000000000053
:204D6000000000000000000000000000000000000000000000000000000000000000000033
:204D8000000000000000000000000000000000000000000000000000000000000000000013
:204DA0000000000000000000000000000000000000000000000000000000000000000000F3
:204DC0000000000000000000000000000000000000000000000000000000000000000000D3
:204DE00000000000000000000000004300030201000000000000000000000000000000006A
:204E0000000000000000000000000000000000000000000000000000000000000000000092
:204E200000000000000000000000000000011200020000000000000000000000000000005D
:204E40000A0028020000000000000A00270200000000000016001F020000FFFFFFFFFFFFBA
:204E6000FFFFFFFFFFFFFFFFFFFF42001A02000000000000000000000000000000000000DE
:204E8000000000000000000000000000000000004245464800424554414650564634303516
:204EA000000000000000000000000100090038000200000A07860004000000000000000013
:204EC0000000000000000000000000000000000000000000000000000000000000000000D2
:204EE0000000000000000000000000000000000000000000000000000000000000000000B2
:204F0000000000000000000000000000000000000000000000000000000000000000000091
:204F200000000000000000000000000000000000000000000000000000000012002B020032
:204F4000000000000000000000000000FF080007020000023C0C001D0200000000000000D8
:204F6000001800060201000000000020030000000020030000000020030B00390000000063
:204F8000000000000A00270000002003000043000B0202000000000000000000000000006B
:204FA0000000000000000000000000000000000000000000000000000000000000000000F1
:204FC00000000000000000000000000000010000001A000D020100000000000000000000A6
:204FE00000000000000000000000000C001E0200000000000000000700100200000000006C
:20500000DEAD0000FFFFFFFFFFFFFFFFFFFFFFFFFFFFFFFFFFFFFFFFFFFFFFFFFFFFFFFF21
:20502000FFFFFFFFFFFFFFFFFFFFFFFFFFFFFFFFFFFFFFFFFFFFFFFFFFFFFFFFFFFFFFFF90
:20504000FFFFFFFFFFFFFFFFFFFFFFFFFFFFFFFFFFFFFFFFFFFFFFFFFFFFFFFFFFFFFFFF70
:20506000FFFFFFFFFFFFFFFFFFFFFFFFFFFFFFFFFFFFFFFFFFFFFFFFFFFFFFFFFFFFFFFF50
:20508000FFFFFFFFFFFFFFFFFFFFFFFFFFFFFFFFFFFFFFFFFFFFFFFFFFFFFFFFFFFFFFFF30
:020000040800F2
:020000040800F2
:20800000F0B401292A4C2B4D23684FF0000694BF00270127EE626662A6626763676B47EA45
:2080200042076763EE63EC6B002A38D144F49574EC631C6824F001041C601C68E407FCD46A
:20804000490289085960D8601968EAB921F04001196019498B421DD018494FF47410C860F8
:20806000196841F01E011960596941F080015961196841F00101196022B90E4AD36A43F0B8
:208080000803D362F0BC704741F0400119600A498B42E1D14FF0746041F8500CE0E744F0DD
:2080A0001A04EC63EC6A44F00804EC62C1E700BF481E0020002C0140586402400064024071
:2080C0001148002302461178032902F1060216D00133062BF7D10D4AD36D052B0ED0591CFF
:2080E00003EB4303D16500EB4303032040F2EB3140F2FF32187059809A807047704703EB3A
:20810000430300EB4303F0E7801E0020481E002070B4C3080D4CE25C00F00706B24004EB69
:20812000D004D2B20020C6F108038B4228BF0B46C3F108052A419840C91A40EA02004FF0AE
:20814000000614F8012FEED170BC7047E81E0020084AD2E9553199420AD0D118013391F827
:208160005C110170C3F30A03C2F854310120704700207047481E0020064BD3F86009D3F89A
:208180005C29D3F85C39824298BF03F50063181A704700BF481E0020012380F85130704782
:2081A00007B501A8FFF7D4FF0028FAD09DF8040003B05DF804FB044BD3E95503984288BF7B
:2081C00003F50063181A7047481E002001207047024BC3F86429C3F868197047481E0020EF
:2081E000024BC3F86C29C3F870197047481E00207047704730B4134DD5E955239A4286BF58
:2082000003F50064A21A9A1A0A44B2F5006F13D8A9B101444A1E013810F8014FE9188242E6
:2082200003F1010381F85C41C3F30A03F4D1C5F85831002030BC7047022030BC704708468C
:20824000F8E700BF481E002041B370B5144C0144D4F860394E1E451E1A4604E0012045F06E
:20826000F9FBD4F86029D4F85C19531CC3F30A038B42F3D0D4F85C19B1F5006FEED094F812
:2082800074190029EAD115F8011FC4F860392244B54282F87819DFD1002070BD00207047AF
:2082A000481E002010B5094CD4F88030084611465BB1D4F88030052B07D1002AD4F88430C3
:2082C00003DDFFF7C1FFD4F8843010BD402F002010B590F85010002380F8503081B10B4CDB
:2082E000D4F8802072B1D4F88020052A0CD13C30D4F88430FFF7A8FFD4F88430012010BD80
:208300000120FCE71046FAE71846F8E7402F0020002280F85120DBE790F85020531C0244DC
:20832000DBB280F8503082F83C1090F851200AB1132B00D9CCE77047212838B50C4605D060
:2083400022282FD0202813D0002038BD0029FBD0072AF9D11A4BD3F8880093F88C1093F83B
:208360008D2093F88E30206021716271A371EBE70029E9D0072AE7D1124AD2F868391BB1DE
:20838000D2F86409096898470D4B256820796179A279C3F8885083F88C0083F88D1083F8B6
:2083A0008E20D1E70029CFD0022ACDD1054AD2F87039002BC8D00988D2F86C099847C3E7E7
:2083C000402F0020481E0020024B0020C3F88000704700BF402F0020054B064A00200521F5
:2083E000C2F88010C3F87009C3F86809704700BF481E0020402F0020704700BF704700BF5C
:20840000704700BF704700BF704700BF704700BF704700BF042301480B80704788010020B3
:2084200010B4074A074B92F89000122403F114020C8001280CBF184610465DF8044B7047EC
:20844000402F00208C01002000487047D01E002000487047D01E0020034B93F8840003283E
:2084600094BF002001207047481E0020034B93F88400032894BF002001207047481E0020D2
:20848000034B93F88400003818BF0120704700BF481E0020A0B182680D4B12B107229A70CA
:2084A00070471978DA6003294FF004000CBF80214FF48071C3E901111A611A7598707047A4
:2084C000034B41F2E47101225A545A70704700BF1CA100200378022B10D0006908B9012005
:2084E00070470C4B1B78032B0EBF0B4B80B24FF6F773984294BF002001207047054943688B
:2085000041F650028A58B3EB422F2CBF01200020704700BF1CA10020F7FFFF0F0378022BB6
:2085200014D030B4104A4368006941F6480402F5C2511559096841F63C042B4012595B0AE7
:20854000023801FB0030104430BC7047064B426841F6340141F630005958185800EB4100A3
:2085600000EB5220704700BF1CA100202DE9F84F494B98420ED003F56853083398424ED0BC
:20858000464B0020C3E94000A3F8FC00A3F80801BDE8F88F414C424FDFF810810223C4F870
:2085A000943004F198060025FB6AAB42294605F1010503D0D4F8180159F0F8FA94F81C31B6
:2085C000D4F8182186F8243032623046414659F001FDD4F894309D4206F13006E4DB00236E
:2085E00084F80A31D4E92803D4F89410B4F89C20B4F8A850C4F8283112FB01F203FB01F359
:20860000A4F8FC20B4F89E10264AA4F80851C4E94003A4F8FE10C4F8F8200120B8E71F4C4A
:208620001F4F0223C4F8943004F198054FF0000B4FF4806A4FF040094FF40068FA6A012660
:208640005A455946B34403D0D4F8180159F0AEFAD4F8181194F81C21296285F824204FF4EF
:2086600000314FF00062C5E90212A5F804A0A5F81090A5F80680AE74FFF722FD28466E763C
:2086800059F0F4FBD4F89420074B45F8303B9345D4DB84F80A61A5E71971EF00402F002026
:2086A0008801002074460708484607081940EF002DE9F04FD84DDFF89083DFF89CA307469C
:2086C0000E4693460FCD44462DED068B0FC40FCD0FC495E8070089B09AF82E31CDF808B0AF
:2086E00084E80700CDE90476042B00F26781DFE813F0D201650160010500E2019FEDC78AA5
:20870000DFEDC78AC749C8F81C10C749C74BC84AC8F818100299002918BF134638EE887A08
:20872000F5EE006A86EE87AAC24EDFF830B3C8F824300025DFEDC07A9FEDC09A28EE278A91
:20874000F0EE679A059BAB4200F02D811BF8013B0AEB030292F83341002C00F03481DFF820
:2087600000C3002202E0152A00F02D8102EB420157001CF80100A04202F10102F3D1514488
:2087800091F85111002900F084812046039344F037F8039B81464846039344F051F80178F2
:2087A000002940F01081039B57440133DBB2032287F8913187F89021B9F1000F00F0038112
:2087C0002709013F052F04F00F0000F24D819C4C04EB4701B1F884C04CFA00F111F00101EC
:2087E00000F04281012101FA00F0013800EA0C002744039369F044F997F89070DFF864C267
:20880000039B38440CEBC0070322FB71BA715CF83000776100F13F4303F57E0304EB9324D6
:20882000012194F8983099F8082003F01F045B09032B01FA04F100F01D81042B00F024811F
:20884000022B00F01C81BB880693B3FA83F3C3F11F03C3F3CC0100EB810103F007030C6A26
:208860009B000F279F4024EA07040C620C6A02FA03F323430B62022306A907930CF0B0FE6E
:20888000029B002B00F0AE80BAF82C3100EE103AB8EEC00AFCEEC07A17EE901AD9F8003067
:2088A000684A934200F09B80A2F58062934200F0968002F58042934200F0918002F580626A
:2088C000934200F08C8002F58062934200F08780DAF8BC2450084FF6FF73B0FBF1F21A4475
:2088E000120CB0FBF2F20298002800F08480B2FBF1F19AF82E0104288BB200F0828007EE75
:20890000902AF8EE676A66EE887A29EE677A9AF82F0104990091A8EEA67A0190494630465C
:20892000C6ED027A86ED037A37F0F8FC002D40F39D807368D8F83820934200F09980012D71
:2089400000F09480D8F85020934200F09180022D00F08C80D8F86820934200F08980032D7C
:2089600000F08480D8F88020934200F08180042D7CD0D8F8982093427AD0052D76D0D8F861
:20898000B020934274D0062D70D0D8F8C820D31A18BF012301350122082D3374727406F1C9
:2089A00018067FF4CFAE284809B0BDEC068BBDE8F08F9FED268AF0EE488AA3E69FED248A73
:2089C000F0EE488A9EE6234A194BC8F81C200020C8F8243009B0BDEC068BBDE8F08FDAF879
:2089E000BC0478E7B0EE4A0A6AF04AFAFCEEC07A17EE901A52E79AF82E01042819467FF4FD
:208A00007EAF07EE901A07EE102AF8EE677AF8EE476A67EEA97A78E7A0460708ACC5A737E2
:208A2000ACC5A73699CC030861A704082DC7030855A704083C0000106F12833A00007A4415
:208A4000484607080004014008000010282930386F12033925CA0308402F00207E3000204F
:208A600090300020FC300020716109E7012391E700238FE7114B1C6C21431964E3E60F4BEB
:208A80005C6C21435964DEE60C4B1C6B21431963D9E689467FE69FED0A8A0A4BC8F81830FB
:208AA0000023094A049301230293C8F81C20074BF0EE488A32E69FED068AEEE7003802406F
:208AC0006F12833A61A7040899CC030855A7040800000000F8B5104ED6F8BC440546006840
:208AE0000F4664080CF080FCB4FBF7F1B1F5803F03D3012CFAD96408F6E72246284689B211
:208B000043F032FC054BC6F8243D28460449BDE8F840002243F06CBB402F00201D4002087B
:208B2000643C002010B5044C04480A4621460BF09DFA204610BD00BF6C3C002014E007080E
:208B400010B5044C04480A4621460BF08FFA204610BD00BF6C3C002024E0070810B5044C97
:208B600004480A4621460BF081FA204610BD00BF6C3C002030E0070810B5044C04480A46F2
:208B800021460BF073FA204610BD00BF6C3C00203CE0070810B5044C04480A4621460BF00E
:208BA00065FA204610BD00BF6C3C002048E0070810B50D4C94F852210023C4F8803012B1F6
:208BC0000A4AC2F82C3E61F075FF20B10423022084F8843010BD054BD3F88430636709237C
:208BE00084F8843010BD00BF481E0020402F002070B50D4D95F88430042B04460E460AD03D
:208C0000082B06D1EB6F83420CD0FFF7D1FF022801D0012070BD0823C5E91F4685F88430D1
:208C2000022070BD022070BD481E002070B50379234C002B14BF0123002384F8B03003D18B
:208C4000002384F8843070BD1E4D002195F9332E032045F0DDFB0028F2D04668304645F0A6
:208C6000C5FB84F851010028EAD095F8313E003B18BF0123304684F8523162F0A9FE0BF0E9
:208C8000A3F938B994F8783084F88400013384F8783070BD61F0F8FF40B194F878300022FF
:208CA000013384F8783084F8842070BDD5F884306367012384F8780084F8843070BD00BF90
:208CC000481E0020402F002010B561F0DDFF58B10C4C94F878300133DBB2072B84F87830E1
:208CE00003D9002384F8843010BD0BF06DF90028F7D0054A0123D2F88420626784F884304E
:208D000010BD00BF481E0020402F00202DE9F041884C94F8B050002D00F0FA8094F8842044
:208D2000854E0227531E082B41D8DFE803F03739A0406A511540050061F0BCFE002840F0F8
:208D4000EE80636FD6F88420FA3393422CD2FFF7BBFF94F88420E5E761F0ACFE0028F0D0D2
:208D6000D4F880300022012B84F8782040F2DB80E16F94F85201013B0131C4E91F1310B14B
:208D80006D4BC3F82C2E082284F88420A2F10805B5FA85F56D092846BDE8F08184F8847089
:208DA00061F088FE002843D194F88420531EDBB2022B0AD8604B616FD3F884305B1AC82B01
:208DC000E4D9FFF781FF94F88420042ADED1E2E7236B002BDAD1584BE66ED3F884306367E6
:208DE000072284F88420002ED0D0D4E91821236F0120B047D8E7636FD6F8841064338B4265
:208E0000C4D2D4F82C80B8F1000FF4D161F052FE00289ED0E66E84F87880042384F8843071
:208E2000002E7AD0D4E91821236F4046B047BBE761F0E6FA0028B7D196F8353E002BA3F172
:208E40000203B3FA83F314BF022201225B0984F8792084F87A3061F0D3FA00287FF477AF52
:208E6000364A0323926CC4F8882084F8843061F0C7FA002898D1304BC4F8800093F8646E03
:208E8000B3F8660ED3F868EED3F868CED3F8687ED3F8682E84F88E6093F86C1EA4F88C00D8
:208EA00093F86D6E84F8922093F86D0ED3F8702EC4F89420B3F8768EB3F8762E84F8931022
:208EC000B3F8761EC2F30B1343EA182303F00F0301F00F024FEA1E6E4FEA1C4C3F0A360923
:208EE00000F00F0003F5FA63042184F8990084F88FE084F890C084F8917084F89860A4F8A0
:208F00009A3084F89C2084F884102846BDE8F08184F884502846BDE8F08105463BE7042353
:208F200084F8843037E7FAD1FFF742FE94F88420531E3CE7481E0020402F0020783D002034
:208F40002DE9F84FBA4C94F8901E0546C1F34001D4F8980E48F046FC94F8901ED4F8940EA0
:208F6000C94301F0010148F03DFC002D00F0CD806E1EB04FB04D5FFA86FB4FF01008D4F892
:208F8000980E48F095FAD4F8940E48F091FAB4F8A03E002B40F0438194F8A21ED4F8A40EC0
:208FA00048F020FC4FF0FA094FF47A704FF0010C7B68C3F30803002B40F00881EFF31183A4
:208FC000002B40F00381D4F88420A968D4F884309A42F8D1D4F8C83E9942F4D8D4F8C46E95
:208FE00000FB06F35B1AB3FBF6F300FB02327B68C3F30803002B40F0A880EFF31183002B7A
:2090000040F0A380D4F88430D5F808A0D4F884108B42F7D1D4F8C81E8A45F3D8D4F8C46EC9
:2090200000FB06F1A1EB0A01B1FBF6F100FB03139B1AB3F57A7FDAD3B9F10109B8D1D4F8F7
:20904000980E48F035FAD4F8940E48F031FAB4F8A03E002B40F0D78094F8A21ED4F8A40E2C
:2090600081F0010148F0BEFB4FF0FA0C4FF47A704FF0010E7B68C3F30803002B40F08680C7
:20908000EFF31183002B40F08180D4F88420A968D4F884309A42F8D1D4F8C83E9942F4D8DF
:2090A000D4F8C49E00FB09F35B1AB3FBF9F300FB02327B68C3F308034BBBEFF3118333BB3F
:2090C000D4F88430D5F808A0D4F884108B42F7D1D4F8C81E8A45F3D8D4F8C49E00FB09F137
:2090E000A1EB0A01B1FBF9F100FB03139B1AB3F57A7FDED3BCF1010CBCD10BF1FF365FFA5A
:2091000086FBBBF1FF0F7FF43AAFBDE8F88FEFF3118988F31288AE682B68DB0344BFC4F8B5
:20912000C0EEAE68D4F88430D4F8C01E5FFA89F989F31188D4F8C49E0B4400FB09F1891B3B
:20914000B1FBF9F100FB0313D0E7EFF3118E88F31288D5F808A02B68D90344BFC4F8C0CEEA
:20916000D5F808A0D4F88430D4F8C01E5FFA8EFE8EF31188D4F8C46E0B4400FB06F1A1EB86
:209180000A01B1FBF6F100FB031351E7EFF3118188F31288D5F808902B68DA0344BFC4F8CB
:2091A000C0EED5F80890D4F88430D4F8C02EC9B281F31188D4F8C41E1A4400FB01F3A3EB51
:2091C0000903B3FBF1F300FB023272E7EFF3118188F31288AE682B68DB0344BFC4F8C0CE0C
:2091E000AE68D4F88430D4F8C02EC9B281F31188D4F8C41E1A4400FB01F39B1BB3FBF1F354
:2092000000FB0232F3E6D4F8BC3E002B3FF42CAFD4F8A83EC3F8009084F8B99E24E7D4F8A0
:20922000BC3E002B3FF4BEAE44F0D8FCBAE600BF402F002000ED00E010E000E02DE9F84F7A
:20924000B74CB84F94F8901ED4F8980EB64DC1F3400148F0C7FA94F8901ED4F8940EC943B3
:2092600001F0010148F0BEFA4FF0050B4FF01008D4F8980E48F01CF9D4F8940E48F018F9EF
:20928000B4F8A03E002B40F0438194F8A21ED4F8A40E48F0A7FA32264FF47A704FF0010CB1
:2092A0007B68C3F30803002B40F00781EFF31183002B40F00281D4F88420A968D4F88430D2
:2092C0009A42F8D1D4F8C83E9942F4D8D4F8C4EE00FB0EF35B1AB3FBFEF300FB02327B68D0
:2092E000C3F30803002B40F0A780EFF31183002B40F0A280D4F88430D5F808A0D4F88410E3
:209300008B42F7D1D4F8C81E8A45F3D8D4F8C4EE00FB0EF1A1EB0A01B1FBFEF100FB0313B1
:209320009B1AB3F57A7FDAD3013EB9D1D4F8980E48F0BEF8D4F8940E48F0BAF8B4F8A03E1F
:20934000002B40F0DA8094F8A21ED4F8A40E81F0010148F047FA4FF0320C4FF47A700126D1
:209360007B68C3F30803002B40F08780EFF31183002B40F08280D4F88420A968D4F8843013
:209380009A42F8D1D4F8C83E9942F4D8D4F8C49E00FB09F35B1AB3FBF9F300FB02327B6869
:2093A000C3F308033BBBEFF3118323BBD4F88430D5F808A0D4F884108B42F7D1D4F8C81E06
:2093C0008A45F3D8D4F8C49E00FB09F1A1EB0A01B1FBF9F100FB03139B1AB3F57A7FDED38B
:2093E000BCF1010CBCD10BF1FF3616F0FF0B7FF43FAFBDE8F88FEFF3118988F31288D5F8FA
:2094000008A02B68DB0344BFC4F8C06ED5F808A0D4F88430D4F8C01E5FFA89F989F31188B7
:20942000D4F8C49E0B4400FB09F1A1EB0A01B1FBF9F100FB0313CFE7EFF3118E88F3128830
:20944000D5F808A02B68D90344BFC4F8C0CED5F808A0D4F88430D4F8C01E5FFA8EFE8EF3D6
:209460001188D4F8C4EE0B4400FB0EF1A1EB0A01B1FBFEF100FB031352E7EFF3118188F321
:209480001288D5F808902B68DA0344BFC4F8C06ED5F80890D4F88430D4F8C02EC9B281F3E2
:2094A0001188D4F8C41E1A4400FB01F3A3EB0903B3FBF1F300FB023271E7EFF3118188F376
:2094C0001288D5F808E02B68DB0344BFC4F8C0CED5F808E0D4F88430D4F8C02EC9B281F3A1
:2094E0001188D4F8C41E1A4400FB01F3A3EB0E03B3FBF1F300FB0232F1E6D4F8BC3E002BB0
:209500003FF429AFD4F8A83E1E6084F8B96E22E7D4F8BC3E002B3FF4BEAE44F05FFBBAE6A6
:20952000402F002000ED00E010E000E000F01F0240090123032803FA02F304D004280CD088
:20954000022805D07047074A116C0B4313647047044A516C0B4353647047024A116B0B432E
:20956000136370470038024000285FD00368374A2DE9F04103F13F4404F57E0402EB942225
:20958000012492F8982002F01F055209032A04FA05F456D0042A4FD0022A48D08588B5FA5C
:2095A00085F0C0F11F00C0F3CC0603EB860600F0070082000F24306A944020EA04003062AD
:2095C000306A01FA02F20243002132624FF0010E0A464FF0030C02270EFA02F838EA0500CA
:2095E00002F101021CD118680CFA01F420EA04001860186807FA01F606431E609E6826EA32
:2096000004069E6098689860586820EA0800586058685860D86820EA0400D860D868D8604A
:20962000102A01F10201D7D1BDE8F0817047084A556C2C435464B1E7054A156B2C431463FF
:20964000ACE7034A156C2C431464A7E74846070800380240134B0268196821EA020119604D
:20966000596821EA0201596019680A431A609968026821EA02019960D96821EA0201D96020
:209680004179102907D001F1804303F59E3319680A431A607047996811439960D9680A43A7
:2096A000DA607047003C014000286BD0F0B58388B3FA83F3202B85B00446C3F11F024CD04B
:2096C000314D32484FF00041104405EB820205F60C7731FA03F390F8A060C2F8CC7E05D04A
:2096E0002B4A116821EA0301116053612046002143F0E8FAA3882268B3FA83F4C4F11F03FC
:2097000003F0FC0101F1804101F59C3103F0030398000F2702F13F438A68874022EA0702D9
:2097200003F57E038A60C3F38723834088684FF000420343354422FA04F48B604FF440628F
:20974000012302A88DF80E300294ADF80C20FFF781FF95F8103FF02B01D805B0F0BD0D4B11
:209760009B5D8DF80430F02103224FF4807301A885F8101F8DF80520ADF806300BF0E6FC15
:2097800005B0F0BD704700BF402F002048460708003C0140C8E00708002869D0F0B5838880
:2097A000B3FA83F3202B85B00446C3F11F024AD0304E314D16444FF0004005EB820230FA5A
:2097C00003F396F8A060C2F8CC1E05D02B4A116821EA0301116053612046002143F072FA44
:2097E000A3882268B3FA83F4C4F11F0303F0FC0101F1804101F59C3103F0030398000F278C
:2098000002F13F438A68874022EA070203F57E038A60C3F38723834088684FF000420343C8
:20982000354422FA04F48B604FF40062012302A88DF80E300294ADF80C20FFF70BFF95F886
:20984000103FF02B01D805B0F0BD0D4B9B5D8DF80430F02103224FF4807301A885F8101F99
:209860008DF80520ADF806300BF070FC05B0F0BD704700BF48460708402F0020003C01407B
:20988000C8E00708034BD3F8B820136A002BFCD1704700BF481E002030B5134A134B8DB0D2
:2098A000082102F1B80082F850110693694400230DF107050124CDE9073302938DF8143013
:2098C00009938DF828300B93CDE903544AF056FBFFF7D8FF9DF80700A0F1FF00B0FA80F0C6
:2098E00040090DB030BD00BF481E00201916010870B51C4D90B00024FD220DF1030305F1ED
:20990000B800012601A98DF803200693CDE90144CDE90A44CDE90C44C5F880408DF8104026
:20992000059407948DF824408DF838400F94039608964AF023FBFFF7A5FF30460AF0FAFADD
:20994000FF2809D0084BD3F884306B672046092385F8843010B070BD0423022085F8843039
:2099600010B070BD481E0020402F0020F0B50379284C002B14BF012200228BB084F8B02086
:2099800003D184F884300BB0F0BD054604F1B80795F9001038464AF061FCAD786DBB1E4BF3
:2099A0001E48C4F84C310126C4F8C05084F8C4604AF08AFC03464FF47A70A4F8BC3044F083
:2099C00049F8D4F8C00047F007FF2822684600216AF0E9FD0A236946384602934AF0CEFA33
:2099E000FFF750FF0E4B84F88460D3F884306367002384F878300BB0F0BD284647F0A0FA32
:209A0000054608B11E23C3800921284643F036FBC5E700BF481E0020A81E0020801A06004B
:209A2000402F002070B5064690B008200D460AF081FAFF2821D0FE2802D0022010B070BDD7
:209A4000002402230E48089301A9CDE90265CDE90544CDE90A44CDE90C4401948DF8104092
:209A600007948DF824408DF838400F944AF086FAFFF708FF204610B070BD012010B070BDAA
:209A8000001F002030B593B040F040020B0E0D0C04468DF80810080A8DF80420952101AAB8
:209AA0008DF805308DF80650002306258DF807008DF809100DF1030001210392134A0493ED
:209AC000CDE90733CDE90D33CDE909018DF818308DF82C300F938DF84030119305950C92BF
:209AE000FFF7DAFE00B974B9094B082203F1B80003A983F850214AF041FAFFF7C3FE9DF82F
:209B0000030013B030BDFF2013B030BDF1150108481E00202DE9F8431A4C94F88460042ED5
:209B20000546894690461F4608D0082E02D00020BDE8F883FFF7DCFE0228F8D1D4F8C00061
:209B400047F044FE94F87A309BB969021120FFF799FFA0B90C4BC4F86090D3F88420656642
:209B60000523C4E91B87626784F884300120BDE8F88329461120FFF785FF0028EAD00AF03E
:209B8000FFF9D4E7481E0020402F002070B51E4C94F88430042B06460D4608D0082B22D162
:209BA000E36F83422DD0FFF7A3FE02281BD1D4F8C00047F00BFE00213720FFF763FF2946D9
:209BC0001720FFF75FFFB0B994F87A306BB971021920FFF757FF70B90823C4E91F6584F83E
:209BE0008430022070BD012070BD31461920FFF749FF0028F0D00AF0C3F90AF0F7F903207B
:209C000070BD022070BD00BF481E00202DE9F0412D4C0546884617461E4694F884000428AD
:209C200036D0082806D1E36FAB4206D0FFF760FE0228F2D00120BDE8F0814FF0FC0CD4F878
:209C4000B8202248117B224B80F817CFC3F8588051B1526942B194F84021002A0CBF4FF403
:209C600080724FF4007201E04FF480721A66194919484AF083F901220623C4E91885C4E9EB
:209C80001B7684F8682084F884300020BDE8F081D4F8C00047F09AFD94F87A305BB96902BA
:209CA0001820FFF7EFFE40B994F88430082BC4D04FF0FE0CC3E72946F2E70AF061F90AF000
:209CC00095F90320B7E700BF481E0020402F002088010020B8010020001F00202DE9F04F4B
:209CE000D14C94F8B06095B0002E00F0978194F88420CE4F04F1B80804F1A009531E082BEC
:209D000000F2A180DFE813F0370060002F019F008E00B1001A009F000900FFF7BDFD002827
:209D200040F03982636FD7F88420FA33934280F087800AF05BF994F88420DFE7FFF7ACFD97
:209D40000028EFD0D4F880300022012B84F8782040F23782E26F013B511CC4E91F13082250
:209D600084F88420A2F10806B6FA86F67609304615B0BDE8F08FD4F8C00047F027FD002110
:209D80000846FFF77FFE05460AF0FAF8012D57D1D4F8C0004FF0000A84F879A047F016FDC1
:209DA00040F2AB110820FFF76DFE052800F08F81012800F056810AF0E3F894F87920002AEB
:209DC000CED0022384F88430D4F8C00047F0FEFC94F87930022B0CBF4FF08045002500215C
:209DE0003720FFF74FFE29462920FFF74BFE05460AF0C6F825BB94F87930022B00F07C81A0
:209E000084F87A50D4F8C00047F0E0FC00210920FFF738FE002875D00AF0B2F894F88420A6
:209E2000531E10E0206E4FF40071FFF7FBFD012800F03581022800F03981002800F04A810B
:209E400094F88420531EDBB2022B0AD8774B616FD3F884305B1AC82B84D90AF0C7F894F8AA
:209E60008420042A7FF47EAF81E7D4F8B820117B136A002900F0DE805269002A00F0DA80B5
:209E800094F84021002A00F0D580B3FA83F35B09002BD5D004A900250DF10F030222059173
:209EA000404605A94FF0010ACDE90B3A0792CDE90955CDE90E55CDE91055ADF810500695A8
:209EC0008DF820508DF834508DF8485013954AF055F8FFF7D7FC9DF80F3003F01F03052B56
:209EE00000F062810AF082F8D4F86CB0BBF1000F00F0EA802A46236F616E5046D84794F80C
:209F00008420FBE610214846FFF78CFD8246002882D101217F20FEF7FBF8012805467FF4AB
:209F20007BAF50460221FEF7F3F8002800F0148101287FF471AF16213A20FEF7E9F801305D
:209F40008002C4F888000AF01BF8D4F8C00047F03DFC00210A20FFF795FD002840F0F58092
:209F6000032384F88430102105A8FFF75BFD00287FF466AF9DF821309DF822109DF81C2031
:209F80009DF815009DF816501B01DBB243EA111303F5FA63A4F89A30DDF81D3001F00F0144
:209FA00084F89C101BBA110902F00F0245EA002084F8981084F899209DF814109DF817205A
:209FC000C4F89430069BC4F89030A4F88C0084F88E1084F88F2009F0D3FF94F87A3073B94A
:209FE000D4F8C00047F0F2FB4FF400711020FFF749FD054609F0C4FF002D7FF49AAE0C484E
:020000040800F2
:20A000004AF062F900220423A4F8BC003046C4F8802084F8843015B0BDE8F08F304684F82D
:20A02000846015B0BDE8F08F481E0020402F002040787D01236E94F868106A4803EB0121B1
:20A0400000224FF480734AF05FFB94F868300133DBB284F86830A3F10203B3FA83F35B09FB
:20A0600016E7042304AA5F48079305A90692CDE909AACDE90BAACDF814A08DF820A08DF870
:20A0800034A0CDF838A049F079FFFFF7FBFB9DF81330AB2B04BF022384F879308BE6636FB4
:20A0A000D7F8842064339342BFF4CAAE09F068FF09F09CFFE56E3DB100221046236F616E88
:20A0C000A84794F8842019E694F8842016E684F8795070E6019009F053FFE56E019884F857
:20A0E0007800042384F88430002D3FF440AED4E91821236FA847A3E6D4F8C00047F066FB1F
:20A1000029463A20FFF7BEFC04AA8246042305A9404606920793CDE90955CDE90B550595FF
:20A120008DF820508DF834500E9549F027FFFFF7A9FBBAF1000F08D109F022FF049B1BBA64
:20A14000C3F3807384F87A305CE609F019FF09F04DFF94F88420D1E504212C20FDF7D8FF76
:20A16000032182464E20FDF7D3FF0C2183463620FDF7CEFF0BF1020B421C02FA0BF205FA53
:20A180000AF5A2FB0501420A42EAC152C4F8882009F0F6FED9E6019009F0F2FE0198042348
:20A1A000064684F88430E2E50F4BE56ED3F884306367072284F88420002D3FF4D3AD5046A7
:20A1C00095E708D0042384F8843009F0D9FE94F88420531E37E6FFF78BFB02287FF430AE4F
:20A1E0001AE600BF001F0020402F002010B4B8B10D4CD4F8183F102B05D15DF8044B05214E
:20A20000002043F087B803EB4302224482F81D1F01210B4482F81C0F82F81E1FC4F8183F7D
:20A220005DF8044B704700BF402F002080782021DCE700BF2DE9F04FDFF8ACA32DED028B98
:20A240009AF8601F002297B0CAF8502FCAF8542FCAF8582FCAF85C2FCAF84C2F19B19AF8CF
:20A26000612F8AF84C2F9AF8622F1AB19AF8632F8AF85B2F9AF8662F1AB19AF8672F8AF897
:20A28000562F9AF8642F1AB19AF8652F8AF8512F9AF8683F05935A1ED3B257B203937B1C1D
:20A2A00000F0AA80C54AC64E52F83790029602EBC70200231279019308EE102A1D463446B3
:20A2C00098462678394630464AF060FD83463046BBF1000F1ED046F033FEEA1D1321D2B268
:20A2E00020B14FF0000E827180F807E042F0C6FE20784AF07DFD4FF0070308F101022371D3
:20A300004FF0010384F802806070CDF804B05FFA82F8E3700135042D04F10504D1D118EE80
:20A32000100A029ECDF81080FFF700F9A549A64A4868024042F440324A600FB9019B5BB985
:20A34000A24C4820FFF7F2F82046022166F09AFBA26842F00102A2609A489C4A4168BAF8EF
:20A360006A4F41F400014160516821F480515160916B21F4401141F480119163D16841F473
:20A380006001D160956B85F44011C1F3015101EB81011F2000FA01FC25EA0C0C112505FA5B
:20A3A00001F141EA0C019163D16841F4E011D160956BC5F30151C1F10401C9B201EB810145
:20A3C00088404FF0100C25EA00000CFA01F108439063E4B1BAF86C1FCAF8744FA1B1BAF8BA
:20A3E0006E2FCAF8781F62B1019B7948521A90FBF2F2CAF87C2F6BB917B0BDEC028BBDE8E9
:20A40000F08F744A1288EFE7734A1188E7E7734A1488DFE74846049966F034FB684B0120C8
:20A4200003F114080723F278441CE4B252B375783279A5F10A0101EB410105EB450C092D9F
:20A4400003FA01FE03FA0CFB02FA01F140F2A080D9F80C2022EA0E0E41EA0E01C9F80C1080
:20A46000421E02EB82021F21062801FA02FC05FA02F273D8D9F8341021EA0C010A43204686
:20A48000C9F834200536B045CDD1D9F80820039942F40072C9F80820D9F8082042F4807292
:20A4A000C9F80820D9F80820574442F00102C9F8082097F9702F022043F0AAFF0446002862
:20A4C0009AD04668304643F091FF454A431E242101FB032393F89C50002D8DD1059983F8B9
:20A4E0009D10062283F89C20002885D0304643F07DFF61F099F960680AF0D0FE07A80AF092
:20A500008FFE049EA26837480792012E8CBF4FF4806300230D9309F14C034FF48072CDE953
:20A520000A56089309904FF4003360680C9507A94FF400674FF40056CDE91023CDE90E7692
:20A540000AF080FE6268136843F001031360D9F8083043F08043C9F808304DE7C11FA0F1F7
:20A560000D0201EB81014FF01F0E02EB82020C280EFA01FC0EFA02F005FA01F113D8D9F8A1
:20A58000302022EA0C0211432046C9F8301079E7D9F8101002FA0CF221EA0B0B42EA0B02F1
:20A5A000C9F810205CE7D9F82C1005FA02F221EA00010A432046C9F82C2063E7F846070804
:20A5C0008C3E002000230140E030FCFF00200140803801002E7AFF1F2C7AFF1F2A7AFF1FBC
:20A5E00088010020C03E0020402F00202DE9F0472E4C054600EB800004EBC004D4F88C7FFE
:20A600002FB10E4694F8A11F01F0FF0821B14FF000084046BDE8F0879946924643F0EEF936
:20A6200071000123C9B284F8A21F84F8A3AF84F8A53F84F8A68F84F8A43F84F8A13F84F8B7
:20A64000A08FBA88C4F8A89F91050646C4F8AC9F1CD43B88DA050FD442F20F7404E043F05A
:20A66000CDF9831BA34215DC3B889B05F7D43B889BB243F480733B80BB889BB243F4407303
:20A680004FF00108BB804046BDE8F08798464046BDE8F087064A32F8F83C01339BB2284678
:20A6A00022F8F83C65F010FDB3E700BF402F00203840002070B5464E16F8F64C04EB44032B
:20A6C00006EBC303650013F8F43C032B6ED8DFE803F059291E02254406EBC50555F8F00CE6
:20A6E000002870D116F8943C9C425FD0013404F00302934206F8F62C58D002EB420406EB97
:20A70000C404022344F8F00C04F8F43C70BD2B1906EBC30353F8F02C72B1013A43F8F02CA4
:20A72000002070BD2B1906EBC30353F8F02C002AF3D1022203F8F42C254406EBC50515F80C
:20A74000E83C013BDBB205F8E83C8BBB214B16F8946CD3F8C01255F8EC0C621C02F00302D4
:20A760004B1E0324B242034405F8F44CB3FBF1F045F8F00C1AD0994218D8013845F8F00CE2
:20A78000012070BD4AF0F8F980B1124B2C44D3F8C02206EBC404012102F51C5304F8F41C48
:20A7A0000F33B3FBF2F344F8F03C70BD012070BD084BD3F8C022012002F2E733B3FBF2F31F
:20A7C00045F8F03C70BD013845F8F00C002070BD3840002088010020054B13F8932C002A9F
:20A7E000FBD1D3F8D03A03491B6801F10C00184738400020A83F00202DE9F84F3249DFF83E
:20A80000D4B091F8351E01240229074619461046CBF82C404FF000022C4C1D4618BF7F02E3
:20A82000FDF7EEFB2A4B63626B02A362E36A40F2FF5943F093034FF400704FF48A62E362C8
:20A840000121C4F83890A0601020E2605FF024FF012D40F251434E46C4F83890CA4640F220
:20A8600052488EBF4FF0120998464FF011090A25C4F838A00121A7604846C4F80C805FF04F
:20A880000BFF03464FF0000C40F2774201213720A6632BB900231846CBF82830BDE8F88F01
:20A8A000A663C4F808C0E2605FF0F6FE013DA6630028EFD015F0FF05DAD10346CBF82C501C
:20A8C000CBF82830BDE8F88F402F0020002C014000E1F505481E00202DE9F843DFF87480B8
:20A8E00098F88450042D0446894617461E4608D0082D02D00020BDE8F883FEF759F9022859
:20A90000F8D101234A4620460021FFF775FF68B1FEF7DAF9D8F86C40002CEBD00022D8F893
:20A920007030D8F864101046A047E3E7084BC8F86090D3F88420C8F864400523C8E91B76EC
:20A94000C8F8742088F884300120BDE8F88300BF402F0020481E00202DE9F84F2F49DFF8AE
:20A96000C49091F8351E1E4602292D4B07464FF0010418BF4702012E40F259481C6398BF17
:20A980004FF48B683B469346474640F2FF55B0468CBF4FF0190A4FF0180A0A241E4640F24C
:20A9A000FF53C9F838300121C9F808605046C9F80C705FF071FE03464FF0000C40F27742C1
:20A9C00001213720C9F83850A3B9584641460122FDF716FB4646134A134B536276029662A0
:20A9E000D36A43F09103D3620D4B002108469962BDE8F88FC9F83850C9F808C0C9F80C2071
:20AA00005FF04AFE013CC9F838500028DDD014F0FF04C4D1024B1C63BDE8F88F402F002021
:20AA2000481E0020002C014000E1F5052DE9F047374C82B005460E461746984694F884005C
:20AA400004280CD0082806D1E36FAB4207D0FEF7AFF80228F2D0012002B0BDE8F087DFF883
:20AA6000B8A02666DAF82C9E6566C9F34F210F294FEA592223D8D4F880300193FBB194F830
:20AA80005201E0B1B9F5005F13D0224831464FF40072484469F026FD09F50072C2F34F21AF
:20AAA0001029CAF82C2E4FEA522202D0019B012B21D192B2013A174EAD1A0B4600E0012308
:20AAC00032462846062601250021E766C4F8708084F8685084F88460FFF73EFF0028BBD0AA
:20AAE000FEF7F2F8E66E86B12846236F616E0022B0470320B0E7E26F013B01320421C4E9B8
:20AB00001F2384F884100220A6E70320A4E700BF481E00201C710020402F002003681A7808
:20AB2000012A01D00020704793F90430044A03EB830302EBC30393F8A10FC0B2704700BFEA
:20AB4000402F0020F0B53B4CD4F8D45A2B78022B95B018D0012B02D0002015B0F0BD95F925
:20AB600004506B1CF8D0022DF6DC0091134694F8D81A0246284665F049FC0028ECD0284627
:20AB800065F0F4FCE9E72B6A002BE5D10DF10F0C8DF80F00002601200027CDE90833CDE968
:20ABA0000A12CDE90E6705938DF81C300D9310931293CDF810C006908DF830008DF8440054
:20ABC000EFF31180102383F31288D4F8D43A1B6A13B3069B04AE32461BB1D3691432002B56
:20ABE000FBD12B6A13B3996839B993420AD0196829B15B6899680029F7D01433F3E70E4A04
:20AC0000C3E90026C0B280F31188D4F8D42A136A002BFCD10120A0E704ABC0B22B6280F3DC
:20AC2000118804F6D42062F051F9EEE7024A1A60FFDE00BF384000200C4B002070B503681B
:20AC40001D78022D14D0012D01D0002070BD044693F904000A4B421C83F8A05BF5D002280E
:20AC6000F3DC0A4603F53A632179BDE87040BDE41B6A002BE9D1012249F0A6FC012070BDDA
:20AC80003840002010B50C4CD4F8D43A1B78022B10D1D4F8DC0A46F09FFDD4F8DC0A08B195
:20ACA0002123C380012142F0E9F9044849F00CFBA4F8D80A10BD00BF3840002080969800FB
:20ACC00030B583B00D46012301460DF107020446074849F0E9FD9DF8072035EA020304D02B
:20ACE00003482A43214649F075FE03B030BD00BF0C4B002038B505460A460C46064829461C
:20AD000049F062FC45F08001034849F007FB231A5842584138BD00BF0C4B002013B53A4C77
:20AD20000023D4F8B02B8DF80730137803F0FD01012905D194F8B41B11B90C2184F8B41B74
:20AD4000022B1ED0032B2ED001220B212F485DF05FFC042042F07EFE2C4801230DF10702CD
:20AD600000215DF077FC002839D09DF80730482B35D1274BC4F8A43B264BC4F8A83B02B0AD
:20AD800010BDD4F8B80B46F027FDD4F8B80B08B13523C380012142F071F91F4849F094FA2E
:20ADA000A4F8B40BD0E71D4B50681B6846F2A8111961002380F88830122237215DF0FCFB50
:20ADC000D4F8B03B0D22586824215DF0F5FBD4F8B03B302258686A215DF0EEFBB4E7D4F85A
:20ADE000B03B1A78022A03D0032A07D00020C6E7D4F8B80B48F01AFA0020C0E75868102272
:20AE000037215DF0D9FBF1E738400020E84B0020B38606083587060880969800985000202F
:20AE20002DE9F04FB64CB74E95B0002305464FF4F0728B4604F56B70202184F8A83384F8A5
:20AE4000A933019569F0AFFB202104F28C504FF4F07269F0A8FBDFF8C4C2AB4932274FF0E0
:20AE6000100E4FF47A704FF00108DCF80430C3F30803002B40F0BC80EFF31183002B40F00E
:20AE8000B780D6F884208D68D6F884309A42F8D1D6F8C83E9D42F4D8D6F8C49E00FB09F347
:20AEA0005B1BB3FBF9F300FB0232DCF80430C3F30803002B7BD1EFF31183002B77D1D6F85C
:20AEC0008430D1F808A0D6F88450AB42F7D1D6F8C85EAA45F3D8D6F8C49E00FB09F5A5EB8F
:20AEE0000A05B5FBF9F500FB03539B1AB3F57A7FDBD3013FB9D194F86D27002A52D094F88E
:20AF00006E37013B022B4DD803EB830104EBC1007E4D90F8707705EBC1014FF0010C022F73
:20AF2000C4F8E81784F870C800F0C382DBB204EB0313D3F88038C0F874379BB302234FF43F
:20AF4000807780F8703705F18803C435A0F87C77C0F88837C0F88C571509013D052D02F044
:20AF60000F0200F289826A4F07EB4503B3F8840040FA02F3DB0740F17F82012303FA02F249
:20AF8000013A10403D4466F07BFD95F89020614B104403EBC000C4F8F0078379002B47D0FB
:20AFA000412B45D06FF0010015B0BDE8F08FEFF311898EF31288D1F808A00B68DD0344BF69
:20AFC000C6F8C08ED1F808A0D6F88430D6F8C05E5FFA89F989F31188D6F8C49E2B4400FBFC
:20AFE00009F5A5EB0A05B5FBF9F500FB03537CE7EFF311858EF31288D1F808900B68DB031D
:20B0000044BFC6F8C08ED1F80890D6F88430D6F8C02EEDB285F31188D6F8C45E1A4400FB89
:20B0200005F3A3EB0903B3FBF5F300FB02323CE72323C380092141F045FED4F8F037002B51
:20B0400000F065821A68D4F8E8179B881383D6F8BC24314BB3EB920F80F03182B3EBD20F08
:20B0600080F02F82B3EB121F80F02F82B3EB521F80F02F82B3EB921F80F02F82B3EBD21F90
:20B0800080F02F82B3EB122F80F02D824FF480720023FF200DF10F08A4F8EC270122CDE97D
:20B0A0000483CDE90833CDE90A338DF80F000D9306928DF81C208DF83020EFF3118010231D
:20B0C00083F31288D4F8E8371B6A002B00F0D881069B04AD2A461BB1D3691432002BFBD175
:20B0E0000B6A002B00F01C82996839B99A421AD01968A9B15B6899680029F7D01433F3E7B9
:20B1000030510020402F002010E000E0A058002048460708FC300020404B4C0000ED00E08A
:20B12000B74AC3E90025C0B280F31188D4F8E8170B6A002BFCD18C220120CDE908330DF1C9
:20B140000E0A05938DF81C300D93109312938DF80E2000230022CDE90E23CDF82880CDF875
:20B1600010A006900B908DF830008DF84400EFF31180102383F31288D4F8E8371B6A002B1F
:20B1800000F08781069B2A461BB1D3691432002BFBD10B6A002B00F0C381996839B99A42BE
:20B1A0000AD0196829B15B6899680029F7D01433F3E7934AC3E90025C0B280F31188D4F88D
:20B1C000E827136A002BFCD19DF80F301B2B40F09081D4F8F037012284F8A8230BB1232232
:20B1E000DA80DFF81C92402248460A2149F0ECF98A21002301228DF80E1000200021CDE9AC
:20B200000E01CDE90833D4F8E817CDF810A0CDF8288005938DF81C300D9310931293069298
:20B220000B928DF830208DF84420EFF31180102383F31288D4F8E8371B6A002B00F03181C0
:20B24000069B2A461BB1D3691432002BFBD10B6A002B00F06281996839B99A4209D01968FC
:20B2600029B15B6899680029F7D01433F3E7C3E90095C0B280F31188D4F8E827136A002BDD
:20B28000FCD19DF80F2094F86C17C2F3801284F8B028002900F0D480022900F0B980D6F8E4
:20B2A000BC345849B1EB930F80F01F81B1EBD30F80F00981B1EB131F80F00981B1EB531F61
:20B2C00080F00981B1EB931F80F00981B1EBD31F80F00D81B1EB132F34BF4FF480768026F0
:20B2E00094F8B418A4F8B268182914D1464F474800215B08B3FBF6F3A7FB03730F465B0B08
:20B3000066F30F076BF30F0163F31F4762F31F41C4F8B81847603A48A4F8EC6702220021F6
:20B3200049F052F9C82042F03DF9D4F8E8074FF0800B0026002700230122CDE90E67CDE940
:20B3400008338DF80EB0CDF810A0CDF8288005938DF81C300D931093129306920B928DF882
:20B3600030208DF84420EFF31182102383F31288D4F8E8371B6A002B38D0069B002B3DD060
:20B380002B46D96914330029FBD1006A002800F0C180816839B9834209D0016829B1406897
:20B3A00081680029F7D01430F3E7C0E90095D2B282F31188D4F8E807036A002BFCD19DF811
:20B3C0000F3013F00203B6D1019841788278007884F8C008C1F12001C2F11002184684F825
:20B3E000C11884F8C22815B0BDE8F08F0562D2B282F31188024861F069FDDBE72B46C4E74D
:20B4000018590020809698005917B7D1E8590020D6F8BC344448B0EB930F73D2B0EBD30F4B
:20B4200051D2B0EB131F52D2B0EB531F53D2B0EB931F54D2B0EBD31F34BF802640264FE791
:20B44000D6F8BC343949B1EB930F4ED2B1EBD30F39D2B1EB131F3AD2B1EB531F3BD2B1EB34
:20B46000931F3CD2B1EBD31F41D2B1EB132F34BF4FF48076802633E70023C4F8F037E6E5D0
:20B4800004ADC0B20D6280F31188294861F01EFD4CE60D62C0B280F31188254861F016FD41
:20B4A0008DE60D62C0B280F31188484661F00EFDE2E690F87D37634480F87D374CE5022216
:20B4C000E6E50422E4E504260AE70822E0E5082606E71022DCE5102602E72022D8E5202636
:20B4E000FEE64022D4E58022D2E50226F8E64026F6E6D4F8F00738B1202141F0E3FB4FF071
:20B50000FF3051E50E46EBE64FF0FF304CE5D4F8E8179CE5C0F80090FFDEC3F80090FFDE69
:20B52000034A1A60FFDE00BF002D3101404B4C00185900200146014848F0F0BEF4590020FE
:20B54000014488420ED010B40346074C074813F8012B04FB00F0994280EA0200F7D15DF8C5
:20B56000044B70470148704793010001C59D1C81094B93F82E31042B08D9053B032B08D895
:20B5800001231A4600B103701046704700230122F8E700231A46F5E7402F0020F0B40D68CA
:20B5A00000240CE0BCF1050F18D8A0F137030A2B14D104EB840415F8010B03EB4404A0F18E
:20B5C0003003DEB2092EA0F16107A0F1410CF0D9052FE7D8A0F157030A2BEAD00D60146023
:20B5E000F0BC70479FED727A07EE901A20EE070AF8EE677A27EE800AFDEEC07A17EE903A58
:20B600002033402B00F2C480DFED6A7AB4EEE70AF1EE10FAF0EE407A0CDD9FED676ADFED60
:20B62000676AB0EE677AB4EEE67AF1EE10FA77EEC67AF6DC9FED627AF4EEC77AF1EE10FAE4
:20B640000CD59FED5D6ADFED5F6AB0EE677AB4EEE67AF1EE10FA77EE867AF6D49FED5A7A28
:20B66000F4EEC77AF1EE10FA00F38A809FED577AF4EEC77AF1EE10FA44BF9FED517A77EE99
:20B68000677A27EEA76ADFED525A9FED527ADFED526AA6EE257A67EE865AE6EE076AB6EEFA
:20B6A000007AE5EEA67A27EE877ADFED476A70EE267ABDEEE76A16EE103A2033402B64D848
:20B6C000B4EEE60AF1EE10FA0CDDDFED3B5A9FED3B6AF0EE676AF4EEC66AF1EE10FA77EE65
:20B6E000E57AF6DCDFED366AF4EEE67AF1EE10FA0CD5DFED315A9FED336AF0EE676AF4EE90
:20B70000C66AF1EE10FA77EEA57AF6D4DFED2E6AF4EEE67AF1EE10FA3DDDDFED266A76EE59
:20B72000E77A67EEA75A9FED2A5A9FED2A6ADFED2A6AA5EE856A27EEA55AE5EE866AB8EEC3
:20B74000006AE5EE267A67EE867AC7EE206AB7EE006A76EE865A76EE666A86EE257A80ED71
:20B76000091A67EE277A66EE876AC0ED017AC0ED037A80ED007A80ED027AC0ED046A704777
:20B780009FED0C7A77EE677A7BE7DFED147ADCE79FED127A89E7DFED0D6AF4EEE67AF1EEE6
:20B7A00010FA44BFDFED066A76EEE77AB9E700BF27D4D236DB0F4940DB0FC940E4CB1641AD
:20B7C000DB0F49C0E4CB16C1DB0FC93FDB0FC9BF92E741B99730083C15A82ABE0000000069
:20B7E0002DE9F843E14FDFF8E4E3D7ED3E7A2DED028BF8EE670A9EF85C4907F26C63C3EDFD
:20B80000000A002C6FD1DFF8C8C397F87866C7F874469CF80040002E39D0BEF862399FED82
:20B82000D46A9FEDD47A07EE903AF8EE677A20EE877AC6EE276AD04B0022012E1A6076EECC
:20B84000876AC7EE267AC3ED017A20D0022E9A60C3ED037A1BD0032E1A61C3ED057A16D084
:20B86000042E9A61C3ED077A11D0052E1A62C3ED097A0CD0062E9A62C3ED0B7A07D0072E5A
:20B880001A63C3ED0D7A02D09A63C3ED0F7ABB4B9FEDBB6A93F84E319FEDBA7A9FEDBA0A1B
:20B8A000BA4A07EE903AF8EEE77A9CF8583BC6EE276A1C4414FB06F6F6B207EE906A60EEC2
:20B8C000870AF8EEE77AC2ED006AA7EEA00A67F0E3FBBDEC028BFCEEC07A17EE903A87F85B
:20B8E000C837BDE8F883BCEEE06A9FEDA97A9EF85D39BEF860299FEDA72ADFEDA76ADFF80A
:20B90000D0C297F87866C7F874C6F8EE465A07EE903A87EE255A8CF8004007EE102ABEF84D
:20B920005E298CED025A16EE103AF8EE677A06EE102AB8EEC77A27EE822AB8EE466A67EE15
:20B94000266ACCF81430012322EE252ACCED017A8CED036ACCED046A87F87036002E96D0D2
:20B96000DFED8E7A9FED8E4ADFED8E5AC7EE871AC6EB0615A6EB06190CEBC5054FEAC9093D
:20B980004FF00008B1EE611A9FED876A09EB05009FED863ADFED863ADFED866A03460022D1
:20B9A00007EE902AB8EEE77A27EE027AFDEEC77A17EE901A2031402900F2D080B4EEC47A89
:20B9C000F1EE10FAF0EE477A0CDDDFED7B4A9FED7B5AF0EE672AF4EEC52AF1EE10FA77EE76
:20B9E000E47AF6DCF4EEE57AF1EE10FA0CD5DFED724A9FED735AF0EE672AF4EEC52AF1EE0C
:20BA000010FA77EEA47AF6D4F4EEC67AF1EE10FA40F39A8074EE677A27EEA75AB0EE630A13
:20BA2000A5EE030ADFED674AE5EE004A65EE272AB7EE005AE2EEA47AB0EE458AF0EE454A61
:20BA4000A1EEA78AE1EE274AC5EE088A84EE880A77EE067ABDEEE75A15EE101A20314029E5
:20BA60006FD8B4EEC67AF1EE10FA0CDD9FED525A9FED527AF0EE674AF4EEC74AF1EE10FAD0
:20BA800077EEC57AF6DCF4EEE57AF1EE10FA0CD59FED495A9FED4A7AF0EE674AF4EEC74A24
:20BAA000F1EE10FA77EE857AF6D4F4EEC67AF1EE10FA3CDD74EE677A27EEA75AF0EE632A87
:20BAC000E5EE032A9FED3F7AA5EE227A65EE274AB8EE005AE4EE877A67EE857A87EE887A90
:20BAE0000132A24203F1280343ED048A03ED037A03ED017A43ED028A83ED000AC3ED056A25
:20BB0000C3ED026AC3ED016AC3ED046AC3ED036AFFF646AF783085427FF43AAF08F5707819
:20BB2000B8F5346F05F570757FF42EAF75E69FED267AF4EEC77AF1EE10FA48BF75EEE77A28
:20BB4000BAE7F0EE667AC9E79FED1F5AF4EEC57AF1EE10FA48BF75EEE77A5DE7B7EE000A09
:20BB6000F0EE408AB0EE408A72E700BF0800001083F9223EBD378635945A0020402F00205D
:20BB8000555555406E12833A48E1FA3ECC0700100060EA4827D4D2360AD7233C0000484286
:20BBA000DB0F4940DB0F49C0DB0FC93F92E741B99730083C00000000DB0FC940E4CB1641B6
:20BBC000E4CB16C115A82ABEDB0FC9BF305100204C1800102DE9F04F07EE900A2DED068B24
:20BBE0009FEDF07AF04BDFEDF16AB3F8A429F04F93F8AA59C7F81C08B8EE679A0AEE102AEC
:20BC000087EE095AB3F8A629C7F8D85783B008EE102AB3F8A829DFEDE77AB8EE4AAA08EE48
:20BC2000902AB8EEC88A3AEE0A7AF8EEE88AB4EEC78AF1EE10FA68EEA77AB4EEE65A07F220
:20BC4000CC73B8BFB0EE478A0022F1EE10FA83ED028A83ED01AAC3ED007AC7F8DC2700F1C0
:20BC6000038307EE905AF8EEE77AB7EE007AC7EE279AD14BDFF878A3194614319C4601915D
:20BC80009AF8982003F12C04F6EE005A65EE256AF7EE007A86EE887ADFEDC83ADFEDC84A95
:20BCA0009FEDC86AD3ED05AAB4EEE77AF1EE10FAB8BFB0EE677ABDEEC77AB0EE004A17EE9C
:20BCC000106AB8EEC77AC7F8786AC5EE076A87EE875A66EEA36AACEC015A8AEE267AC8EEC6
:20BCE000267A37EE257A77EEA57AB4EEC47AF1EE10FAB8BFB0EE447AF4EEE47AF1EE10FA97
:20BD0000BDEEC77A88BFF0EE647A17EE100AFDEEE77A00F1FF3B17EE901ABBF1230FA8BFAA
:20BD20004FF0230BCCED006A012E01F1010CB8BF0126BCF1230F2BEAEB7BE04629EE066AA0
:20BD4000A8BF4FF02308E345C8BFD846C7F8840AC7F8881A83ED046AA8EB0B0797FBF6F795
:20BD60000137002A40F0E380DFED970ADFEDA15A9FEDA12A9FED955ADFEDA32A9FEDA33AC6
:20BD8000DFEDA33A9FED924ADFEDA21A0AF19C0107EE902AB8EEE76A66EE207A37EEA57A9A
:20BDA000FDEEC76A16EE903A2033402B00F21582F3EE026AB4EEE66AF1EE10FA0CDDDFED75
:20BDC000904ADFED8E6AB0EE471AB4EEE61AF1EE10FA37EE647AF6DCB4EEC57AF1EE10FA9C
:20BDE0000CD5DFED874ADFED876AB0EE471AB4EEE61AF1EE10FA37EE247AF6D4B4EEE57AF0
:20BE0000F1EE10FA40F3FE81DFED726A36EEC77A67EE076AB0EE431AA6EEA21AB0EE630A5E
:20BE2000A1EE260A67EE264AFDEEE76AA4EE807A16EE903A2033402B27EE047A00F2D7814D
:20BE4000DFED656AB4EEE66AF1EE10FA40F300829FED6B0A9FED691AF0EE676AF0EE664A6A
:20BE6000F4EEC14AF1EE10FA76EEC06AF6DC9FED591AF4EEC14AF1EE10FA13D59FED601AC9
:20BE8000DFED604AB0EE660AB4EEE40AF1EE10FA76EE816AF6D4DFED506AB4EEE66AF1EE35
:20BEA00010FA0CDD9FED566ADFED546AF0EE674AF4EEE64AF1EE10FA77EEC67AF6DCF4EED6
:20BEC000C57AF1EE10FA0CD59FED4D6ADFED4D6AF0EE674AF4EEE64AF1EE10FA77EE867AA4
:20BEE000F6D4F4EEE57AF1EE10FA40F38381DFED396A76EEE77A67EEA76AF0EE434AE6EE3E
:20BF0000A24AB0EE631AA4EEA61A27EEA66AE6EE017A67EE847A0132242A81ED007AC1EDEA
:20BF2000017A01F108017FF433AFDFED2CAA4FF0000944E9059B44E902764FF49072002174
:20BF4000204644F80C8C68F02EFB4FF49072A018002168F028FB224B04F51574A342E8D100
:20BF6000019BDFED207AC3ED00AA012329EE279A8AF89830002D00F02B81DFED1B7A1B4E8C
:20BF80009FED142ADFED112AC7EEA81AA6F1140406F5117738EE4A8AB1EE611A69EE889A9A
:20BFA0003EE000BF00247449305100200000FA44080000100AD7233C840A0010398E633C88
:20BFC00000000C429C534937C3B8B23DDB0F49C072F97F3FDB0F494000001042BC297E3FB7
:20BFE000AC11001027D4D23600004842E807001000110010DB0FC93F00000000E4CB1641CF
:020000040800F2
:20C00000DB0FC940E4CB16C192E741B99730083C15A82ABEDB0FC9BF000010C20000807F41
:20C020005FED0C5A5FED0C6A234630460022B7EE005A07EE902AF8EEE77AB6EE007A77EE13
:20C04000877AB0EE4A7AA7EEA97AF0EE477A29EE077AE0EC017AFDEEC77A17EE901A20311B
:20C06000402900F2D780B4EEC27AF1EE10FAF0EE477A0CDD1FED1E4A5FED204AB0EE676A26
:20C08000B4EEE46AF1EE10FA77EEC47AF6DCF4EEE27AF1EE10FA0CD51FED274A5FED274A10
:20C0A000B0EE676AB4EEE46AF1EE10FA77EE847AF6D4F4EEE57AF1EE10FA40F3B58072EE19
:20C0C000677A67EEA74A5FED303A1FED304A1FED306AA4EEA34A67EEA43AA4EE246AF0EEA7
:20C0E000454AE3EE867AB0EE456AE1EE274AA1EEA76A84EE864AC5EE064A77EE257AFDEE7F
:20C10000E73A13EE901A2031402900F28A80B4EEE57AF1EE10FA0CDD1FED473A5FED493A6E
:20C12000B0EE677AB4EEE37AF1EE10FA77EEC37AF6DCF4EEE27AF1EE10FA0CD51FED503A86
:20C140005FED503AB0EE677AB4EEE37AF1EE10FA77EE837AF6D4F4EEE57AF1EE10FA6DDD02
:20C1600072EE677A27EEA73A5FED590A5FED593A1FED597AE3EE203A63EE270AA3EE237A40
:20C18000F8EE003AE0EE877A67EEA37A87EE867A0132AA4203F12803C3ED0B4A83ED0C7A90
:20C1A00083ED0E7AC3ED0D4A83ED0F4A83ED145AC3ED116AC3ED106AC3ED136AC3ED126A2B
:20C1C0007FF437AFC834A74206F114067FF428AF03B0BDEC068BBDE8F08FFDEEE76AB0EEDB
:20C1E000427A16EE903A2033402B7FF629AEF0EE427A90E6F4EEE17AF1EE10FA48BF75EE0B
:20C20000677A78E6B4EEE17AF1EE10FA48BF35EE477AFDE5B7EE004AF0EE444AB0EE446A85
:20C220006BE7F0EE667AB1E71FED866AF4EEC67AF1EE10FA48BF72EEE77A42E71FED8B7A4D
:20C24000F4EEC77AF1EE10FA48BF72EEE77A89E75FED8F6AB4EEE66AF1EE10FA48BFF0EE95
:20C26000676A3FF50BAE2AE65FED949AC7F8D8271546FEE40848002302461178022902F119
:20C28000060204D00133062BF7D10020704703EB430300EB43007047801E002000B5002111
:20C2A000084B83B00846C3F8AC1934F00DF80422054B01930DEB0201062033F0F9FF03B008
:20C2C0005DF804FB305100205475C52A70B5461E00F13105344614F8011F601E801BFF291A
:20C2E000C0B201D033F0F0FFAC42F4D1A02056F0A3FB0121022033F0E7FF40F2E93401E015
:20C30000013C04D04220FFF715F90028F8D16220FFF710F91321242033F0D6FF2520092155
:20C3200033F0D2FFBDE87040A02056F085BB00BF0D4B0E49D3F8BC340A8810B40C4C5B0834
:20C34000A4FB034322F45C729B0C01381204013B012480B2120C9BB20A80C8620B858C82CE
:20C360005DF8044B704700BF402F0020000C004083DE1B4338B50C4C0546A11CD52254F081
:20C3800049FC2B68A342C5E90043A3EB04000AD004F14002611C2960237802F8013BD5E9B7
:20C3A0000041A142F6D138BDE05A002010B5204B84B0C82403F51F6103F6B1122128CDE9C0
:20C3C000022183F8B04918D00CD802281ED0082825D102A801900AF0EDFE0198FFF7CAFF44
:20C3E00004B010BD29281AD102A801900AF09CFD0198FFF7BFFF04B010BD02A801900AF0AF
:20C40000DDFD0198FFF7B6FF04B010BD02A801900AF01CFF0198FFF7ADFF04B010BD02A8C7
:20C4200001900AF03DFE0198FFF7A4FF04B010BD3051002010B582B00A788DF80720040AAF
:20C4400018238DF804308DF806008DF8054056F081F901AA03481146042348F055F902B027
:20C4600010BD00BFF459002010B582B0040A192200238DF801408DF800200C468DF80330EB
:20C480008DF8020056F066F96A4605481146052348F03AF99DF80430237002B010BD00BFEF
:20C4A000F459002010B58CB000234CF20502044601A9CDE90633CDE90833ADF800208DF888
:20C4C000023003220B930123CDE903128DF814308DF82830CDF808D048F05CF9204602A997
:20C4E00047F04CFD204648F055F99DF806000CB010BD00BF2DE9F043764D774F83B005F1F2
:20C5000038002422002168F04EF897F8314A0023EB65002C39D1714ED6F8F83053B39B6A6B
:20C5200043B36F489847836823B303886D4F013B9BB2BC46384600210678032E00F1060097
:20C540001CD001310629F7D100223978022907F1060700F09E800132062AF6D1E96D052907
:20C5600008D0481C02FB01C2E86502200021938010705180204603B0BDE8F083062303FB73
:20C5800001514B8F013B9BB2DEE797F8300A07F63823C7F8343A10B9504E0024BCE744F071
:20C5A000CFFCC7F8400A18B183790BB1412BF3D121464D4847F052FE04460028ECD0D7F876
:20C5C000343A474A9868C3F8942008B12023C380092140F053FDD7F8343A404E986845F004
:20C5E000FBF84248D7F8348A47F06EFE4FF00109A8F804003220C6F8188186F81C9141F09C
:20C6000029FA0423D7F8340A4FF0000C0DEB03029F21CDF804C047F083FF9DF805809DF8CA
:20C6200004309DF806104FEA082848EA034848EA0108414606F1F80055F0CCFC00287FF4DC
:20C640006BAF4046FBF792FF034600287FF464AF9DF806009DF805209DF80710000240EA93
:20C660000240234A0843904217D0C6E94033A6F8FC30A6F80831FBF779FF804600287FF479
:20C680004BAF97F8300A44F05BFC46F0CFFD444642E7062101FB02C267E7164AC6F8FC2028
:20C6A0004FF400334FF00062C6F800314023A6F80831C6F8042186F80A91FBF701FD06F157
:20C6C000F80086F8119155F0D1FB0B4BC6F8F83022E700BF481E002030510020402F002077
:20C6E00038300020801E0020685B0020404B4C0021AAEF0000040008484607082DE9F04190
:20C70000C94BCA4ECA4DCB4C0822C3F88820336B82B043F00103336307464FF4C052284685
:20C7200040F2023388466946CDE9002308F058FF6B6AC14ADFF848C323F470436B626B6ABF
:20C7400043F420436B626B6A23F470236B626B6A43F420236B62736CB84D43F4804341F2F9
:20C76000B4017364736B44F8018041F2BC0143F08003675041F2B80EB14973630227C4F887
:20C78000D41AB04EB04BB14944F80E5084F8D87A4FF0A045AE4FC4F8DC5AC4F8E06AC4F87B
:20C7A000E83AC4F8241B05F5326506F5A07603F51073A1F5D071C4F8EC7AC4F8285BC4F84B
:20C7C000F06AC4F82C3BC4F8F41A012307F51077A5F5E465A6F5A066A1F58C61C4F8D0CA0E
:20C7E000C4F8307BC4F8E45AC4F89C6B84F8DB3A05F5A075536106F5B076C4F8601B84F8ED
:20C80000E23B1946934B944AC4F8685BA7F5BC67A035C4F8746B914EC4F8707BC4F8783B3D
:20C8200007F5D45703F56953C4F87C5B4FF050250020DFF850E2DFF850C2C4F8A02BC4F881
:20C84000A47B02F5A04207F5A047C4F8A86BC4F8AC3B06F5A046A3F54853C4F8B05B04F5B7
:20C860002D65C4F8B42BC4F8BC6BC4F8DC3BC4F864EBC4F86CCB0246C4F8B87B2B4684F8B3
:20C88000E40B402683F81C21A3F822210132042AC3E9496083F81D1183F81F01C3F83001C7
:20C8A00003F12803EED1002211462B46402083F87423A3F87A230132042AC3E9DF0183F89E
:20C8C000751383F87713C3F8881303F12803EED14FF0A04362489A6822F001029A60DA6878
:20C8E00042F04002DA6007F001FF94F8D93A0022212161F317420BB142F4801294F8D31AE6
:20C90000D4F8DC3A01299A6300F0E380DA68D4F8DC6BD4F8E00AC2F3076121F0600141F0F0
:20C92000400161F31F620021DA603160026861F3CC22026094F8DB2A012A00F0B7801021D3
:20C94000484808F025FA474808F008FAD4F8E00A94F8D13A00224FF0FF31026142618161E1
:20C96000C26153B305F114073F4E114607EB83074FEA830C4FF0FF0E56F8042F1368002BE2
:20C98000ACBF00234FF09043B74213601161C2F808E0F1D105F15003344963440027FF26FC
:20C9A00051F8042F1568002DACBF00254FF090459942156017619660F2D1036994F8D31A47
:20C9C00043F480730129036160D0D4F8DC2A28480023936100294FF0FF336FF080415161AA
:20C9E0005360516114BF00231023906143F47013916943F4605343F008030B43936141F267
:20CA0000B8019368615843F0010393600B689847184B194ADA606846184B009308F096FB00
:20CA200002B0BDE8F08100BF00E100E0003802400000024030510020003C01404C04002064
:20CA4000400040010008005000090050000B005020090050C00500500010005000300050DB
:20CA60000C5C0020005C0020145C0020505C00200008008000ED00E00005FA0543020001B7
:20CA8000080401002005005060050050D4F8DC2A144B03636FF08041134D00234FF0FF30B7
:20CAA000936151615060516195619FE701680F4A0F4E41F003010160802159629E62C3F826
:20CAC0000421E022C3F80821C0F24002C3F80C2135E79A6822F03E0141F02A0161F3070247
:20CAE0009A6013E70301810000080080A00040008000200010B51A4C14F8330CC0B9194B62
:20CB000083F8B100C3F8B40014F8303C012B05D0022B21D054F82C3C1BB910BD124B44F8F5
:20CB20002C3C12495B68BDE81040A1F10C00184744F006FA14F8312C0A49003A18BF012259
:20CB400081F8B120C1F8B4000028DDD01F22C280202140F093FAD7E7054B44F82C3CE0E74F
:20CB600028620020481E00208C040020006200206804002091B10A6B824214D9144B5A693D
:20CB8000914220D34C3991421DD30B6B9842F9D38B6B9842F6D80B46184670470C4B59694E
:20CBA0000A6B904212D30B680BB9F5E70A6B90420B4602D38A6B9042EED951F84C3F002B3C
:20CBC000F4D1184670470023184670470A46D9E7286200202DE9F047CC0143D10346224AA6
:20CBE00043F8082B4FF0FF324260022418467E26DFF87880D8F818902644013E051D4946EC
:20CC00006FF070474FF0010A08E0A3421CD0631C45F8043C321B1C460435CAB10B6BA34241
:20CC200002D88B6BA34204D22046FFF7A3FF014690B10A794B6B002AE7D1A34204D0E6D257
:20CC400045F8042C631CE5E745F8047C631CE1E7C8F81810BDE8F08745F804AC321B631C5B
:20CC60004946D8E78026C3E7F8FFFF0F2862002070B4447941BB03684FF400524FF40076D1
:20CC8000202502213CBB1A8C22F001021204120C1A841A8B188C22F0F30280B2120420F000
:20CCA0000A00120C014342F0010241F001011A8319841A8B22F00C021204120C1A831A8B2B
:20CCC00092B270BC1A83704700220368164615461146002CD7D0042C21D0082C38D0198C20
:20CCE00021F480510904090C19849C8B1D8C45F6FF7040F6FF4128402140024342F4805289
:20CD000041F4807199831A849A8B22F440621204120C9A839A8B92B270BC9A8370471A8CF6
:20CD200022F010021204120C1A84188B198C89B240F6FF4221F0A00102400D4342F4807297
:20CD400045F010051A831D841A8B22F44062B3E71A8C22F480721204120C1A84998B1A8C0A
:20CD600021F0F30192B2090422F42062090C324342F4807241F0010199831A849A8B22F0EF
:20CD80000C02C4E738B50E4D0446006808F02CFBD5F8BC24204652084FF6FF713FF0E4FA92
:20CDA00020460021FFF764FF064BC5F8283D05F6285120460022BDE838403FF019BA00BF46
:20CDC000402F0020B9130208036870B55E6A26B133460522BDE87040184704460D464E1D63
:20CDE00000E023689B68204698470028F9D0236815F8011B1B6820469847B542F1D170BD2D
:20CE0000036870B55E6A26B133460822BDE87040184704460D4601F1080600E023689B6881
:20CE2000204698470028F9D0236815F8011B1B6820469847B542F1D170BD00BF0A4491427A
:20CE400017D010B40139541E11F8013F08225840430010F0800F08BF400083F0D50314BF79
:20CE6000D8B2C0B2013AF3D1A142EDD15DF8044B704770472DE9F047164D0746002095F959
:20CE8000259005F12C0684B007EB010805F5337504464FF0B60A3368ABB193F83830142B72
:20CEA00011D019F1020F01D04B450CD1002269463046CDE90244CDE90078ADF808A08DF8F5
:20CEC0000D4034F00DFEE036B542E4D104B0BDE8F08700BF286200202DE9F0479AB0DDE97E
:20CEE000226ADDF8909004460D461746984602E0206841F0EBFA206841F0F0FA0028F7D1C6
:20CF00000146642201A867F04EFB264B8DF80450CDF85CA00293002D40D0AB1E012B3FD911
:20CF2000042D14BF002203221F4B0396D3F884308DF805201E440123CDE9059404968DF886
:20CF40005B3037B14246394607A867F0CBFA8DF85A80164E96F80E9300231893B9F1000F13
:20CF600019D196F80D03642202FB006001A900F5447067F0B7FA012386F80D9386F80E33EA
:20CF8000236843B143463A46294620461AB0BDE8F04712F045B81AB0BDE8F0870522C3E7D8
:20CFA0000222C1E7F4640020402F0020286200200C480D4BD0F8901310B40C4CC0F8803356
:20CFC0008A1E2231B0F8AE331B01A4FB03C3DB08A3F5B06322F8023F9142F3D15DF8044B28
:20CFE000704700BF28620020B97E0208CDCCCCCC70B5084C251D2E4614F8010B37F060FAD7
:20D0000028B1037805F8013BB442F5D170BDFF23F8E700BFFC6500202DE9F0471D4F012679
:20D0200007F10805B2464FF03C094FF0000817F8010B43F085FF044690B180F80690C67186
:20D04000FB7803F07F02012A18D013F0800F20460DD185F8048044F0B9FB85F805802C6089
:20D060000136052E05F10805E1D1BDE8F08785F804A044F0B1FB85F805A0F0E71B0605D481
:20D08000012120463FF0FAFFFB78DEE744F0A4FBF6E700BF046600202DE9F04FDFF8FC91F6
:20D0A000DFF8FCA183B009F10C06012419F8018BB8F1000F00F0C6804FEA1815013D052D37
:20D0C00008F00F0200F2C1800AEB4503B3F8840040FA02F717F0010700F0D280012393402D
:20D0E000013B1840554464F0CBFC95F89030664F184407EBC00704237761FC71BB71002316
:20D1000002E0152B00F09E8003EB43025F49895C41454FEA430B03F10103F2D15C4B1A4452
:20D1200092F85111002900F0AD8040463FF068FB054628463FF084FB0378002B40F0828066
:20D14000534B5B44042283F8914183F89021002D78D0002F5DD03B68287A03F13F4202F571
:20D160007E020AEB92224FF0010C92F8982002F01F015209032A0CFA01F171D0042A67D0C0
:20D18000022A75D0B7F804E0BEFA8EF2C2F11F02C2F3CC0103EB810102F007020F6A920087
:20D1A0004FF00F0C0CFA02FC27EA0C070F620F6A90403843002208624FF0010B11460BFA85
:20D1C00001FC3CEA0E0001F101011ED118680327974020EA07001860D3F8008002209040F4
:20D1E00040EA08001860986820EA0700986098689860586820EA0C00586058685860D8683E
:20D2000020EA0700D860D868D860102902F10202D5D1204B204AB3F80414B3F80634009169
:20D22000002001340190B2FBF3F330469BB22946E4B233F073F80123092C737406F11806CA
:20D240007FF434AF03B0BDE8F08F0027776156E7DFF850C0DCF830200A43CCF8302091E781
:20D26000DFF840C0DCF840201143CCF8401089E7DFF830C0DCF844201143CCF8441081E7F8
:20D2800077613CE70D4654E7FC30002090300020402F00202862002040420F003066002059
:20D2A000484607080038024070B5044684B04FF4004039F08DF880B300234FF4E1310325B0
:20D2C00090F904000293CDE900151A464FF4004139F0DBF8124BC3F8D404F0B1012C40F68D
:20D2E000980208BF4FF496620E480F4DA3F8E0244FF461710D4AC3F8EC040A2683F8D84463
:20D30000C3F8DC64A3F8E214A3F8E414C3F8E854C3F8F024012004B070BD0020FBE700BF65
:20D32000286200205514020879FF01086DFF01082DE9F041214E224F96F8133587F8903E90
:20D3400006F5A26607F6946500244FF0050816F8010B20BB28600134032C05F10405F6D1BD
:20D3600097F8901ED7F8940EC94301F0010144F039FA97F8901ED7F8980E81F00201C1F3BF
:20D38000400144F02FFA97F8901ED7F89C0E81F00401BDE8F041C1F3800144F023BA43F074
:20D3A000CFFD013401212860E3B210B180F80680C37128683FF062FECEE700BF28620020FD
:20D3C000402F00202DE9F0412A4C2B4DB4F81865A5F8A06E82B0EEB994F8140543F0B0FD57
:20D3E00094F81525C5F8A40E003A18BF012285F8A22E48B194F816152B22002914BF11214C
:20D400000121C2803FF03AFE002002B0BDE8F04145F044BC94F81485002240462B213FF01C
:20D4200045FA0746404643F08BFDF8B1F7B12B22C5F8BC0EC280397AFCF796F84FF000083D
:20D440000E4AB2FBF6F3C3F34F0000909BB23946CDF8048005F6A860A4F81A6532F05EFF97
:20D46000D5F8A83EC3F8008085F8B98E02B0BDE8F08100BF28620020402F002040420F00A9
:20D480002DE9F84F254C94F8283584F81C3504F21F57002604F23C545FFA86FB0BF1010811
:20D4A0005FFA88F8012117F8010F42460E448A463FF0FCF94FF00009054640B3387804F852
:20D4C0000E9C04F80D9C04F80FBC04F810AC44F8045C43F035FD18B180F806A080F8078097
:20D4E000297AFCF741F80E4A002128463EF03CFF0C4B23600C4B221D21462846C4E90139E1
:20D500003EF076FE697928684A4632F083FE082E04F11C04C0D1BDE8F88F00BF2862002053
:20D5200040420F004D020408FDC4030870B52C4C2C4B94F85406C4F84C3600220221C4F8FA
:20D540000C26C4F81026C4F81426C4F84826A4F850263FF0ABF9002841D0234B0668054642
:20D5600003F1C0015A7C12B15A6896422BD018338B42F7D1002394F85406C4F8385584F81A
:20D580002C3543F0DDFC08B10223C380297AFBF7EBFF2846154A00213EF0E6FE144A1549C2
:20D5A000C4F83C150026111F2846134BC4F84035C4F844653EF01CFE697928683246BDE8CF
:20D5C000704032F027BE30465DF04AFD328D0B4992B2531CB0FBF3F081F82803CAE770BDB4
:20D5E0002862002000FFFF003C00001040420F006867002025C50308C1C603088801002087
:20D600002DE9F04FC04F87B00B460446C022BF480393002166F0C7FF97F855368BB9BC4DB1
:20D62000D5F82432002B7ED00022039883F82C00012183F82D101A6383F82E2007B0BDE86E
:20D64000F08F97F85636002B7CD0DFF8D88298F83C31012B00F0A180022B00F08180AD4E35
:20D66000AB4D98F832C198F82E710FCE05F5F87404940FC40FCE0FC496E80700BCF100066A
:20D6800018BF0126A44B85F82862072F84E80700C5F8083200F21881042F00F25581DFF899
:20D6A0006CA2DFF88CB20026039BB3424FF0030137DD1BF8019B08EB090309F1010793F8FC
:20D6C0003341FFB220463A463FF0F0F8034620461C46002B00F0108143F032FCCAF8140034
:20D6E00018B14FF003038371C77198F82F2198F82E31F1B2002A00F0FD80E27982F0010217
:20D70000009220464A4601365EF046FA002800F0F3804FF00103082E8AF811300AF1180AD8
:20D72000C2D1049B9EE07D4E7D4C0FCE0FC40FCE0FC496E80700A4F1200384E80700C5F8D8
:20D7400024327BE7774B039993F83021704D003A204618BF0122FAF7ABFFC5F824025FE7BC
:20D7600098F83231002B3FF47AAF98F82E31082B13D1684E664D684F0FCE05F5F87404942E
:20D780000FC40FCE0FC496E80700012384E8070085F82832C5F8087299E05D4D624E039B6B
:20D7A000C5F82C320FCE05F5DE740FC40FCE0FC496E8070098F832C10023BCEB030C84E855
:20D7C000070018BF4FF0010C1946584898F82E3187F890364FF44C7285F828C287F8581697
:20D7E0008B4666F0E0FE494B0593514B049305F50E76D5F82C325B455EDD049A12F8013B5D
:20D800000492434493F8334120463FF0D5F88146204643F095FB98F82F310446002B4DD018
:20D8200099F8073083F0010A0AF0010995F8280209F1010987F8579608B18AF0010A002C0D
:20D8400049D0A17989B141290FD03A4B3A493B4AC5F8D831012387F85836C5F8D411C5F82F
:20D86000E0210023C5F82432DAE6204645F054FA4FEA49110BF1010B41F009014FF00303AD
:20D8800071617060F46086F810A084F807B0A37120463FF0F3FB1AF0010F204611D043F006
:20D8A00095FF059AF3685361BBF1080F02F1180306F1200605939CD1214BD3E799F807A0D5
:20D8C000B2E743F089FFECE7082F7FF4E8AE1D4BC5F83032E3E6204645F01EFA4FEA491943
:20D8E00049F009010BF1010B71617060F46086F810A0CDE7E27903E7104B0E4AC5F814320A
:20D90000C5F80C220023ADE7286200203C000010001100103C470708419406081047070873
:20D9200084680020402F002068470708BC6800207E3000205DA7040861A7040855A7040850
:20D94000BC120010ED34050898F83131064AC5F83022012B05D0022B06BFBCFA8CF35B09DE
:20D96000002385F834329AE61D350508F8B56D4F97F8A80397F8A95343F0E2FA60B12D2324
:20D98000C380202104463FF079FB0A203FF00AFE204645F0B7F918B9D7F8C439DA0000D51E
:20D9A000F8BD013D092DFBD897F8A743D4B9402038F00EFD0028F3D090F9043097F879130F
:20D9C000092BC8BF143B3B440A2993F8C84900F09B8093F8D43997F8A623002A08BF1C46A1
:20D9E000002CDDD0204643F0ABFA0546002800F083802D23C38001213FF040FB012108461B
:20DA000043F0F8FE2B68AA881A833C2040F022F80021012043F0EEFE97F8A933002B4CD0C2
:20DA2000414C00261FE02B68AA885A833FF0BAFD94F8901ED4F8940E01F0010143F0D2FE0E
:20DA400094F8901ED4F89C0EC1F3800143F0CAFE2B68AA881A8378203FF0A4FD97F8A933B1
:20DA600001369E4229DA94F8901ED4F8940EC94301F0010143F0B6FE94F8901ED4F89C0E4E
:20DA800081F00401C1F3800143F0ACFE7820002DC9D178203FF086FD94F8901ED4F8940EAD
:20DAA00001F0010143F09EFE94F8901ED4F89C0EC1F3800143F096FECDE797F8A7339BB987
:20DAC000D7F8A83303F0FF13B3F5803F7FF468AFD7F8C43913F080537FF462AF87F8A93325
:20DAE000BDE8F84053F010BA32203FF0B3FF284600213FF0C3FAE3E701213FF0BFFA012198
:20DB0000084643F077FE80E7D7F8EC395B057FF547AF0AF057F900287FF442AF002C7FF475
:20DB200061AF3DE728620020402F0020084B03F51F600DC8904202DC114602460846984262
:20DB400004DD9A42B8BF1A4610467047704700BF28620020144AD2F8FC09D2F8003AD2F809
:20DB6000081A984230B4D2F8044AD2F80C2A02DC1D4603462846914202DC15460A462946EA
:20DB80008842A8BF08469342B8BF1346844202DB224604461046984203DD9C422046B8BF41
:20DBA000184630BC704700BF286200200B6810B414681B1B036054684B681B1B43608B6874
:20DBC00092685DF8044B9B1A836070472DE9F047041E0D4612DB092C26DC824A0B4682488B
:20DBE000A0FB0410C00800EB8000A4EB40000021125C1A7059702846BDE8F08764422D2312
:20DC0000092C01F8013B24D8764A774BA3FB0403DB0803EB8303A4EB43030020D35C487044
:20DC20000B702846BDE8F0876F4B632CA3FB04264FEAD60621DC6B4A0B466B49A1FB06015F
:20DC4000C90801EB8101A6EB4101515C03F8011BC5E7654A632CA2FB04364FEAD60637D809
:20DC6000604A614BA3FB0603DB0803EB8303A6EB4303D35C01F8013BC7E7A3FB0627B4F5F3
:20DC80007A7F4FEAD7070DD2564A0B465649A1FB0701C90801EB8101A7EB4101515C03F8A6
:20DCA000011BCAE7A3FB072842F20F7294424FEAD80836D84B4A0B464B49A1FB0801C90828
:20DCC00001EB8101A8EB4101515C03F8011BDDE7A2FB0637B4F57A7F4FEAD7070CD2414A7D
:20DCE000414BA3FB0703DB0803EB8303A7EB4303D35C01F8013BB4E7A2FB073842F20F7330
:20DD00009C424FEAD80821D8364A374BA3FB0803DB0803EB8303A8EB4303D35C01F8013BD4
:20DD2000DEE7324AA3FB080994424FEAD90921D82C4A0B462C49A1FB0901C90801EB8101E8
:20DD4000A9EB4101515C03F8011BB5E7274BA2FB08099C424FEAD90921D8224A224BA3FB04
:20DD60000903DB0803EB8303A9EB4303D35C01F8013BCAE71E4AA3FB090394424FEAD30A53
:20DD800021D80B461849174AA1FB0A01C90801EB8101AAEB4101515C03F8011BCAE7144BE6
:20DDA000A2FB09029C424FEAD20A13D80E4B0D4AA3FB0A03DB0803EB8303AAEB4303D35C21
:20DDC00001F8013BCAE70A22BAFBF2F052F08CFE0346D7E70A22BAFBF2F052F085FE0146F8
:20DDE000E4E700BF60E00708CDCCCCCC9F8601003F420F0070B4344890F8103AA3F130012C
:20DE0000092957D800F52164224600F61F2012F8015FA5F13001092904D88242F7D100209F
:20DE200070BC7047141B022C4ADD2848002101E010F8013B01EB810103EB4103161A303B8A
:20DE4000022E044603F0FF01F2DC214B03FB01F1A2424FF000030DD903EB830314F8016B33
:20DE60005B00303B3344A24203F0FF03F4D1194800FB03F32E2D06D01748A0FB032301EB38
:20DE8000930070BC7047013204200024157804EB8404303D6400092D00F1FF30A4B202D836
:20DEA0002C44A4B2013210F0FF00EFD1642202FB0433E1E700211D4600F521620B46D9E71B
:20DEC000064C0021C4E700BF28620020396C00208096980040420F00ABAAAAAA386C00204A
:20DEE00038B504460D460A460068FF2166F05BFB21682944216038BD83B50C461646054677
:20DF000036F00CFD204636F009FD0021204B0846002E08BF1E4643F06DFC0021012043F0FC
:20DF200069FC284640F0DAFAB0B10121002043F061FC284640F0CAFA0746204640F0CAFACE
:20DF40000028FAD03946204640F0CCFA3846B0470021084643F04EFC204640F0BFFA00281C
:20DF6000DFD00121002043F045FC204640F0AEFA01462846019140F0ADFA01990028F8D056
:20DF8000284640F0AFFA0021084643F033FCC8E70D460408F0B50023C1E90033C1E90233D7
:20DFA0000B610268DFF888C089B004ADC2F385572E4647FA03F0C007344604D513F80C0018
:20DFC00004F8010B26460133062BF2D1164CDFF864C0C2F303200023205C33708DF8180091
:20DFE000C2F305370DF1190647FA03F0C007344604D513F80C0004F8010B26460133062BD5
:020000040800F2
:20E00000F2D100233370C2F3834406ABCDE90134084602F00F0305490095C2F3031253F01D
:20E02000B1FA09B0F0BD00BFB8E0070888E00708C0E00708B0E0070870B5094CD4F8202A14
:20E04000054662B10026D4F8200A2D21013646F0DBFCAE42F7DBBDE8704046F0BDBF70BDBE
:20E06000286200202DE9F04F5FFA81F9002185B007460846164643F0BDFB0021012043F021
:20E08000B9FB42F029FF022E0AD0042E44F6C01818BF4FF49648B9F1070F07D900200CE080
:20E0A000B9F1FF0F4FF41648F5D10326CD4D95F8243A2BB90020C5F8280A05B0BDE8F08F47
:20E0C000032EC94C0DD0A144002299F8330103213EF0ECFB0028EDD0C4F80405C3799A0791
:20E0E000E8D495F8240A84F81F6D002203213EF0DDFBC4F808090028DCD0BC4ABC4BC4F8EB
:20E10000C03402F1480003234FF48061A4F8C434C4F8D404002302F24C404FF0010A032E40
:20E12000C4F8C884C4F8EC34C4F8CC14C4F8E034C4F8DC34C4F8D804C4F8D014C4F8E834B3
:20E14000C4F8E43484F8103DA4F80CADC4F8183DA4F81C3D84F81E3D91460ED0D4F804B5B6
:20E160009BF8040042F0ECFEC4F80005584615F067FE5146484615F077FE32203FF06AFC9D
:20E18000002E5FD1D4F80889D8F8000007F02CF94046984A22213EF0E7F8974B9749C4F8A2
:20E1A000243D324640463EF023F8D4F80485D8F8000007F019F98F4A4FF6FF7140463EF047
:20E1C000D3F831464046FEF753FD8D4B8D49C4F8283D324640463EF00BF8C5F8289A4FF076
:20E1E000060A022E12D0D5F8280A40F077F968B10121002043F0FEFAD5F8280A40F06EF942
:20E200000146002840F09A8043F0F4FA384640F065F988B10121084643F0ECFA4FF0050B07
:20E220004FF00008384640F059F90146002840F08E80012043F0DEFA042ED4D005203FF094
:20E2400009FCCEE7012E09D1D4F808094146FAF741FCD4F80405FEF795FDBEE7022E09D15E
:20E26000D4F8040515F0DBFDD4F808094146FAF731FCB2E7032E59D14FF0000A51466248EC
:20E2800084F820AD402266F08EF98DF80FA0DFF87CA19DF80F30072B09D95448012115F023
:20E2A000E3FDD4F808094146FAF714FC95E79DF80F3003EB43030AEBC30393F8453073B3B4
:20E2C0009DF80F3003EB43030AEBC3039B6C33B39DF80F30234493F8330100B3002203219B
:20E2E0003EF0E4FA8346D0B115F099FD9DF80F3094F8202D03EB43030AEBC30305EBC201DE
:20E300009B6CC1F82C3A9BF80730DB0748BF012302F1010248BF81F8303A84F8202D9DF8C2
:20E320000F300133DBB28DF80F30B2E7042E7FF454AFD4F8040515F072FD85E7D5F8280A24
:20E3400040F0C4F80146384640F0CCF854E7384640F0BCF895F87A3A01468BB9242803D18F
:20E360004FF0010385F87A3A012E04D13846019140F0B8F80199D5F8280A40F0B3F851E789
:20E38000012B06D14D280CBF0223002385F87A3AEAE7022B06D13C280CBF0323002385F8F7
:20E3A0007A3AE1E7032B10D10A2802D985F87A8ADAE7042385F86D0A85F86C8A85F86F8A7F
:20E3C00085F86E0A85F87A3ACEE7042B20D195F86E3A85F87B0A434085F86E3A85F87ABAB2
:20E3E000C2E700BF28620020402F0020003400209447070840420F00F53E0208643C0020B0
:20E40000D5120208683C0020546C002008000010052BA9D195F86C3A95F86D9A95F86E0AD9
:20E420004B4509D25A1C2B44484085F86E0A85F86C2A83F8701A97E78842B7D195F87B3AE5
:20E4400085F87AAAF42B8FD1B9F1000F8CD12421384685F87A9A40F045F84D21384640F0A9
:20E4600041F83E21384640F03DF84946384640F039F8F421384640F035F8F421384640F000
:20E4800031F8032E1BD0D4F80405437901689D080223AB40DB439BB20B828D892B408B8103
:20E4A0000079202115F0AAFCD4F804054A4649463DF09EFED4F80435186806F095FF002209
:20E4C000D4F8080911463DF093FED4F80839186806F08AFF0120F0E530B583B04D1C009334
:20E4E00003688572C2729C690023A04703B030BD03685B6C0BB102211847704770B51D4C22
:20E500000968D4F8805A1C4ED4F87C4AD6EDCB7ADFED1A6A491B00EE901A0168F8EEE00A5B
:20E52000091B60EEA70A00EE101A20EEA07AB8EEC00A1C46A0EE007AB1EE400AF1EEC77A95
:20E5400067EEA67AFCEEE77AC2ED007A53F0EAF89FED0B7ADFED0B7AE0EE077AFDEEE77AB0
:20E5600017EE902A002ABCBF02F50C42A032226070BD00BF28620020880100202C7D8E3FE9
:20E58000A00CB34500A00C4638B50F4C94F89B1A01F03F018B1C024601F10A0584F8993AEC
:20E5A00084F8965A04F6942084F8972A083120F0B5FB254485F8920A94F8963A1C44000AC3
:20E5C00084F8930A38BD00BF2862002038B50B4C002501228021204637F0E6FE30B194F9B8
:20E5E000040037F013FF08B1006838BD0135092D04F10C04EDD10020F7E700BFE46C00206C
:20E6000038B5041F00F1080554F8043FD81780EA430017F001FEA542F6D138BDF8B5C94C56
:20E62000DFEDC97A94EDCE7A94F8A033B4F8A2732DED028BB8EE478A28EE278A002B5FD1A2
:20E64000D4F8AC3394F8BD23002B40F30E8107EE902A9FEDBE6ADFEDBE6AF8EEE77AB7EE73
:20E66000007AA7EE867AF0EE477A07EE103AF8EEC78AB7EE087A87EE270AC6EEA87A20EEC5
:20E68000270A64F08BFC0F28B8BF0F2094F8A13385B2A4F8A253002B00F04781AF4234D091
:20E6A000B4F8A4339FEDAB6A94F83C6307EE103A07EE905AB8EE477AF8EE677AC6EE076A9A
:20E6C00086EE277A76EE887A37EE087AC8EE276AC8EE077AB6B394F8A633B4F8A853C4ED74
:20E6E000D37AC4EDD77AC4EDDB7AC4EDDF6AC4EDE37AC4EDE77A002B5BD0BDEC028BF8BD6A
:20E7000094F8A133002B00F0858094F83C63002E40F00381B4F8A433DFED8E6A07EE907A26
:20E7200007EE103AB8EE676AB8EE477AC6EE877A86EE867A77EE887A37EE087AC8EE276A3E
:20E74000C8EE077A94F8A663B4F8A8530023C4F84033C4F84433C4F84833C4F85033C4F88F
:20E760005433C4F85833C4F86033C4F86433C4F86833C4EDD37AC4EDD77AC4EDDB7AC4ED1B
:20E78000DF6AC4EDE37AC4EDE77AC4F87033C4F87433C4F87833C4F88033C4F88433C4F849
:20E7A0008833C4F89033C4F89433C4F89833002E66D1D4F8AC3394F8BD23002B40F38E802D
:20E7C00007EE902A9FED616ADFED616AF8EEE77AB7EE007AA7EE867A07EE903AF8EEE77A9B
:20E7E000B7EE086A86EE070A86EEA77A20EE070A64F0D4FB0F28B8BF0F2080B2A4F8A80350
:20E80000002E3CD0A8423FF478AF00286DD1BDEC028BF8BDD4F8AC3394F8BE23002B40F3B3
:20E82000878007EE903AF8EEE78A3D4607EE902A9FED466ADFED466AF8EEE77AB7EE007A6B
:20E84000A7EE867AF0EE477AB7EE087A87EE270AC6EEA87A20EE270A64F0A0FB0F28B8BF05
:20E860000F2080B2A4F8A40318E794F8A1330F25A4F8A253002B7FF411AF2846F2E70546E0
:20E8800094F8BC3384F8F936002D3FF436AF07EE905A9FED306AD4EDF06A2F4BF8EE677AAC
:20E8A000BDEC028B86EE277A1946002241F8042B012084F8F8060A609A601A615A619A61F4
:20E8C0001A625A629A6237EE267AC6EE877AC3ED037AC3ED077AC3ED0B7AF8BD0F20A4F877
:20E8E000A80346B30F2D3FF408AF07EE900A9FED196AD4EDF06A194AF8EE677ABDEC028B35
:20E9000086EE277A37EE267AC6EE877AC2ED007AC2ED087AC2ED047AF8BD94F8A633B4F81B
:20E92000A853002B7FF4E9AE43E794F8BE237DE73D460F2096E794F8BC3384F8F93605460C
:20E94000A5E700BF00110010BD378635CDCCCC3D002474494E2DA63DC8170010D4170010D1
:20E96000F8B5214C1D270E46054684F82C7B20F0FBFA002020F09AFA082020F097FA0E20B7
:20E9800020F094FA384620F091FA042020F08EFA042020F08BFA002020F088FA302020F039
:20E9A00085FA002020F082FA304620F07FFA002020F07CFA20F0C4FA04F62D3020F0CAF98F
:20E9C000234670B194F82D2B62B994F82E2B302A00D03AB993F82F2B22B993F8303B2B705B
:20E9E0000120F8BD0120FCE728620020114B10B50446185C14F0DCFC0F4800EB8404D4ED4D
:20EA0000007AFDEEE77A0A2317EE901AB1F5FA6FA8BF4FF4FA61B1F57A7FB8BF4FF47A71FC
:20EA2000A1F57A71BDE81040B1FBF3F10920C9B214F0ECBC98E00708686D00201D4991F815
:20EA4000102AA2B3F0B4002605463346304637461BB991F8104A2D2C23D02E2A19D0CA1880
:20EA600000EB800092F8104AA4F13002092A4FEA40009CBFA0F13002A0180E2B14D80133A5
:20EA8000CA1892F8102A002AE2D106B14042F0BC70470133002DF8D0CA182A4482F8107ADA
:20EAA000DDE701231E46EBE70020F0BC70470020704700BF286200202DE9F0410C4F0124AE
:20EAC000A0231825E6B2FF2B0BDCC5F11B0103F10108D7F8880BDBB23246C9B2FFF7FCFCEE
:20EAE0004346013DEFD10134052CEAD1BDE8F081286200201FB503AC8DF80C3000940023B3
:20EB00008DF80D300CF0A6FE04B010BDF8B50546262029F0E3FC154C014610BBD4F88C0B06
:20EB200090F838301E3B012B02D894F8993B0BB13FF0D8FC0E4F0026AE420ADBB4F8BA3B6E
:20EB40000133A4F8BA3B0B4BD3F88430C4F8CC3BF8BD17F8011BD4F88C0B3FF0C3FC0136F0
:20EB6000EAE7002384F8C83BEDE700BF28620020C26D0020402F002010B58021044605F062
:20EB80009BFA2046002105F097FA2046BDE8104005F0D2BD2DE9F041B14C94F8E33BC4F84A
:20EBA000D00B82B088465A2B00F2B980DFE813F0CC00B700B700DC00B700B700B700B7000E
:20EBC000B700B700B700B700B700B700B700B700B700B7000F01B700B700B700B700B7006C
:20EBE000B700B70033017400B700B7007400B700B700B700B700B801B7006201B700B70000
:20EC00007C00B7000902B700B700B700B7005B00B700B700B700B700B700B700B700B700C7
:20EC2000B700B700B700B700B700B700B700B700B700B700B700B700B700B700B700B70064
:20EC4000B700B700B700B700B700B700B700B700B700B700B700B700B700B700B700B70044
:20EC6000B700B700E40194F8E43B9B0700F16982B4F8EA3BD4F8E52BD4F8241C5BBA9BB2FD
:20EC800012BAD0188842C4F8303CC4F82C2C03D905F0D2F9002854DB0020A4F81C0C054698
:20ECA000284602B0BDE8F08194F8283C002B40F0FF8094F9E03B002B31DAD4F8183C084608
:20ECC0009B689847002840F01E82B4F8EA0BD4F8E52BD4F8243C40BA80B212BA15189D42AD
:20ECE000C4F8300CC4F82C2C07D905F0A5F9002827DBD4F82C2CD4F8300CD4F8203CD4F84B
:20ED0000DC6B03FB00F003FB02F20225B042C4F82C2CC4F8300C84F8285C00F0CF8094F8DC
:20ED2000F43B5A1CD2B204EBC30305204FF40051042A84F8F42B83F8F80BC3F8FC1B00F033
:20ED4000A0814FF0FF35ABE7D4F8DC3B002BE6D1D4F8183C08469B6898470546002840F0D5
:20ED6000D281A4F81C0C9BE73E4B002203F1120103F8012F8B42FBD13B4994F81E3C94F88E
:20ED8000F40B70250D7098424FF00C05CD7110D004EBC300013390F8F85B8D70B0F8FC0BAD
:20EDA000DBB2042B40BA888114BF84F81E3C84F81E2C94F8E73B12229342A4F81C2C98BF33
:20EDC000A4F81C3C0025284602B0BDE8F08194F8E43BDA0700F13E81D4F8183C94F8E70B0A
:20EDE000DA6901EBC10102EB81010A79531D834228BF0346A4F81C3C002BE3D0013B1A485B
:20EE00009BB201331944034411F8012D03F8012D8342F9D1D6E7154E154F35460823073E6F
:20EE2000C5F10700A4F81C3C002202E092F884211D462B46B54203F8012900EB030217FAFD
:20EE400082F2F3D1D4F8183C4046DB6898470028B8D0AB7863F07F03AB70002520E700BF04
:20EE6000286200201B9100201C9100202391002048460708D4F8183CC74A5B680846111D6E
:20EE800098470546002840F03E81D4F8243CC34AD4F8201C013B180E1070180C09BAD370E4
:20EEA00050701B0A082093705160A4F81C0CF7E6D4F8306CD4F82C2CD4F8203CD4F8185CFC
:20EEC000B2FBF3F24FF48057BE4228BF3E462D69B249A4F81C7C4046B6FBF3F39BB2A847FD
:20EEE0000028C0F2BC803346AC4AD4F8D00B812105F016F9D4F82C2CD4F8300CD4F83C3CD0
:20EF00003244851B9E1BC4F82C2CC4F8305CC4F83C6C002D7FF456AF032384F8283CBFE612
:20EF20009E4E0027334606F10C0203F8017B9A42FBD1D4F8183C40465B686A4601A998477F
:20EF40000546002840F0E980019BBDF80020013B190E52BAF3713171190C1B0A717108206B
:20EF6000B371022172810C23BDF80220F07031727272A4F81C3C93E6894E8A4F30460823AC
:20EF8000073EC0F10705A4F81C3C002202E092F88C2118460346864203F8012905EB0302B7
:20EFA00017FA82F2F3D1D4F8183C4046DB68984700283FF407AFF37863F07F03F370002567
:20EFC0006EE694F8283C002B61D194F9E03B002BFFF6A5AED4F8183C08469B6898470028FD
:20EFE00040F09180D4F8183C4046DB6898470546002840F0BA80B4F8EA3BD4F8E52BD4F8B2
:20F00000241C5BBA9BB212BAD0188842C4F8303CC4F82C2C00F29F80D4F8201CD4F8DC0BC8
:20F0200003FB01F302FB01F28342C4F82C2CC4F8303C7FF474AEB3F5805F28BF4FF48053D4
:20F040000121D4F8D00B554A84F8281C9BB205F091F925E607235449A4F81C3CCEE694F8B6
:20F06000F43B5A1CD2B204EBC30304204FF48851824284F8F42B83F8F80BC3F8FC1B7FF450
:20F0800060AE002384F8F43B4FF0FF3508E6D4F8306CD4F8180CD4F8203CD4F82C2C4569E1
:20F0A000B2FBF3F2B6F5805F28BF4FF480560846B6FBF3F339499BB2A847002862DBD4F860
:20F0C0002C2CD4F8305CD4F83C3C3244AD1B9B1BC4F82C2CC4F8305CC4F83C3C2DB9D4F806
:20F0E000D00B294605F09AF9DAE5B5F5805F28BF4FF48055ABB2D4F8D00B284A012105F06A
:20F1000039F90025CCE594F8F43B5A1CD2B204EBC30302204FF468510AE694F8F43B04EBC5
:20F12000C3020133DBB202204FF46851042B82F8F80BC2F8FC1B22D084F8F43B4FF0FF359E
:20F14000AEE594F8F43B5A1CD2B204EBC30305204FF41051ECE504F06FFF0028FFF6F1ADFB
:20F16000D4F82C2CD4F8303C56E794F8F43B5A1CD2B204EBC30302204FF41C51D8E584F881
:20F18000F47BDEE594F8F43B5A1CD2B204EBC30304204FF440716BE7486E00201C910020C6
:20F1A0002391002048460708C447070810B51C2041F0C6FE112104463DF060FF204642F02E
:20F1C00005FBC8203EF046FC2046BDE8104042F003BB00BF08B5002041F0B2FE054BC3F804
:20F1E000440C08B12A23C380BDE8084040213DF045BF00BF286200202DE9F04FB34CD4F86E
:20F20000DC3A5A69D2078BB002D50BB0BDE8F08F5A699B6912EA030AF7D0CAF307431AF49F
:20F22000002F009340F00281009B5D0743D41AF0020F5FFA8AF503D0D4F8DC3A02225A61BC
:20F24000BAF1000FC0F211821AF4006FCAF3072740F084812E0708D59D4B9E48D3F83C33F8
:20F260009847D4F8DC3A08225A61ED0600F1E981F80600F1A981B90600F12E81009BDA06A7
:20F2800009D5934B9348D3F84C339847D4F8DC3A4FF480125A61009B9B06B6D58C4B8D48C9
:20F2A000D3F850339847D4F8DC3A4FF400125A610BB0BDE8F08FD4F8E02A9369D2691340F0
:20F2C0001FFA83FBBBF1000FB1D0DFF80882CDF80CA045464FF0000909E05FEA5B0B09F124
:20F2E000010908F1040805F1280500F0DA811BF0010FF2D0D4F8E01A5FFA89F708694A6BEF
:20F3000004EB8703FA40D3F8E83AD2019B68D2B202431A40D007D3B216D54B6BD8F818204F
:20F32000012000FA09F023EA00034B63684B6948D3F83433012191603946984794F8D36A2B
:20F34000012E00F0FE8101231A0703D5D8F8182008239360DE0603D5D8F8182010239360E2
:20F36000580603D5D8F8182040239360990703D5D8F81820022393601A06AED5D5E94C6054
:20F38000D5F82431D8F818C0311A8B42DCF8182028BF0B46033392B2B2EB930F9DD9D4F84C
:20F3A000E02A323704EB8703CDE9019890469946B04238D2BEB3D5F8241194F8D33AD5F888
:20F3C0002821371AB94228BF394601F1030E4FEA9E0E83B98FB20337BF10D9F8D8AA0AD097
:20F3E000013352F8040BCAF800009F42F8D1D5E94C60D5F82821DCF8183008440A44B042EC
:20F40000C5F82821C5F834010AD195F81C11D8F83420012707FA01F122EA0102C8F83420FD
:20F420009BB29E45C4D3DDE9019856E7D4F8E03A9D69DB691D402D0C3FF4F6AE04F52D6640
:20F44000DFF88CB0B046B146002708E06D0807F1010706F1040608F128083FF4E5AEEB0746
:20F46000F4D5F9B204EB8102D4F8E03AD2F8242B92685B691A40D007D3B218D594F8D30ADD
:20F48000726D01239842936007D11269D8F87C33C2F312029B1AC8F88C33DBF83033484609
:20F4A000984794F8D33A012B00F0598101239A0702D5726D022393601B07C7D5DBF838334F
:20F4C00048469847736D08229A60BFE73051002088010020005C0020D4F8E03AD4F8E81A9B
:20F4E0009A680868C2F34102022A08BF03224FF0000514BF65F30A0062F30A0008605A6888
:20F5000042F480725A6006A806F01CF8D4F8DC2AD4F8E00AD368C049079D6FF38D23D3609C
:20F520008068C0F34100014491F89411032900F0D180BA49BA480126294484F8D26A8142FB
:20F540004FF04006A4F8D46A00F217810E2161F38D234FF40051D36051618FE6B14B94F819
:20F56000E22BD3F84433B04800218DF817108DF817209847D4F8E01AD4F8DC2A94F8DA3AA4
:20F5800088684FF400615161002B3FF463AEC3077FF560AE94F8E53B012B7FF45BAE9DF881
:20F5A0001730032B7FF456AED4F8DC3B9F491A6842F001021A601A6842F003021A600B69BC
:20F5C00043F006030B6145E6D4F8E02A964853684FF0000823F001034146536005F0D8FB89
:20F5E00094F8D16A414656B1914BFF2203EB860653F8045FD86BAA609E428260F8D1D4F8ED
:20F60000E03A89484FF0FF329A614FF00112DA610B2262F3070162F30708C3F81480196150
:20F620001A686FF30A121A6005F086F8D4F8DC2A7C4B7D48D3F840334FF48051516198479C
:20F6400019E6D4F8DC3A9A6922F010029A611A6AC2F34340022802F00F0146D0062823D088
:20F660009A6942F010029A6102E694F8DA3A3BB1D4F8DC2B136823F0030161F3070313609E
:20F68000D4F8E02A67495368D1F84813664823F0010353608847D4F8DC3A4FF000425A61A0
:20F6A000D2E5DDF80CA0C2E5D4F8A05B614E286801EB810104EBC10141F29C0CC2F30A129A
:20F6C00044F80C00D1F85C0E024428683060C1F85C2EC5E700214FF4007084F8D21A0921F4
:20F6E000A4F8D40A61F38D2333E747F6F0701042B6D001EB8100C2F30A1204EBC00002F11D
:20F70000030C5FEAAC0CD0F8505ED4F8A0EB4FEA810818BF002006D00130DEF8006045F8D9
:20F72000046B8445F8D1414404EBC101D1F8505ED1F85C0E15440244C1F8505EC1F85C2E9F
:20F740008EE7B9F1000F7FF4FEAD94F8E13B042B7FF4F9AD344804F0EFFF3346F4E5002F8E
:20F760007FF4A4AE94F8E12B052A7FF49FAE4846019304F0E1FF019B99E62F48A5F57401A6
:20F78000A1F51051814203D80D2161F38D23E0E62A492B482944814203D20C2161F38D23C0
:20F7A000D7E62848A5F18C71A1F54341814203D80B2161F38D23CCE62349244829448142E7
:20F7C00003D20A2161F38D23C3E6214921482944814203D2092161F38D23BAE61E48A5F1DA
:20F7E000B771A1F55851814203D2082161F38D23AFE61A491A482944814203D2072161F302
:20F800008D23A6E6174918482944814234BF0621052161F38D239CE648460708401E1BFFE1
:20F820003F420F0088010020005C002000ED00E0145C0020D0610020DFC810002013FBFE82
:20F8400020D61300FF69180000D3CEFE40771B00C05BB3FEC091210040AC2700C01D6AFE18
:20F8600040E13300803C36FEE09C4100704700BF704700BF704700BF704700BF2DE9F04168
:20F880004FF0FF35324A33482C46002304E001330B2B02F1100215D0917A0429F7D103F539
:20F8A000B17100EB0111C979CF07F0D4661C116801D0A942EBD21C4601330B2B0D4602F1C7
:20F8C0001002E9D1631C02D10120BDE8F081214D04F5B17705EB07139988F1B9DFF8808098
:20F8E0002601AB1958F82C2C1B4916691B4A41F2186001EB442118580023B047D0B10228FC
:20F9000008D141F2CC6205EB0717AB58013B0121AB50B9710020BDE8F081DFF8448005EB58
:20F92000041358F82C2C41F21860D268185826019047D6E741F2CC6205EB0717AB58032162
:20F94000B97141F2D061013B0124AB506C54BCE738B700201CA1002034A100207DF90008FB
:20F9600028620020044B41F2E472995C09B90121995401225A7070471CA1002038B5174D6D
:20F98000174B41F2D0640020285504E001300B2803F1100314D053F80E4C8C42F6D11C7800
:20F9A000032CF3D16AB10F4B03EB40239A4201D0FFF7D8FF00F5B17005EB001001238371E6
:20F9C00038BD41F2CC6100F5B1736A5805EB03130420013298716A5038BD00BF1CA1002046
:20F9E00042B7002034A1002038B5134B00209C7B14B11D688D4205D001300B2803F110031E
:20FA0000F5D138BD72B10D4B03EB40239A4210D0FFF7A8FF0A4B00F5B17003EB0010012379
:20FA2000837138BD064B00F5B17003EB0010827138BD022CECD1EDE734B7002034A10020D1
:20FA40001CA100202DE9F84F12F0020E9B4606D028B9FFF787FF02252846BDE8F88F804CB9
:20FA600041F638056559002D5BD14FF0FF367D4FB146B046B24600253B68984200F0B6800E
:20FA800097F80EC0BCF1000F5BD0BCF1010F15D105F5B17C04EB0C1C9CF807C01CF0010FCA
:20FAA0000CD11CF07E0F09D15FEADC1340F0A880D7F808C0D44501D2E246A94601350B2D5E
:20FAC00007F11007D8D1751C04D1B8F1FF3F00F09F80464641F2C86806F5B17754F808505C
:20FAE000013544F8085004EB061C41F21C694FEA07184CF8095044F8085041F2186904EB47
:20FB000007154FF000084CF80900C5F8048004EB0715AD79042D9CD8DFE805F01A330F33D3
:20FB20004D0004F5C25741F63C063F68A65907FB0565A84299D3FFF715FF00252846BDE843
:20FB4000F88F2E4601350B2D07F1100794D1BAE712F0010C70D104EB0710D51090F80780DD
:20FB6000BBF1030F65F3C71880F8078062D94FF6FF7083455B4628BF03469BB204EB0710B6
:20FB80008380BEF1000F16D004EB061303F5B0531833987B04280ED041F2C8654FF0040CA4
:20FBA00060590130605141F2CC65586083F80EC0635901336351500705D504EB0710C3792E
:20FBC00043F00103C371D30608D504EB0714E379C3F34502013262F34603E371224B0125E9
:20FBE00003EB46260E602846BDE8F88F05F5B17704EB07164FEA071CB67986B92E4669E7E7
:20FC0000A84601350B2D07F110077FF435AF5AE7B9F1FF3F18BF4E467FF45CAF8DE741F269
:20FC2000C8682E4654F80850013544F8085044F80C506CE76346A1E70C4B0B4953F82C3C38
:20FC40000B4AD3F8088001EB46210023C04700283FF473AF04EB07140223A371FCE600BF1E
:20FC60001CA1002034B7002034A1002028620020E9F90008F0B5124D2B7841F63002022BD6
:20FC80000BBF070AC0F3D417C4B200F07F04A85883B00E4600230122384401A9FFF7D2FE49
:20FCA00001280AD12B78022B019B16BF53F8243033F8143023F07043336003B0F0BD00BF79
:20FCC0001CA1002010B5144602070B4610D50B4941F2C472581C8B58834204D305D1002340
:20FCE0002360012010BDFFF73DFE2060012010BD21461846BDE81040BCE700BF1CA10020FB
:20FD00002DE9F0414268C2F308030B44B3F5007F82B004460D4657D390F91A30591C0AD0A1
:20FD2000304A03F5B17302EB0313FF21DA796FF30002DA71817694F91B305A1C0FD0294A71
:20FD400003F5B17302EB0313FF20DA79C2F34501013921EAE17161F34602DA71E0762378A8
:20FD6000022B37D01F4A02F5C2531B68B5EB432F4FEA432824DC41F648036768D6583E40A4
:20FD80007342AB421CDCAB19434511D32169207E01AAFFF797FF012812D16768236963610F
:20FDA0004744019B2361A5EB0801BF1B67608D192046F8F78FFB20B93D446560012000E0B9
:20FDC000002002B0BDE8F08115444560012002B0BDE8F081616801202944616002B0BDE8E5
:20FDE000F08100BF1CA1002070B5154604460E46FFF786FF50B994F8280028B9022384F81E
:20FE00002830C4E90B5670BD022070BD1DB12046A847012070BD012070BD00BF10B4D0E905
:20FE2000011390F91A208B4238BF0B46511C83600AD0144B02F5B17203EB0212FF21D379C5
:20FE40006FF30003D371817690F91B305A1C0FD00C4A03F5B17302EB0313FF24DA79C2F339
:20FE60004501013921EAE17161F34602DA71C4760022436A5DF8044B426142601146036111
:20FE8000B2E700BF1CA1002038B544220021114864F089FB104B41F602011A784FF6FF74A9
:20FEA0005C52022A41F2E87118BF032203F5C05041F64C055A5441F60C0441F601020321FD
:20FEC0005D5900F8181910211D519954FFF7A6FF012038BD04B900201CA100202DE9F04105
:20FEE000B1F904300F2B82B00C461646054632D02846F8F713FB95F91B80B8F1FF3F0746F5
:20FF000033D02D4B41F2186203EB08118A58904211D1183303EB4823A188013109B203EB74
:20FF20004113A18028463360F8F7F8FA2060012002B0BDE8F081FFF715FD2846F8F7CAFAD8
:20FF400028B100230120336002B0BDE8F081002002B0BDE8F0814FF40071FFF7D1FE0028A0
:20FF6000F5D04FF6FF73A380C2E72846F8F7B2FA0028E2D10FB9FFF7F5FC384600231122D2
:20FF800001A9FFF75FFD0128D7D1019B0B4A9A1A48BF02F2FF12B2F5B05F4FEA622106D299
:20FFA0004FFA81F885F81B80002BB5D1C5E7FFF7D9FC019BF6E700BF1CA1002034A1002035
:20FFC00030B50446C06983B010B9012003B030BD0D460023032201A9FFF734FD0128F5D1B1
:20FFE000B4F92030002B03DAFFF7BCFC0220EDE7019A012D4FEA431102EB431303D0022DBD
:020000040801F1
:2000000012D1E5255554A268DA612278032A04D100221A775A779A77DA77626A5A83C2F325
:200020000F429A8203B030BDE268DA61EDE700BF10B50378023B012B0446037E02D913F049
:20004000060F5AD198063AD494F91A30591C0AD02D4A03F5B17302EB0313FF21DA796FF323
:200060000002DA71A17694F91B305A1C0FD0264A03F5B17302EB0313FF20DA79C2F34501F3
:20008000013921EAE17161F34602DA71E076237E1B070BD51C4841F2C873C35C072B01D0F5
:2000A000FFF760FC41F2C8730022C254E26A0023237084F82830FAB1BDE810401047002358
:2000C0001249E0691A018A58904206D001330B2BBAD01A018A589042F8D10B4A03F5B173DA
:2000E00002EB0313DA79C2F34501013921EAE17161F34602DA71A7E710BD0121FFF760FF5F
:200100000128F9D1237E9DE71CA1002034B7002030B1027822B190F828201AB1002070473F
:200120000120704710B5D0E90142A242C16238BF22460321826080F82810FFF779FF01207B
:2001400010BD00BF2DE9F04FDFF868918A4699F80010DAF800300229174683B0834641F6C0
:20016000300240F08B8059F80250DEB2A6EB030805EB1325B8444FF480729044BB4208F120
:20018000FF38B8FBF2F875D2A844032906EB0704A4EB03040CBF80224FF48072944228BF3B
:2001A0001446A8EB050366B994422CBF0A220B2201A92846FFF746FC012809D003B0BDE867
:2001C000F08F0B2201A92846FFF73CFC0128F5D199F80020DAF80010022A01F1010321D098
:2001E000A64210D2019906F18042013A081F00EB840001EB820242F8043F824203F1010368
:20020000F9D1DAF80010A61B7318BBF1010FCAF800301BD09F4205F101052BD999F80010CB
:200220000026B2E7A642EED2DDF804C006F10042013AACF1020000EB44000CEB420222F827
:20024000023F904203F10103F9D1DCE7BB42E1D199F80030022B21D004F18044019B013CE6
:200260004FF0FF3243F82420DAF800309F4205F10105D3D8012003B0BDE8F08F59F802209A
:2002800003F07F060329C3F3D415A6EB03081544B84414BF4FF4807280226EE704F10044F2
:2002A000019B013C4FF6FF72584623F8142003B0BDE8F08F1CA100202DE9F04190F83830D7
:2002C0000446032B51D8DFE803F002323B462D4BC0681978E76A03F5C252032911680CBF10
:2002E00080264FF4807601FB06F141F2C47C00EB412041F2A87841F2AC7E53F80C20E06006
:2003000053F80E0053F808502261A5EB4125A0EB4121901943F8085043F80E1043F80C009F
:20032000C4E90C205FBB6262012384F8383016480021FFF745FE012811D1022384F8383032
:20034000626B04F130010120FFF7FCFE012806D1032384F8383000212046FFF731FE431E82
:20036000DBB2012B02D9BDE8F081022094F82830062B04BF002384F82830BDE8F081921B1F
:200380002263D1E71CA10020BCB800202DE9F04FDFF8248198F80060012887B08CBF002320
:2003A0000123032E02930C460B68154639D0022E62D14FF480724FEA1329DFB201920138C0
:2003C000012823D8012203929D421AD9384E06F1880A06F11C0B32681AB1DBF8001099421F
:2003E0004ED0DAF8000000234844092205A9FFF729FB01281FD002280FD020B123689D420F
:20040000E9D82560032007B0BDE8F08F87B1FFF7A9FA022007B0BDE8F08F022007B0BDE84C
:20042000F08F80220192C3F3D41903F07F07C6E7019A0392C8E7DDE902C1059ADDF804E07F
:2004400098F80030022B14D0032BE6D152F8273023F07043B3FA83F35B0963450F44236872
:2004600023D00B4477452360EAD309F101090027C5E732F81730EDE74FF480720192D2E7A1
:200480000C490968013A02EB41224902B2FBF1F203991344B3FBF1F201FB12320AB10B4462
:2004A0009B1A9D42236096D8ABE7AB42ABD3A8E7C4B800205CB900201CA10020F0B5104D7B
:2004C0002B7841F63002022B0BBF070AC0F3D417C4B200F07F04A85883B00E4600230322B2
:2004E000384401A9FFF7AEFA012807D12B78022B019B0CBF23F8146043F8246003B0F0BD52
:200500001CA100202DE9F04390F83C30002983B0044614BF02210021042B7BD8DFE803F0C8
:20052000030C3C476900FFF74BFD012870D1626B002A75D184F83C00404EDFF80881404DA8
:200540004FF6F7771DE01FFA80F9B94594BF4FF000094FF0010901A9B9F1000F46D1FFF707
:2005600089FB0128494650D1206BFFF7A7FF01284BD1019B2A682363013B934228BF1346AD
:200580002B603378206B032BDDD1404594BF4FF000094FF00109DEE7426B04F1300100209D
:2005A000FFF7D0FD012833D1032384F83C30234BE16A41F2C47003F5C2521D5812681950B9
:2005C00041F2A87741F2AC76D8596D1A995902FB05F200EB422501EB422203F5BD5000210E
:2005E000DD519A51FFF7ECFC012811D1042384F83C3094F82830042B04BF002384F828301D
:20060000A36B8BB120469847012003B0BDE8F0830228FAD194F82830042B09D00220F4E781
:20062000022384F83C30B8E7012003B0BDE8F083002384F828300220E7E700BF1CA100209F
:2006400060B90020F7FFFF0F38B590F834300446052B46D8DFE803F01F033F101963006BDA
:200660004FF0FF31FFF72AFF01283AD1E06A002839D1032384F8343000212046FFF7A0FC1D
:2006800001282ED1042384F8343094F82830082B2DD0012038BD41F63803224DEA5800F1ED
:2006A000300102320120FFF771FE012824D00238C0B2012815D8052384F8343094F8283084
:2006C000082B04BF002384F8283041F2E5730122EA54022038BDC06A216BFFF7EFFE012868
:2006E000C7D0002038BD022384F83430F4E7002384F82830012038BD05F5C252E36811688F
:20070000D4E90B2003EB412341F644016850C4E9033002B96062012384F83430A0E7014D35
:20072000CCE700BF1CA100202DE9F04F436883B0C3F308081646002A00F0E180714B054693
:200740008946A3F1180B4FF0000AC8F5007495F91A70B44228BF3446791C28462ED0F7F73B
:20076000DDFE0BEB071341F218629B58984205D0FFF7F8F8504603B0BDE8F08F614B03EB52
:20078000472022464946404463F0ACFE002221462846FFF729FBA2440028EBD02B7E1B07D5
:2007A00006D5594B2A691B689A4201D3FFF7DAF8361BA1444FF00008C7D1DBE7F7F78AFEDF
:2007C000002849D12846F7F7A9FE6968C1F308032BBB21F4FF7323F0010303F50072AB6843
:2007E0009A422CBF062207222B7E03F00C030C2B1CD0002301A9FFF725F90128BAD10198E5
:20080000404BC31A48BF03F2FF13B3F5B05F4FEA63224FD257B2AF760028B2D1AAE72B7EB9
:2008200003F00C030C2B4FF00702E2D19BF800C0364BBCF1030F1B680CBF4FF0800C4FF495
:20084000807C03FB0CF34FEA432C0CF1FF3C0CEA0101A3EB5123CDE72B7E1A072ED59BF8B1
:2008600000102A4B95F828201B6803290CBF80214FF4807103FB01F3062A4FEA43233FF4DB
:2008800079AF23490868834230D891F83D30002B7FF470AF002A7FF46DAF6B6985F8382072
:2008A000062185F82810EB622846FFF705FD012888D05FE7FFF756F80198ACE7154B1A7880
:2008C000002A7FF457AF95F82820002A7FF452AF082185F8342085F82810D3F85F206B6935
:2008E0002846C5E90B32FFF7AFFEE0E741F2E573012250460BF8032003B0BDE8F08F92461C
:2009000038E700BF34A10020E0B800205CB90020C4B8002001B900202DE9F04390F8384058
:2009200083B00546032C00F29F80DFE804F0021A890BFFF789FE012811D002280BD10323DB
:2009400085F838302B6C002085F82800002B00F0878098470224204603B0BDE8F08385F881
:2009600038002B78022B77D0404A6F6841F64803D3581F40C7F34F272846F7F7CFFDDFF88C
:20098000F08006463F1A0AE0D8F80030013B99454AD2FFF7B5F908B9FEF7E4FF013602228A
:2009A00001A900233046FFF74DF8BC1901281FFA84F94FF400724FF000010446CBD10198B1
:2009C00063F0F1FDEB694FF400712846002BDBD06B68002BD8D1019B4FF020324FF02E0C3D
:2009E0001A605A6083F800C0C3F807204FF0100E6C6A1A625A6283F820C083F821C0C3F8C9
:200A0000272083F80BE0EA6B5C83C2F30F4CC4F30F4483F82BE09C825A87A3F834C0D8F8F7
:200A20000030013B9945B4D3C3EBC35359022846FFF766F908B9FEF795FF022385F83830AF
:200A40002B6C002285F8282063B1284698470124204603B0BDE8F0836F68C7F34F278BE7E8
:200A6000022478E7012476E7002474E71CA100205CB900202DE9F04F90F8303089B004461E
:200A8000042B00F2A880DFE813F0A900B20005008A00E800B64D41F61003EB5C002B40F082
:200AA0009A80B44F04F11C09B84607F1380BBA4601AE324649464046FFF710FA012840F031
:200AC00018810198002800F0FA800378E52B01D0002BEED1A84A821A48BF02F2FF12B2F5CB
:200AE000B05F4FEA622380F03C811B01A34A13449A7B042A0CD041F2C86104266A58013202
:200B00006A5041F2CC615A609E736B5801336B5041F60202AB565E1C09D003F5B17305EBA3
:200B20000313FF26D979AE546FF30001D97141F603016B565A1C0ED003F5B17305EB031307
:200B4000FF26DA796E54C2F34501013921EAE17161F34602DA712022002163F024FD2346A2
:200B6000019A53F8311F58685060116019899B7A93721181019B627EDA7205A84FF0DEFF7F
:200B8000BDF81430002B40F02F8144F28172019903200A82CB810A83CB8284F83000237E6C
:200BA000980600F1A9802046FFF738F92369002B00F0AE80237E03F0F70213F004032276EC
:200BC00040F0B480122A00F0BA80002384F828302046E36A984709B0BDE8F08F6548FFF742
:200BE0001DF94FF6FF720123228484F83030614F04F11C0801AE04F131093246414638465F
:200C0000FFF76CF901282FD00228E4D1584D41F60202AB56591C09D003F5B17305EB031321
:200C2000FF20D979A8546FF30001D97141F603016B565F1C0ED003F5B17305EB0313FF2004
:200C4000DA796854C2F34501013921EAE17161F34602DA71042384F830300020E36A20700C
:200C6000984709B0BDE8F08F019D0B2249462846002D00F087802B78002B00F0838095F87E
:200C80000BA01AF0080FB8D163F0B9FC0028B4D1637E8AEA0303DB0640F1C780344D41F6DE
:200CA00002016B565F1CC1D003F5B17305EB0313FF26DA796E5460F30002DA71B6E73B7818
:200CC0002F49022B4FF009025046C3D00B78002BC0D1C1E905330A708BF800304A6B0B737B
:200CE00051F8143CC1E90132FFF716FE01283FF4E0AE0228AED06EE7E0690023112205A940
:200D0000FEF7A0FE01283FF44EAF09B0BDE8F08F237E19077FF559AF154A41F2C873D15CD3
:200D200000297FF458AF0721D1544EE70023E26AA16884F828302046FFF756F84BE7626A9A
:200D4000E06AA0630421C4E90233C4E90B2284F83C30636384F8281063622046FFF75EF88C
:200D600039E7FEF7FFFD01986FF00F03BEE600BF1CA1002004B9002034A1002034B700203B
:200D80002CB90020474D41F60202AB565E1C09D003F5B17305EB0313FF20D979A8546FF33A
:200DA0000001D97141F603016B56581C0ED003F5B17305EB0313FF20DA796854C2F345014F
:200DC000013921EAE17161F34602DA71237EDA067FF540AF3448FFF721F84FF6FF7202234B
:200DE000228484F8303056E6304B05A9B3F9482C02A84FF0C1FE9DF80C309DF80D609DF8DC
:200E00000A509DF80B20BDF808109DF80E00DB0243EA461342EA4512A1F2BC7143EA500322
:200E200042EA41229BB292B2B1E6A98A6B8B204A43EA014312686362EB69A3605202B3FB5F
:200E4000F2F102FB113109B113445B1A154DE36041F6020184F819A06B565E1C09D003F5CA
:200E6000B17305EB0313FF20DA7968546FF30002DA7141F603016B56581C0ED003F5B17301
:200E800005EB0313FF20DA796854C2F34501013921EAE17161F34602DA71032384F83030A3
:200EA0007DE600BF1CA1002004B90020286200205CB900202DE9F04390F82830013B83B0DF
:200EC0000446082B41D8DFE803F048054D525865406A4300384B4668056B41F6480103F513
:200EE000C2525F5813683740EA19B2EB432F4FEA432816D258E02169207EFEF7E3FE012838
:200F000023D1256B666823696361A5EB08053D444644F61B019B6660A84525634F46236186
:200F200042D82046F7F7D6FA01AA81460028E2D06668A368E26A9E4238BF1E460023A6609E
:200F400084F828300AB12046904703B0BDE8F083FFF7E2FC03B0BDE8F083FFF78BFD03B02A
:200F6000BDE8F083FFF764F803B0BDE8F0830021FFF7C8FA03B0BDE8F0830121FFF7C2FAC4
:200F80000128E2D10023216C84F828302046FFF7BFF8DAE7FFF790F903B0BDE8F083FFF7DD
:200FA00053FB03B0BDE8F0832046F7F793FA0028BFD12E446660BCE71CA100202DE9F0477A
:200FC00082B0054602AF18461C460E46904660F0A9F8083020F00700ADEB000D0DF1080A04
:200FE000013CD14614F8013F5BB989F800304246CDF800A03146284642F0CCF8BD46BDE81C
:20100000F08718464FF070FBC3B2A3F120023F2A88BF202309F8013BE4E700BF2DE9F0471F
:2010200004460D469046002144221E46089F63F0BAFA01234FF6FF722676628384F8283075
:201040002B782E2B4CD02E4604F1310A307804F1390968B12E280BD04FF046FBC0B20AF8B7
:20106000010BCA4506F1010607D030780028F1D120200AF8010BCA45F7D130782E2808BF04
:20108000707804F1380908BF013604F13B0A58B14FF02AFBC0B209F8010FD14506F10106F6
:2010A00007D030780028F3D1202009F8010FD145F7D118F0100F14BF0323012384F819803D
:2010C0002370E7622B782E2B26D16B7823BB0323204684F83030FFF7CDFC2046BDE8F087D7
:2010E0006B78002BAFD1114B41F2F47241F60C0041F2F0719A5818585958E26041F6010207
:201100006062A1609A5C627641F2E8729B5C2370E7622B782E2BD8D00023204684F83030D5
:20112000FFF7A8FC2046BDE8F08700BF1CA1002010B5114C94F8DA3A23B9104B4FF4802219
:201140005A6110BD0E4A136823F0060313605FF0A9FF94F8DA3A002BEFD0D4F8E03A9B683B
:20116000DB07EAD5D4F8DC2B136823F0030161F307031360E1E700BF30510020003C0140F3
:2011800010ED00E008B50121032004F039F872B650F05EFB2DE9F04FCF4CDFF848938DB02B
:2011A00000270090A4F1370504F61D4A54F80B0C002800F0FE803DF091F90646002800F032
:2011C000D681D9F8843044F8073CE0260023A4F10B0B04F8033C7E4354F80B0C3DF07EF9DD
:2011E000002800F0E68054F80B0C3DF06FF914F8023C5A1E80460B2A0DD8DFE812F01F00EF
:201200003A004600530083009B00E30017013701420175018D0124280CD0009A3AB995F821
:201220002A2B824240F07E81012204F8032C0D2BD2D186E0012304F8023CCDE700234D282D
:20124000C4F8C53084F8CD3084F8CE3004D0582808D004F8023CBFE7022204F8022C84F814
:20126000C430B9E7032304F8023C022384F8C430B2E704233C2804F8023C0BD0B8F13E0FB6
:201280000CD0002304F8023CA6E70A233C2804F8023CF3D1002304F8013C9DE7012304F8F9
:2012A000013C99E7D4F8C500AB190344421CC4F8C52083F8378094F8CD00022A88EA0001AC
:2012C00084F8CD1088D12378C02BDAD86278FF2A08D1052BD5D9012384F8C430072304F8B0
:2012E000023C79E7A4F8C12000229342C4F8C93014BF0523062384F8C320C4F8C52004F807
:20130000023C69E7D4F8C500AB190344421CC4F8C52083F8378094F8CD00D4F8C93088EAE2
:2013200000019A4284F8CD107FF456AF062304F8023C51E794F8CD308342A2D10D2304F877
:20134000023C14F801CCBCF1000F40F0F180634B08940FCB04AE86E80F00D4F8C930D4F835
:20136000D100ADF82AC023440993B4F8C130ADF8283094F8C3308DF82C3001238DF82D300A
:20138000324603AB08A9CDF80CC035F001FD48B1049B059394F8C420514B049331465846DA
:2013A00030F09EFB039E002304F8023C002E40F0D6800137032F04F1E0047FF4F7AE0DB0AA
:2013C000BDE8F08FD4F8C500AA190244431CC4F8C53082F8378094F8CD2094F8CE000193A7
:2013E00088EA020284F8CD204146D5224FF034FC019B84F8CE00072B7FF4EEAEB4F8053019
:20140000C02B3FF63EAFB4F80320A4F8C120A27884F8C32000229342C4F8C93014BF082350
:201420000923C4F8C52004F8023CD5E6D522014694F8CE004FF010FC94F8CD3084F8CE0034
:2014400088EA0303D4F8C50084F8CD30AB190344421CC4F8C52083F83780D4F8C9309A422D
:201460007FF4BAAE092304F8023CB5E694F8CD30434084F8CD3094F8CE3083427FF401AF99
:2014800054E7D4F8C500AA190244431CC4F8C53082F8378094F8CE000193D52241464FF08B
:2014A000DBFB019B84F8CE00052B7FF495AEB4F80120B4F80330A4F8C120227884F8C32068
:2014C00000229342C4F8C93014BF0B230C23C4F8C52004F8023C7FE65F620020E0470708D9
:2014E00010900120402F0020D522014694F8CE004FF0B2FB84F8CE00D4F8C500AB19034432
:20150000421CC4F8C52083F83780D4F8C9309A427FF462AE0C239CE694F8CE3083427FF403
:20152000B0AE0BE7232804BF022204F8032C7EE6BCF1010F4FF0000602D004F8026C38E73D
:20154000D4F8C93008942344099308A8B4F8C130CDE90A66ADF828302CF01EFCEDE754F861
:201560000B0C33F0DBF954F80B0CB04721E714F8033C002B3FF41DAFD9F8842054F8071CA2
:20158000521A632A7FF615AF012B28D0022B7FF410AF54F80B3CC5F84C3C012285F84A2CA8
:2015A000C5F8503C0F4AC5F8583C4023C5F8542C85F85C3C85F85D0C0B48C5F820AAC5F806
:2015C000A0AC43F00DFD4FF4005035F009FA074843F0FCFC85F8A46C85F8A56CE9E6FFF76D
:2015E000D1FD00BFF9A60408D0E0070806E10708836D1B6A5B681B78FF2B0AD190F8F03086
:20160000002B03F1FF3380F8F03014BF0120022070470020704700BF826D136A5B681B78BC
:20162000FF2B08D090F8F030013BDBB280F8F0301BB10120704700207047126A52680220CC
:2016400013707047034B93F82400003818BF0120704700BFA81E0020202301480B807047F9
:20166000E4040020642301480B80704704050020432301480B8070476805002010B5074C91
:20168000D4F8C800FF2807D0054951F8042BF6F753FEFF23C4F8C830002010BDE4040020E9
:2016A00070B90020EAE700BF08B5D0F8E4355B6A9847002008BD00BF08B5D0F8E4351B6A48
:2016C0009847002008BD00BFD0F8E43510B504461B689847D4F8E8359B689847002010BD7D
:2016E00008B5D0F8E435DB6903B19847002008BD08B5042290F81211D0F8E83580F8131181
:2017000080F81221DB689847002008BD10B5D0F8E83504461B699847032384F812310020BB
:2017200010BD00BF0B0630B41CD401EB810200EBC202002300EB810582F8741382F8753363
:2017400001241A4604FA01F16D6D61F31F4201696FF3CF332B60CB6923EA0203002030BCDA
:20176000CB61704701F07F0101EB810400EBC404012200EB8105002384F81C1184F81D21D7
:2017800002FA01F11A46AD6961F30F02DFE700BF10B581210446FFF7C5FF20460121FFF712
:2017A000C1FF024B0020187010BD00BF506E002010B581210446FFF7B5FF20460121FFF731
:2017C000B1FF82212046FFF7ADFFF6F7FDFD002010BD00BF38B50D4604468321FFF7A2FF56
:2017E00029462046FFF7E4FF002038BDF0B416460A063AD401EB810500EBC5052824002273
:2018000004FB0104022B85F87413C5F87C6385F8773385F8752304F55D7448D0154600EB93
:201820008107012202FA01F17F6D61F31F45D7F800C01CF4004F11D1E488204946F08052BE
:2018400042F4004242EA834204F00F041C4B42EA845211400CEA0303194339600269D369C6
:201860002B430020F0BCD361704701F07F0101EB810500EBC5052824012204FB0104022B0B
:2018800085F81C11C5F8246185F81F31A5F8221185F81D2104F58E740CD0002500EB810795
:2018A000012202FA01F1BF6961F30F05BFE722711546B4E700252571F0E700BFFF87CC13A2
:2018C000007833EC002310B5194604464022FFF78DFF8021204600234022FFF787FFD4F828
:2018E000E835A078012284F812215B689847002010BD00BF70B44B78012B26D00B784A6954
:2019000000EB83035C6D25682369D2B18A684A6102F07F0223F4002323F07F0342F40022BA
:2019200013432361C378012B04BF0B696361C5F3076363F07B0363F31F652560002070BCCD
:2019400070478A6802F07F02E4E782694C691568136944B38E68B4428CBF06F07F0404F06C
:201960007F0423F4002323F07F0344F4002443EA040388BF4E611361C378012B1DD0C5F30F
:20198000076464F07B0464F31F651560002BD5D14B69002BD2D002690878516B01238340D9
:2019A0000B435363CAE723F4002323F07F0343F400231361C378012BE1D10B780C6900EBD9
:2019C0008300C5F30763816963F07B0363F31F654C610020156070BC704700BF2DE9F043A0
:2019E0004B78012B30D00B784C6900EB83035E6D356837691CB38B681C44013CB4FBF3F452
:201A0000C4F3090203FB02F3C3F312034B61144643EAC44363F31C073761C378012B04BFD1
:201A20000B697361CB78012B44D0C5F3076363F07B0363F31F6535600020BDE8F0838A684F
:201A40000124C2F31203E3E791F800804E6900EB880EDEF818C0DCF80050DCF8107076B33D
:201A6000D1F80890384A06EB0904013CB4FBF9F402EAC444C6F312022243CC7807F06047A4
:201A80003A43012C174649D0CCF81020C278012A55D00269516B03FA08F30B435363C5F3CD
:201AA000076363F07B0363F31F65CCF800500020BDE8F0834B7973B345F00055B5E707F0BE
:201AC000604747F40027CC78CCF81070C378012B2FD0012CE3D102699268D20554BF45F0AA
:201AE000005545F08055C5F3076262F07B0262F31F65CCF80050002B9ED1B0B203308010EB
:201B0000DEF8D04098D0CA6852F8041B216001339842F9D190E745F0805586E764F35E7769
:201B2000CCF81070C378012BD5D10A69CCF81420D1E70A69CCF81420012CB0D1CBE70B69F2
:201B4000CCF81430ABE700BF0000F81F0E4BDA68D20310D4DA68D1060FD4DA68D20510D4C8
:201B6000DA6812F0E00F0AD1DB6813F0020F14BF0820092070470120704706207047072049
:201B800070470220704700BF003C02400020704700207047104AD068A8B113699BB188424D
:201BA0000FD88B4234BF00230123DBB243B193695161994204D0094B9161142083F8CC0098
:201BC00070470023F1E7A1F59C53083BB3F57A7F2CBF00230123E9E770B90020E404002097
:201BE000054B5A7F19778A4204D0044A5977142082F8CC00704700BF70B90020E40400202D
:201C00007047704728B1034B987F012894BF00200120704770B9002008B5FFF7F3FF50B1B5
:201C2000054AD37F127F5B0003F00203002A18BF43F001030B6008BD70B9002008B5FFF7BB
:201C4000E1FF10B1014B1B6A0B8008BD70B9002070B5FFF7D7FF50B10A4A958C35B1966A2C
:201C60000023B3421C4603DB002000E00D7070BD02EB44040133A48DAC42DBB2F1D10B7010
:201C8000F5E700BF70B9002008B5FFF7BBFF10B100230B70137008BD0420704728B1034B4A
:201CA00093F9CE00003818BF01207047E404002008B5FFF7F3FF50B1054B93F9CE20012A40
:201CC000C3BF93F8D130C3F340030B60002008BDE404002008B5FFF7E1FF18B1024B93F871
:201CE000D0300B7008BD00BFE404002070B5FFF7D5FF38B10E4C94F8D130DB0703D5002341
:201D00000B70137070BD0B4D94F9CF3095F83C6093FBF6F301330B7094F9CF4095F83C10F0
:201D200094FBF1F301FB134301331370EAE700BFE404002070B900200320704770B50A4AF3
:201D400092F8403006255E1CB6FBF5F405FB146492F84150AC4205D002EBC303C3E9110183
:201D600082F8404070BD00BF70B90020002230B504461046914200DC30BDA35C082558402D
:201D800010F0800F4FEA400318BF83F0D503013DD8B2F5D10132EDE710B5D9B10E4B586F12
:201DA000814217DCB2B1DB6B9A4213DC0B4C013A013903FB012184F8DC1004F1D8000521B2
:201DC000FFF7D4FF062184F8DD0004F1D800BDE81040B3E710BD00BF70B90020E404002081
:201DE000024B93F878300B600120704770B90020024BB3F87A300B800120704770B9002089
:201E0000024B93F87C300B700120704770B9002000230B70012013707047003818BF012079
:201E200070470120704770470023038083708380C3800381704700BF074A084992F87D30AA
:201E400009780133DBB2994282F87D3004BF002382F87D30704700BF70B9002080060010DC
:201E6000F8B5794CD4F8803083B1784B1B6893F82E305BB1764B94F88420A3FB0013012A38
:201E80004FEA931330D0022A08D002B1F8BD714B9842FBD9012384F88430F8BDD4F8882010
:201EA00064329A423ED894F87D3004EB031393F8FC24FF2A06D068490132012083F8FC2412
:201EC00081F8DE00FFF7B8FF644B1B780122092B84F88420DAD1B4F87E35614A01339BB20F
:201EE000A4F87E355380F8BD94F87D105B48C4F888308C2303FB0143007883F89E20002316
:201F000084F89A3004F190050A2202230928C4F88C5084F89B2084F88430B7D1504B01311B
:201F20001980F8BD94F89A2094F89B309A42ADD104F18F0004F19805002310F8012F0821C2
:201F400053405A0013F0800F08BF5B0082F0070214BFD3B2DBB20139F3D18542EDD194F871
:201F600099209A4239D194F87D6094F8975094F89830B4F89300B4F8952094F891C004EB26
:201F8000061743EA052394F8925087F8FC1440BA52BA81B292B245EA0C202F4DC7F80015AA
:201FA0001BB294F99010C7F80425032E4FF00102A7F8FE04A7F8083587F8FD1485F8DE2044
:201FC00008D8264A12780C2A29D00D2A02D1244B23F81610FFF730FF5CE794F87D3004EBAE
:201FE000031393F8FC24FF2A06D01B490132012083F8FC2481F8DE00FFF71EFF174B1B786F
:020000040801F1
:202000000122092B84F884207FF440AFB4F87C35134A01339BB2A4F87C359380F8BD11493D
:20202000114A91F822100E4803EB830303EB830349089B0093FBF1F382FB0312DB17C3EBBC
:20204000A20320F81630C5E770B9002024130010D34D62103F4B4C00E4040020E459002074
:20206000E85900206C300020676666660B4B93F89A1093F89B2091420ED010B493F89A201F
:20208000D3F88C40511CD2B2C0B2C9B283F89A10A0545DF8044B7047704700BF70B9002098
:2020A000FD2870B522D0F02804D0EF2822D00224204670BD114D0320052641282E444FF070
:2020C000000405F1010580F080030DD0042B0BD9FFF7E6FF2044B542C4B2E9D015F8010B9F
:2020E000412880F08003F1D10420F3E7044D0B200426E2E7034D0C200626DEE798E1070860
:20210000A0E1070890E107080F4B104AD3F88035B2F900005B0707D400EB8000400080B2B6
:2021200000F5C87080B27047094B0A4AD3F8C430323382FB0312D817C0EBA20080B200F5C8
:20214000C87080B2704700BF70B90020002F00100C4B00206766666600B5062983B00A46A0
:202160004FF03203014628BF06220DF101008DF8003062F0B7F9044B6846D3F8843598477F
:2021800003B05DF804FB00BF70B900205E2810B511D05D2805D00D4BBDE81040D3F88835D5
:2021A00018470A4CD4F888359847D4F888353D20BDE810401847054C5D20D4F88835984792
:2021C000D4F888353E20BDE81040184770B9002070B5094E0546D6F888355E200C4698477A
:2021E000D6F8883528469847E0B2FFF7CFFFC4F30720BDE87040C9E770B9002003682DE904
:20220000F041002B3D4D3E4F3E4EB8BF5B42A5FB0321890D07FB0137C7EB0717BF0096F8FA
:20222000923585FB0725FA170446C2EBA555002B57D101EB810101EB810105EB810109B2CD
:20224000DFF8BC801320FFF7C3FF2F4908FB057581FB0531ED17C5EBA11109B21B20FFF787
:20226000B7FF2368254D002BB4BF53214E212320FFF7AEFF636896F8922583EAE376A6EBDD
:20228000E376A5FB0631890D08FB0168C8EB08184FEA880885FB08354FEAE873C3EBA55577
:2022A0002ABB01EB810101EB810105EB810109B21220FFF78DFF124B134903FB058581FBBF
:2022C0000531ED17C5EBA11109B21A20FFF780FF6368002BBDE8F041B4BF57214521222099
:2022E00076E7C1EB011105EB810109B2A8E7C1EB011105EB810109B2DAE700BF6BCA5F6B9D
:20230000806967FF70B90020D34D621007B50DF1060211F037FA68B1084BBDF80620B3F8AD
:20232000B0159A84914205D00549A3F8B025142081F8CC0003B05DF804FB00BF70B90020CC
:20234000E404002013B50446FFF7A8FC08B300230DF106022046ADF8063011F013FAC0B125
:202360000D4C9DF8062094F9CE1084F8E320032908BF62F07F024FF00501084808BF84F8C1
:20238000E320FFF7F3FC062184F8E4000348FFF7D5FC02B010BD00BFE4040020C30500208E
:2023A00008B5044BD3F8B4053CF098F8B0FA80F0400908BD70B900202DE9F04F204B85B06B
:2023C0004FF0000804461E2093F800A093F801B09D78B3F80490DF881E7ACDF80480ADF886
:2023E0000C8026F07BF818B117B1B9460125C246144A92F8B835D9070AD492F8BF253AB916
:20240000012E1BD0022E03D113F0020F08BF01258DF80C608DF804A08DF805B08DF806506E
:20242000ADF80890ADF80A7001AB03CB1B88206020466160238105B0BDE8F08F3546E7E7B6
:20244000B86D002070B90020144B30B4D3F8E44514B300220F2583F8EA15090A83F8E905A4
:2024600083F8EB15C3F8EC25C3F8F025C3F8F42583F8E85503F5BD60012110F8015F0131E8
:202480002A440E29D2B2F8D183F8F6252046044930BC10223BF0F2BF30BC704770B900201B
:2024A00058BF0020034B002183F8F815C3F8FC15CAE700BF70B9002013B50446262001917F
:2024C00026F00CF8019920B9204602B0BDE81040BAE702B010BD2DE9F743B74CD4F8E4350A
:2024E0000D464BB14FF0020800264FF00109D4F8E4053BF0F3FF58B90027A37F042B00F288
:202500005781DFE813F08F00E400F7003D014601D4F8E4053BF0DAFFD4F8FC355A1C234497
:20252000C4F8FC2583F8000694F8F835012B0AD0022B11D0002B70D10F280CBF84F8F895F9
:20254000C4F8FC35D3E7A0F17203012B01D9762863D184F8F885CAE7102AC8D19749002376
:20256000012211F8010F013203440E2ADBB2F8D194F80E2684F8F8659A42C4F8FC65B6D1FE
:2025800094F80F36002BB2D194F80176732F37D0762F0DD0722FAAD194F8032694F80236F9
:2025A00053EA0223A3D0E360B4F804362361A4E794F8032694F8023653EA022397D094F840
:2025C000051694F8042694F80906236242EA012294F80616E17794F8071684F8121694F8E2
:2025E0000816A4F8102641EA0021A4F81416616901B96361A38C002B7FF47FAFA2847CE70D
:2026000094F8072694F8063643EA02231AB2002B3FF46DAFA4F816266FE784F8F865C4F8DE
:20262000FC6564E7722F44D10123A3770022644B1B78402B2FD1634E94F812C6A08CA37FC8
:20264000B4F810E6338005024FEA0C33217F778005F4706503F440532B434FEA0E1543EAC0
:202660008133EDB22B43276A65691BB2BD4214BF0825002513432B43704514BF04200020B9
:202680001843514B614514BF0221002193F8CC30F3800143B180636F1BB1A36A002B40F011
:2026A0009D804A494A481F2203B0BDE8F04361F0B8BFD4F81836474AEB1A934201DC0022C0
:2026C000B5E77220FFF7EEFEC4F81856F7E7762F03D10223A3770022A9E7D4F818363D4AD7
:2026E000EB1A9342EBDD7620FFF7DCFEC4F8185600229CE7344ED4F8183696F8CC20EB1AE8
:2027000082B3344A934230DDE27FD2071BD46169226A91420ED089B24620FFF7CDFE96F804
:20272000CC30C4F81856013B86F8CC300423A37701227CE7A18CB4F810268A4203D05020D8
:20274000FFF7BAFEEBE7217F94F812268A4206D0B1FA81F149094920FFF7AEFEDFE714227D
:2027600086F8CC201C4A9342BDDC762FA7D17320FFF798FE0323A377C4F81856002256E716
:20278000732F9CD0D4F81816124B691A9942A0DC95E7D4F818360F4AEB1A93428FDD76202F
:2027A000FFF780FE0223A377C4F8185600223EE70023A3771A463AE770B9002070BF00209F
:2027C000E4590020E8590020E40400200BE10708C90500203F0D03003F420F00334DD4F81F
:2027E0001C662A2385F8E5300DF1020220230DF10101304685F8E63011F05BF830B19DF860
:2028000001109DF8027051EA070339D1552385F8E730462385F8E830202301A9304685F867
:20282000E93011F040F80346214813B1BDF804209ABB20494EF0A6FEB4F814761E4D87B37C
:202840000DF10301304611F031F850B39DF803100DF10602304610F095FF10B3BDF806207D
:2028600016493B46BA420CBF20222A2228464EF089FEB4F81636A4F8203603B0BDE8F0833B
:20288000304610F0FBFF394685F8E700304610F0E1FF037885F8E830BEE709494EF072FEDA
:2028A000CAE7084928464EF06DFEE2E7E4040020CE0500202DE10708D205002025E1070812
:2028C000FA2208082CE1070838B50B680E4D5A1C0A6005221A700B6895F8CE200C46591CAF
:2028E00021601A70236895F8D120591C21601A70B5F8D41020464DF0F1FC236895F8D62015
:20290000591C21601A7038BDE40400202DE9F0472DED028BFFF7C2F9C8B31E4B93F9CE0057
:20292000012834DD93F804411B4F9FED1C8A15468E1E02EB44084FF03209454504D1BDEC2F
:20294000028B2046BDE8F08737F802AB26F802AF07EE90AAF8EEE70AB2EE040A60EE880A29
:2029600060F0F8FBBCEEC00ABAF10E0F10EE103A9BB209D91933B3FBF9F39BB203EB8303BA
:2029800003EB83035B009BB225F8023BD5E70024D5E700BFE404002092BF0020CDCCCC3D4B
:2029A00038B50D46FFF77AF9044638B10C4890F8D130DB0704D5B0F8D2002880204638BD26
:2029C000084A90F9CF3092F83C2093FBF2F102FB11320132013100F5847010F0E7FEECE780
:2029E000E404002070B9002038B5134C94F8413094F840209A4219D004EBC3030F49D3E9C3
:202A000011200023984212DC93780D4AC4F834065B081370FCF77AF894F84130062101339F
:202A2000B3FBF1F201FB123384F8413038BDD55C01F8015B0133E5E770B90020C26D0020C4
:202A4000F06D0020A1F5AF53B3F5AF7F10B51BD80E4BA3F87A104FF47A7303FB01F4002012
:202A60004FF4C87154F0F8FF2821B4FBF1F101F03F014FF420630120B4FBF3F441EAC41117
:202A8000BDE8104054F0E8BF10BD00BF70B9002013B500230DF106020C46ADF8063010F063
:202AA00071FE30B1044B9DF8060083F87C4055F04FF802B010BD00BF70B90020194B37B542
:202AC00093F8782004461D4651B13AB9D3F83806012283F8782008B13EF07EFE03B030BDEF
:202AE000002AFBD0D3F8380683F8781008B13EF06DFE4FF4AF703AF0ADFF95F97C1000230E
:202B00000DF106022046ADF8063010F03BFE9DF8060055F01DF8B5F87A102046FFF792FF1C
:202B2000DCE700BF70B900202DE9F04FAC4B1B788BB08146002B40F0BB80AA4ED6F81C561B
:202B4000002D00F0B580A84AD2F80C4104F0F021B1F1E02F6FD1C2F80C31D6F83C26944227
:202B600069D004930593ADF81830A04BC6F83C469A881F78ADF8142093F801C01A7A93F8D8
:202B800002A08DF810700DF110088DF811C08DF812A08DF8182098E807000DF11C0EAEE8E9
:202BA00003009349AEF80020C4F34252895CC4F303428F4202F101021F4601D1944508D095
:202BC00028468DF81C108DF81D2010F0EFFDADF82000284611F0ABF8032804F0070B37D019
:202BE000042839D001283BD1824B13F80B309A4501A9284618BF8DF81E3010F051FE48B16F
:202C0000019BC4F3001103F001038B4202D0284610F044FF0A2207A9404661F09CFC50B1BD
:202C20009DF81E30BDF81C20BB703A80BDF82030BB804EF069F996F840A6DFF8B0B104AF9C
:202C400096F84036032B7DD8DFE803F00C3578A5694B13F80B30CAE7684B13F80B30C6E784
:202C60000023C4E73946284610F020FE044658B107A8FFF7A1FB9DF81E109DF810308B4282
:202C800060D0284610F0B6FF96F84036013303F0030386F840360CB99A45D1D196F8B835FB
:202CA000DB0700D524B12B6849461B68284698470BB0BDE8F08F01A8FFF77EFB96F8B885D4
:202CC0009DF8044008F00108ECB1B8F1000F39D13A460DF10301284610F0EBFD044688B35E
:202CE00007A8FFF769FB9DF81C109DF803309DF81D208B4203D19DF81030934222D02846C5
:202D000010F082FFC0E7B8F1000FBDD13946284610F0C9FD0446A8B107A8FFF74DFBBDF84D
:202D20002010BDF810308B420CD086F8418686F842862B6828469B699847A5E796F8B8354F
:202D4000D80701D500249FE707A9284610F0A8FD04460028F6D01E2025F0C0FB96F8433604
:202D600083428046EED086F8430660B1BBF80630002BE7D1079BD907E4D40121284610F09C
:202D80008DFE444680E7079BDA07DBD50146284610F084FE78E73846FFF70EFB97E80700EB
:202DA00007AB03C31A809DF810309BB10DF11D0207A9284610F07DFD0DF11E01284610F0A0
:202DC00075FD0A2207A9384661F0C5FB041E18BF012459E708A9284610F065FDECE700BFA5
:202DE000726E002070B90020E4040020B86D0020CCE10708C0E10708B4E10708A8E1070895
:202E0000024B0146D3F844063BF06CBB70B900202DE9F041FD2984B0044600F0DD80F0291D
:202E200000F0BC80EF2900F02F814AB10346861803AD002003F8010B9E4205F8010BF9D142
:202E4000994B0B2003F1090501E013F8010F814200F0C780AB42F8D14B1E832B00F292809A
:202E6000DFE813F03001370184004101AF01B501480153015F0190009000650165016501A4
:202E80007B017B017B015F019000900086018E0190009000900090009000900090009000A8
:202EA000900090009000900090009000900090009000900090009000900090009000900012
:202EC0009000900090009000900090009000900090009000900090009000900090009000F2
:202EE00090009000A4019000900090009000900090009000900090009000900090009000BD
:202F00009000900090009000900090009000900090009000900090009000900090009000B1
:202F2000900090009000900090009000900090009000900090009000900090009000900091
:202F4000900090009000900090009000900090009000900090009000900090009000900071
:202F600090009000900090001D011D014F4B93F89715002900F0628101922DF033FD019A8D
:202F8000ADF80C003AB1224403AB13F8011B04F8011BA242F9D104B0BDE8F081444F032113
:202FA0004FF00508B844002501370CE0FFF778F8064660193246FFF72BFF70194745C5B231
:202FC000E9D017F8011B412981F08003084601D0042BEBD80426ECE7364F0B214FF00408A5
:202FE000E0E7324BD3F8800580060CD4002AD2D0224403AB13F8011B04F8011B9442F9D118
:2030000004B0BDE8F08193F84806870741D52A4D287D052834BF02260326142916D97C39FB
:20302000C8B20628E2D80629E0D801A050F821F01532010815320108FF310108ED2F01084F
:20304000253201081F3201082B3201080929CDD90A390A29CAD801A757F821F0E531010839
:2030600031320108ED2F0108ED2F0108ED2F0108ED2F0108ED2F0108ED2F0108ED2F0108E1
:20308000F7310108153201080C4F0C214FF0060888E7094B0B29187DA8D10126C9E0084BB2
:2030A000D3F8C03003936DE784E1070870B9002098E10708A0E10708A46C002090E10708E6
:2030C0000C4B00200192FFF71FF8019AADF80C0058E76A4BD3ED037AFDEEE77A17EE903A41
:2030E000ADF80C304EE701922DF07CFC019AADF80C0047E7624D95F8B835DE0700F1A780F2
:20310000B5F87036ADF80C303CE75D4B5D49B3F9943681FB0301DB17C3EBA103ADF80C30EF
:2031200030E7574BB3F89636ADF80C302AE7564BDFED566AD3ED017A0C39C9B203EB8103D3
:2031400093ED137A67EEA67A67EE877AFDEEE77A17EE903AADF80C3014E7494B03EB4101DC
:20316000B1F8723603EB83035B00ADF80C3009E7434B93F8B83503F00103ADF80C3001E798
:203180003F4BB3F88C16CD055ABFCB4303F00103032311F0440F18BF042311F0020F18BF07
:2031A000072311F4806F18BF0923ABE70192FEF7ABFF374B019AD3F8C83043EAC04003908A
:2031C000E0E62F4BD3F88036ADF80C30DAE62C4BB3F87016002934D001922DF01BFC019A56
:2031E00080B2CDE62B8A03EB830303EB83039B00ADF80C30FAE6EB89ADF80C30F6E6EB894C
:20320000244903EBC3039B00A1FB03135B09ADF80C30EBE6B3F84A36ADF80C30E6E66B687F
:203220000393E3E62B680393E0E6AB680393DDE6F6B28DF80C608DF80D00D7E6B3F84C06EF
:203240009EE6D3F8880680F3100080B298E605F25465019225F0A8F9D5ED037A019AFCEEA1
:20326000E77A17EE903A9BB200287FF44BAF0A49096811F0100F18BF002343E7C4BF002091
:2032800070B9002067666666002F001000007A440C4B00201F85EB51146C002070B5214DC5
:2032A00095F89836EA181C4692F89C268AB11E4E09225C1CA6FB04135B0803EBC303E31AED
:2032C000E918DCB291F89C1609B1013AF1D185F8984602681549561C06600C261670026850
:2032E000561C0660002616700268561C066003EB430603EB8603147019440D224CF082FF8D
:2033000095F89816084B4A1CA3FB02035B08294403EBC3030120D31A81F89C0685F898361E
:2033200070BD00BF70B90020398EE33818C000202DE9F04FC31D85B0544C03F4FC7300AF5F
:20334000ADEB030DD4F8203704F5E66B0DEB00025B4506468A46FA60E9462FD094F8701806
:2033600094F871C8D4F8245701F00F0040EA4C1001310DF101088DF8000084F87018C7F83A
:20338000088007F10800ED1AA2EB0808A845194644DD2A464CF036FFD4F82027B968C4F8C3
:2033A00020B72A44A1EB09014846C4F82427C9B2D04700201437BD46BDE8F08F94F870C8B5
:2033C00094F87108B4F92A570CF00F0141EA401141F01001002DC9B2D4F82457B8BF41F059
:2033E00080010CF1010C012884F870C889F80010A5EB0B0822D1B8F1FE0F3ADDFF2394F8C3
:20340000282789F8013007F1080009F103031FFA88F1786089F80220BB6020E042464CF0BF
:20342000F1FED4F82027424448463146C4F82027D04701201437BD46BDE8F08F94F82C3763
:20344000B4F8281789F8013007F1080009F102037860BB604CF042FF78681FFA88F14CF0B2
:203460003DFFD7E90282D4F82457D4F82037786889E794F8281789F8018009F1030889F8BF
:203480000210C7F8088007F108007CE770B9002001297FD9F0B50378654CC3F34115032D98
:2034A00083B084F8715803F00F0700F0848013F01003164606D0012D6ED0052912D80020AB
:2034C00003B0F0BD94F84429002AF8D094F84529013202F00F02BA4255D0184684F84439F9
:2034E00003B0F0BD437884F840394388A4F83C3985884318811DC02D7ED84E4AC4F83429E6
:2035000015444FF0000C0120C4F83859A4F83EC984F84409AA1A5B1A934284F8457966DBA4
:20352000454D002A5CD1B4F93C39FA2B53D0414A4249D4F83439D1F81001C4F83429294687
:20354000151FA2F5A276C4F82457C4F838390025A2F5AA7201ABC4F8206784F84459C4F888
:203560002857019533F014FC013058D0019B0BB100209847D4F82037C4F824370120C4F83C
:20358000206703B0F0BD4318D4F83859D4F83429411CBFE700207047022990D04578837846
:2035A000A4F83C39FF2D1FD1042988D94318B0F80350411D9FE70023214984F8303704F5AD
:2035C000E66204F23173C4F82817C4F82027C4F82437012074E7002EA9D005233370A6E779
:2035E00028464CF00FFE9EE74318C11C83E712481A464CF007FE62E7124BB4F83C09C4F89F
:203600002037032101334FF6F672A4F82807C4F8243784F83017A4F82A27012050E7D4F898
:2036200020370222591CC4F820171A709EE700BF70B90020E4C10020A4C20020E40400203D
:203640000000F6FFA0C000202DE9F0416A4ED6F81C7684B0044638460D4610F068FB86F866
:20366000460957B10DF1090202A9384610F021F9002840F0838096F846090023ADF808306F
:203680008DF80A301A46431EDBB20021FF20FD2B8DF80C20ADF80E108DF80B0003D90020B5
:2036A00004B0BDE8F0819DF80830042B00F09D80052B00F09D80032B00F09C80022B00F0A3
:2036C0009380012B08BF042100F08F809DF809309DF80A10D6F81C06013B0DF10E028DF884
:2036E000093010F04FF896F84639032B7AD0042B76D0012B64D0D6F84829029B3F4F9A42AA
:203700000DF108084FD023680D22591C21601A7023680022591C21601A7023689DF80820CD
:20372000591C21601A7023689DF80920591C21601A7023689DF80C20591C21601A702368E9
:203740009DF80A20591C21601A70BDF80E1020464CF0C4FD23689DF80B20591C216020464D
:203760001A700721FAF7BCFB98E8030087E803000120C6F8505904B0BDE8F08101A9384680
:2037800010F08EF800283FF476AF38460DF10A0110F08CF800283FF46EAF019B96F8460927
:2037A00003F001026FE77A68D8F804309A42AAD1D6F85039124AEB1A93427FF670AFA2E7D6
:2037C000104A9DF80A000121002304E00133082B91D012F8011F8142F8D38DF80A308AE717
:2037E000094AEEE7094AECE703218DF808106DE70121FAE70221F8E770B90020B8C200207E
:2038000080841E00C0E10708A8E10708B4E107082DE9F0412A4C2B4AD4F88036B4F854796D
:20382000B4F8886682FB0352DB17C3EBA2031FFA83F8474582B00D4603D1B4F85639B3422E
:2038400033D002680190511C34230160137002680023511C0160137041464CF03FFD01984C
:2038600031464CF03BFD019847F6FF714CF036FD019847F6FF714CF031FD019847F6FF71B2
:203880004CF02CFD019847F6FF714CF027FD01980221FAF725FB0120A4F85489A4F856695B
:2038A000C4F8585902B0BDE8F081D4F85839064ACB1A9342C5D8002002B0BDE8F08100BF28
:2038C00070B900206766666680841E00026810B57F21541C0460117002680024511C016064
:2038E0000E211470FAF7FCFA012010BD2DE9F04FC24B1B68804613F0800083B000F07181FD
:20390000BF4B93F8480610F0020000F06A81DFF810B39BF81430052B40F26881DBF8003028
:20392000B84D0093002BB8BF5B42A5FB0342B648B649920D00FB0233C3EB03139B0085FB20
:20394000034502EB8202DC1702EB8202C4EBA55400FB043304EB8204A4B281FB0321DB1713
:20396000C3EBA111BCB10025A94F2E46A7FB0432D20802EB8203A4EB4303E8B2A4469BB21F
:2039800080008340BCF1090F94B246EA030605F10105EBD8340489B2B9B100259C4F2E4680
:2039A000A7FB0132D20802EB8203A1EB4303E8B28C469BB280008340BCF1090F91B246EAE0
:2039C000030605F10105EBD83443DBF804E08D4D8D4E8E498EEAEE70A0EBEE70A5FB0032D4
:2039E000920D06FB0200C0EB0010830085FB035002EB8202DD1702EB8202C5EBA05506FB98
:203A0000053305EB8205ADB281FB0321DB17C3EBA111C5B10020DFF8F8C10646ACFB053256
:203A2000D20802EB8203A5EB4303C7B2A9469BB2BF00BB40B9F1090F95B246EA030600F1C2
:203A40000100EBD8350489B2C1B10020DFF8C0C10646ACFB0132D20802EB8203A1EB430300
:203A6000C7B289469BB2BF00BB40B9F1090F91B246EA030600F10100EBD83543DBF8083081
:203A8000634A0193002B1846B8BF5842A2FB0030604E6149030AA6FB0363DB0901FB03F13E
:203AA000C1EBD00189B2B9B1002691463746A9FB0132D20802EB8203A1EB4303F0B28C4601
:203AC0009BB280008340BCF1090F91B247EA030706F10106EBD8B9B2BBF81070DFB10026FE
:203AE000DFF82CA1B446AAFB0732D20802EB8203A7EB43035FFA86F938469BB24FEA8909B8
:203B000003FA09F3092897B24CEA030C06F10106E9D81FFA8CF7BBF812303D4AA2FB030670
:203B2000F608632E28BF6326092B63D9002093468146ABFB0632D20802EB8203A6EB430355
:203B40005FFA80FAB4469BB24FEA8A0A03FA0AF3BCF1090F96B249EA030900F10100E8D886
:203B60005FFA89F9009B019A002BCCBF392338231616BEF1000F26F07F0635DD274A334349
:203B8000964543F00206C8BF43F00606D8F800301622581CC8F800001A70D8F80030002231
:203BA000581CC8F800001A7040464CF097FB214640464CF07BFB294640464CF077FB40462B
:203BC00039464CF08BFBD8F800305A1CC8F8002083F80090D8F800305A1CC8F800200120CC
:203BE0001E7003B0BDE8F08F1E43CFE7002003B0BDE8F08F4FF00009B4E700BF146C002010
:203C000070B900206BCA5F6B806967FFD34D6210CDCCCCCCC55A7C0AA0860100FFC99A3BE1
:203C2000A46C00202DE9F047AB4B1B68064613F0800084B000F09E80A84B93F8480610F0B1
:203C4000020000F09780A64F397D052940F29780632900F292800024DFF898C289B22546AE
:203C6000ACFB0132D20802EB8203A1EB4303E0B28E469BB280008340BEF1090F91B245EA1D
:203C8000030504F10104EBD8EDB2BB68954A82FB0312D917C1EB623189B2002900F0188110
:203CA0004FF0000CDFF84CE26446AEFB0132D20802EB8203A1EB43035FFA8CF088469BB220
:203CC00080008340B8F1090F91B244EA03040CF1010CEAD8E4B2FB8983494FF4F36707FB17
:203CE00003F7A1FB0737C7F38F1742F20F739F4249D8CFB10020DFF8FCE18446AEFB0732D8
:203D0000D20802EB8203A7EB4303C1B2B8469BB289008B40B8F1090F97B24CEA030C00F12D
:203D20000100EBD81FFA8CF7704BD3E9002313433ED14FF0FF3833681722591C31601A704A
:203D400033680022581C306039461A7030464CF0C5FA414630464CF0A9FA33685A1C3260A9
:203D60001D7033685A1C326030461C700621FAF7B7F8012004B0BDE8F087992585E700200F
:203D800004B0BDE8F0870021DFF868C10F46ACFB0302D20802EB8200A3EB40039BB28B40FF
:203DA0000431102947EA030793B2F0D1BFB2BBE701A84CF0C3FE9DF80810002900F08A80CB
:203DC0004FF0000CDFF82CE1E046AEFB0132D20802EB8203A1EB43035FFA8CF089469BB2A3
:203DE00080008340B9F1090F91B248EA03080CF1010CEAD84FEA08289DF80910E1B10020A9
:203E0000DFF8F0E08446AEFB0132D20802EB8203A1EB43035FFA80F98A469BB24FEA89097D
:203E200003FA09F3BAF1090F91B24CEA030C00F10100E8D848EA0C089DF80A104FEA08282E
:203E4000E1B10020DFF8ACE08446AEFB0132D20802EB8203A1EB43035FFA80F98A469BB29A
:203E60004FEA890903FA09F3BAF1090F91B24CEA030C00F10100E8D848EA0C08BDF80C304A
:203E80001B49632BA1FB03214FEA08184FEA51117FF651AF0020DFF85CE08446AEFB01322E
:203EA000D20802EB8203A1EB43035FFA80F98A469BB24FEA890903FA09F3BAF1090F91B22B
:203EC0004CEA030C00F10100E8D848EA0C0832E70C4600E788468FE7146C002070B9002026
:203EE000A46C002089B5F814D34D6210D0C200201F85EB51CDCCCCCC08B5A0F10103B3FAF4
:203F000083F302284FEA531301D0184608BD0F2024F056FA30B9064B93F8B83503F0010332
:203F2000184608BDBDE808400F2024F0D7BA00BF70B9002030B5104A104B8DB0014682F8FD
:203F4000F01002F15800069302A900230DF107050124CDE9073302938DF8143009938DF811
:203F600028300B93CDE9035440F008F8F5F78AFC9DF807000DB030BDA81E0020F115010861
:203F800008B5F5F77FFC0A2039F00CFB024B186EBDE808403DF020BCA81E0020014B1B6825
:203FA0001B6A1847FC610020024B186808B1836918477047FC610020024B186808B1436969
:203FC00018477047FC61002010B5074C606D40B13EF098FE94F8513013B180F00100C0B200
:203FE00010BD012010BD00BFA81E002010B5FFF7EBFF0E4C48B194F82430032B10D8237ED2
:020000040801F1
:204000000133DBB2072B237603D9002384F8243010BD074A01231268626184F8243010BD29
:20402000044840F051F9A4F85C00E8E7A81E0020C42F0020801A060030B40A490A480A784F
:20404000531CDBB20525042B00EBC20400F8325008BF00234FF404520B7062604FF0FF30B2
:2040600030BC70471C6E0020206E0020037870B4FBB10446C0F10106A31914F8015FDBB243
:20408000002DF9D101335B00DCB2032513800C704D7004785CB1022300255A1CD2B2CC542B
:2040A0008D5410F8014F0233DBB2002CF5D170BC704702242346E8E70B0617D401EB810366
:2040C00000EBC30310B400EB81000124002283F8764383F8741383F87523426D5DF8044B1C
:2040E000136843F4001300201360704701F07F0101EB810300EBC303012200EB810083F815
:204100001C1183F81E2183F81D2182691368002B01DA43F0804343F4001313600020704709
:2041200070B501F07F0505EB850400EBC404282101FB05010126C4F830310023C4E94A22EE
:2041400084F81C5184F81D61C4F8343101F58E711DB9FDF7CFFB002070BDFDF73FFC002036
:2041600070BD00BF2249F8B5D1F868390F2B04D05A1CC1F868290020F8BD1E4C2578002304
:20418000C1F86839002DF6D11B4E1C4B3268B2F5006F17D01B689A4227D017D9C2F500630A
:2041A000402B15D9403B02F14005C1F86C3901232370356092B2402311490A448121FFF762
:2041C000AFFFD8E71B6835607BB12A469B1AE7E74FF0000502EB0307C1F86C590CBF022194
:2041E0000121376092B22170E6E700232370C2E770B90020BC270020A4270020A8270020DF
:20420000C0270020AEE700BFF8B51D4C2378012B03D0022B09D00020F8BD01461948D0F848
:204220006C3953B923700020F8BD00231A468121FFF776FF00232370F5E7402B11D9124C90
:204240002268403B02F14005C0F86C39256092B240230E4C084622448121FFF761FF002072
:20426000F8BD094D2A684FF0000603EB0207C0F86C6908BF02202F6092B208BF2070E8E7F6
:20428000BC27002070B90020A4270020C027002038B5134602250A46C0E94E3380F811511F
:2042A0000021FFF73DFF002038BD00BF10B50C7814F0600413D0202C0AD14B78023B092BE8
:2042C00018D8DFE803F01B21171717171717272E22490122FFF7DCFF0024204610BD4B78A0
:2042E000062B24D00A2BF3D01D4B8A78C3F87829204610BDFAF740FC0224EEE719490122FB
:20430000FFF7C6FF0024E8E717490122FFF7C0FF0024E2E74B88124A1B0AC2F874390024EB
:20432000DBE70F4B8A78C3F870290024D5E74B881B0A222B0CD0212B04D021462246FFF725
:20434000A7FFCAE7CA880949092A28BF0922F6E7CA880749362A28BF3622F0E7E8C200205E
:2043600070B90020E4C20020E0C2002042060020F805002038B501EB810400EBC4040D4683
:20438000002184F87453C4F88C1384F87513C4F88833C4F88023C3782821012B01FB0501D2
:2043A00008BFEDB201F55D7108BFC4F884231DB9FDF7A0FA002038BDFDF710FB002038BD1C
:2043C000144B9A6870B5044662B1134A1B7B92F87C592B4316D081212046FFF76DFE022DBC
:2043E00009D070BD0C4B93F87C5981212046FFF763FE022DF5D12046064ABDE870401F235F
:204400000121B7E70121FFF757FE20468121BDE8704051E6FC6D002070B9002070B5094A91
:20442000094D1173094B13600021044629700D238121FFF775FE2046054ABDE870401F2350
:20444000012197E75C6E0020506E002055534253FC6D002010B5064B597B0446FAF79AFB74
:20446000002800DB10BD20460121BDE81040D5E7FC6D00202DE9F041314D2C7834B1012C2F
:2044800001D1FFF7E7FF0020BDE8F0812D4FDFF8D080B0F8B4337A68C8F804201F2BBA68D4
:2044A000C8F80820064606D1274B3A689A4202D1797B01291AD9254A25491378052401F893
:2044C000334001EBC3000133DBB2042B08BF00234FF4005113701F4B41600222304683F8A9
:2044E0007C29FFF76DFF0020BDE8F081BB7B013B0F2BE0D8FAF74EFB002819DB2B78013BE6
:20450000022BC0D9144B1988B1B1BB68D8F8082088F80C408B4228BF0B46D11A0424C8F8B4
:2045200008100E4A2C7030468121FFF7F9FDAAE73046FFF745FFA6E73046FFF76FFFA2E73A
:20454000506E0020FC6D0020555342431C6E0020206E002070B90020446E00201C91002087
:204560005C6E002008B5084B1B78022B07D0033B012B02D80021FFF751FF002008BDFFF724
:2045800069FF002008BD00BF506E002010B501EB8101084A00EBC1010446B1F88C13104617
:2045A000F3F728FE034A204640230121FFF7E2FE002010BDF0C20020E8E700BF70B50A78E9
:2045C00012F060050C46064611D0202D16D1CD88D5B113062AD52A461F496078F3F7ACFE8A
:2045E000E2881D493046FFF753FE00250AE04B780A2B16D00B2B0ED0062B03D13046FAF7C1
:20460000BBFA0225284670BD022260781144F3F793FE284670BD8B78D3B9104BC3F8C059FE
:20462000F0E70F490122FFF733FEEBE70D4964780A4AC1F8C8400321C0E9E45542F8045B49
:204640002B4680F811110021FFF794FE0025D9E7FAF792FAD6E700BF74B9002070B9002032
:2046600030C30020E40400200B7803F00303012B03D0022B04D0002070478B881BB915E6EA
:204680008B88832BFBD099E710B50223044640228121FDF7ABF82046022340220121FDF73C
:2046A000A5F88221204603230822FDF79FF8064B02229A80F3F790FE044A20464023012139
:2046C000FFF758FE002010BDA0010020F0C2002038B509220D46044603238321FDF786F81D
:2046E00029462046FFF7D0FF002038BD82B00023016801930B6901930E4B03E00A6901926F
:20470000013B13D0019A002AF8DA019A094B42F001020192019A0A610A69019203E00A69CA
:204720000192013B02D0019AD207F8D4002002B0704700BF400D0300436D064A1A61C2784B
:20474000012A06D100F2CC5058614FF0802219681A6070471800086010B500230422044625
:20476000194680F811211A46FFF7DAFC2046FFF7E3FF002010BD00BF10B5044629B990F8A1
:204780001131032B0DD0002010BDD0F8E4359B69002BF8D090F81221032AF4D1984700205B
:2047A00010BDD0F89013D0F87C33994214D9C078D4F880230128A1EB030104BFD218C4F8B9
:2047C00080238B4228BF0B46C4F890139BB220460021FFF7CFFDD6E7D0F8E4351B691BB14E
:2047E00090F81221032A03D02046FFF7B5FFCAE79847F9E7F0B5012190F8D17590F8D36529
:2048000090F8CFC590F8CE5590F8D03590F8D22580F8111190F8CC1585B005EB0C2503EB7E
:20482000072302EB062201F01F06AFB292B290F8CD558DF808109BB2012E0446ADF80A7052
:20484000ADF80C30ADF80E20C0F840218DF8095017D0022E1FD036B101F08001FFF72CFC30
:20486000002005B0F0BD092D0FD8DFE815F0BF00AC000E00D5000E00EA0085000E0077007D
:20488000540090F81221032A2FD02046FAF774F9002005B0F0BD01F060012029DAB234D06C
:2048A000012D00F02081032D00F00681002DD7D190F81211022900F0DF800329E5D11B0695
:2048C00000F14B8102EB820200EBC20393F87633002B00F04D81BF4B0122C3F8D429BE49F1
:2048E00020460222FFF7D4FCBAE7DAB2012ACCD8D0F8E43502A99B689847BDF80E30002BE0
:20490000AED12046FFF728FFAAE7D0F8E43502A99B689847A4E7F9B2AE4D012985F8C419E1
:20492000B3D890F81231022B00F02781032BACD1002900F0868190F810110129E1D0D0F845
:20494000E4355B68984795F8C41984F810112046FCF7BAFE2046FFF7FFFE81E7012A94D133
:2049600090F81231022B00F01781032B8DD100F58871FFF78DFC73E73D0A022DADF8062023
:2049800000F05081032D00F00B81012D7FF47DAFD0F8EC3580781B680DF106019847BDF8E0
:2049A0000620002A3FF45CAFBDF80E30002B3FF457AF9A4228BF1A4601462046ADF8062077
:2049C000FFF766FC4CE790F81231023B012B3FF65CAF012F7FF444AFD0F8E43500229B683C
:2049E000C0F8182102A9204698478AE790F81231023B012B3FF649AF764BD0F81821002121
:204A0000C3F8CC1912B10222C3F8CC29734920460222FFF73DFC23E7012F00F09880022F77
:204A20007FF41EAF13F0FF0F7FF41AAF02691B0A023B5268032B00F21D81DFE803F039357C
:204A400031241A437FF421AF90F81231032B3FF41CAF036907F07F0580F81451196867F3CB
:204A60000A120A431A60FFF777FE002D00F0E580022384F81231F3E651063FF4F1AE114629
:204A8000FFF71AFBECE6052363F30612514B012184F816112046C3F8D029FFF75DFEDFE612
:204AA000042363F30612F1E7032363F30612EDE7022363F30612E9E790F81231022BDBD01B
:204AC000032B7FF4E2AE27B9550602D01146FFF7F3FAD4F8E43502A99B6820469847204620
:204AE000FFF73AFEBCE690F812110229C4D003297FF4CBAE002F7FF4B3AE12F07F013FF4AC
:204B000000AF180600F1A78002EB820304EBC30304EB810083F8767383F8741383F8757350
:204B2000282303FB0243416D03F55D73DA780B68023A6FF35553012AD4F8E42598BF43F0DC
:204B400080530B602046936802A99847D9E6D0F8E435C0F818719B6844E702F07F0202EBBD
:204B6000820200EBC20393F81E31002B7FF4B3AE184B0022C3F8D429B1E600293FF4C1AE89
:204B80000121032380F8101180F81231FCF79CFD2046FFF7E1FD63E61149FFF779FB5FE661
:204BA000FDB2052D3FF671AEDFE805F0342C241C0B03D0F8EC3580789B690DF1060198478D
:204BC000EDE6D0F8EC3580785B690DF106019847E5E600BF70B9002044C300203CC3002060
:204BE00038C30020D0F8EC3580781B690DF106019847D4E6D0F8EC358078DB680DF106016E
:204C00009847CCE6D0F8EC3580789B680DF106019847C4E6D0F8EC3580785B680DF10601E8
:204C20009847BCE6D0F8E43580789B6A0DF1060198474570C4F8F005B1E6012384F8123151
:204C40000EE60222D0F8E43580F8101180F812215B68984755E6282202FB014304EB81003F
:204C600083F81E7183F81C1183F81D51816903F58E735BE7012363F3061207E770B5044685
:204C800049B990F81131022B1BD094F81631012B0DD0002070BDD0F8E4355B69002BF8D06F
:204CA00090F81221032AF4D19847002070BD2A4A2369D2F8D0295A60002384F81631002098
:204CC00070BDD0F83831D0F82451AB4217D9C278012AD0F82821A3EB050308BF5219C0F866
:204CE000383108BFC0F828219BB20021FFF718FA00231A4619462046FFF73CFBC5E7D0F824
:204D00003C31B3FBF5F605FB163666B99D420AD8D0F84021934206D233463246FFF700FAAA
:204D2000C4F84061E4E7D4F8E435DB681BB194F81221032A0CD00023052284F81121194638
:204D40001A462046FFF716FB2046FFF7F5FC9CE720469847EFE700BF70B9002082B000233E
:204D60000193019A094B42F010020192C168019A0A610A69019203E00A690192013B02D0AD
:204D8000019AD206F8D4002002B07047400D030082B000230193019A0B4B42F0200201923A
:204DA000019A61F38A120192C168019A0A610A69019203E00A690192013B02D0019A920676
:204DC000F8D4002002B07047400D0300F8B50B7813F060050C4606461CD0202D17D14A7815
:204DE000FE2A44D0FF2A3DD14A88002A56D1CD88002D53D11B0651D43749384B0D7001218F
:204E000083F87C19364A1F23FFF7B4FA00E000252846F8BD4B780A2B4BD00B2B44D0012B6B
:204E2000F6D191F904308988002B47DBFFF796FF21792A4F3046FCF775FC022321794022F6
:204E40003046FCF7D3FC97F87C39022B3BD094F90420002ADCDA012BDAD030460121FFF7A9
:204E6000DDFAD5E70225F9F787FE2846F8BD4D88A5B9CC88012C11D11A060FD5194B1B685F
:204E80009B6998471549C0B281F8D80930B1224601F6D8113046FFF7FBF9B9E7304602253F
:204EA000F9F76AFE2846F8BD0C4B4A8883F8D929AEE70D490122FFF7EBF9A9E701F07F01E8
:204EC000FFF766FFB4E730468121FFF7F5F8002387F87C399CE700BF506E002070B9002021
:204EE000FC6D0020406E002049C3002038B50446FCF74EFC2046022340228121FCF776FCC7
:204F00002046022340220121FCF770FC0C4B0D491B680D4A00250D701B6882F87C592846BA
:204F200098472046FFF71AFF20460121FFF730FF064A20461F230121FFF71CFA284638BDE7
:204F4000406E0020506E002070B90020FC6D0020012905D008B50321FFF71AFF002008BDFF
:204F6000FFF752B90B88F0B433BB028C4C880E898B88C98822F001021204120C0284058B4F
:204F8000028CADB225F0F30592B22B4322F00A0243EA061322439BB242F00102038302840E
:204FA000038B23F00C031B041B0C0383038B9BB21943F0BC01837047042B048C2CD0082B69
:204FC0004E888A880D89C98851D024F480542404240C0484838B078C2C0344EA022440F6BB
:204FE000FF421A4045F6FF733B4043EA063322439BB292B243F4805382830384828B22F4D9
:2050000040621204120C8283838B9BB243EA01239BB2F0BC8383704724F010042404240CD3
:205020004D880F898A88C9880484068B038C12029BB242EA073423F0A00340F6FF42324091
:2050400043EA051322439BB292B243F0100302830384028B22F440621204120C0283038B37
:205060009BB243EA01239BB2F0BC0383704724F480742404240C0484848B038CA4B29BB22F
:2050800024F0F30423F42063224343EA062342EA05129BB243F4807392B282830384838B18
:2050A00023F00C031B041B0C8383838B9BB21943F0BC8183704700BF214A038890429BB290
:2050C00012D002F5806290420ED0B0F1804F0BD0A2F58032904207D002F58062904203D0AA
:2050E00002F58062904203D14A8823F070031343144A904218D002F58062904214D030B4F8
:2051000023F440730C894D6802F56C429BB2234390420C880380C56204850DD18B7A03861E
:20512000012330BC8382704703800B884A68C2620385012383827047034B9842EED0EFE793
:20514000000001400010004000040140104B70B4DA684378017886780E4CD243C2F302223E
:20516000C2F10405E8B283400F2040FA02F23240DBB2134360181B0101F01F050122490946
:20518000DBB2AA4080F8003344F8212070BC704700ED00E000E100E0C27802B1D6E70378DA
:2051A00005485A09203203F01F03012101FA03F340F82230704700BF00E100E000B583B01C
:2051C00009238DF80730FCF7C1FC8DF807009DF80730012BF7D09DF8070003B05DF804FB49
:2051E00082B0064B002201920193019B03EB80000190019B186802B0704700BF502800404C
:2052000082B0064B002201920193019B03EB80000190019B196002B0704700BF5028004032
:205220000023C0E90033C0E90233C0E90433C0E90633C0E90833C0E90A33C0E90C33836337
:20524000704700BF0B6870B4D1E90524CD682B431343D1E9072523431343D1E909422B4350
:20526000D1E90D652343134304680B4A334322402B4313430360D1E90B3442690D6922F05A
:20528000070223431343D1E9014243614560846070BCC260704700BF3F801CF002683649A7
:2052A000002310B422F00102212488420260036043608360C3600361446138D02F4B984210
:2052C0002ED02F4B98423CD02E4B984240D02E4B984232D02D4B984241D02D4B984246D0ED
:2052E0002C4B984217D02C4B98423CD02B4B984216D02B4B984224D02A4B984228D02A4BE3
:2053000098421AD0294B984229D0294B98422ED0284B984208D14FF03D5243F8AC2C03E04C
:205320004FF4746243F8202C5DF8044B7047224B5DF8044B3D229A607047204A43F8642C1C
:20534000F2E74FF474125DF8044B43F8382C70474FF074625DF8044B43F8502C7047184A28
:2053600043F87C2CE0E73D2243F8082CDCE7154A43F8942CD8E700BF10600240286002409E
:2053800040600240586002407060024088600240A0600240B86002401064024028640240D5
:2053A00040640240586402407064024088640240A0640240B8640240006002403D00002022
:2053C000400F002000003D20024A536A23EA00005062704700380240024A136A23EA000032
:2053E0001062704700380240484B98422ED0B0F1804F32D0464B984236D0464B98421ED063
:20540000454B984237D0454B98423BD0444B98423FD0444B98424BD0434B984240D0434BA4
:2054200098424CD0424B984251D0424B984256D0414B98425AD0414B98425ED07047404AFC
:20544000136A43F0040313620420C5E73C4A536A43F0010353620120B6E7394A136A43F030
:20546000010313620120B7E7354A136A43F0020313620220B0E7324A136A43F008031362E6
:205480000820A9E72E4A136A43F0100313621020A2E72B4A136A43F02003136220209BE76C
:2054A000274A536A43F4803353624FF480308BE7234A536A43F002035362022084E7204AAC
:2054C000536A43F4003353624FF400307CE71C4A536A43F4802353624FF4802074E7184AC8
:2054E000136A43F040031362402075E7144A136A43F08003136280206EE7114A136A43F47E
:20550000807313624FF4807066E700BF000001400004004000080040000C0040001000407B
:20552000001400400004014000400140004401400048014000180040001C0040002000402F
:2055400000380240224A936803F00C03042B10B421D0082B22D01F4B03601D4C1E4AA168B8
:20556000C1F30311114491F87011CB404360A168C1F38221114491F8701123FA01F18160A7
:20558000A1685DF8044BC1F342310A4492F87021D340C3607047114B0360DEE754685168E8
:2055A00052686302C2F388124CBF0C4B094B01F03F01B3FBF1F303FB02F3054A5268C2F353
:2055C000014201325200B3FBF2F30360C5E700BF003802400024F400E404002000127A007C
:2055E0002DE9F04700230F6801264FF0030C02E00133102B41D006FA03F232EA0704F7D109
:20560000D0F800E05C000CFA04F52EEA050EC0F800E091F80490D0F800A009FA04FE09F140
:20562000FF394EEA0A0EB9F1010FA846C0F800E06FEA050515D8D0F808E005EA0E058560BB
:205640004D79D0F808E0A54045EA0E058560456825EA020242608A7945689A4092B22A432B
:205660004260C26822EA0802C260CA79C568A24001332A43102BC260BDD1BDE8F0870B4BD6
:2056800093F8B825D20703D5012283F8DA29704793F8DA294AB9D3F81C3633B1044B1A7826
:2056A00010445A78187011445970704770B90020B86D002010B50E4C40F0080284F884215F
:2056C00094F9CE20022A06DD420704D583071CBF012384F8D63005210648FCF747FB062143
:2056E00084F88501BDE810400248FCF727BB00BFE40400206406002010B5FCF7CFFAA8B367
:205700001B4C94F9CE30012B30DD59B3022B2DD094F8D6309BB971B180230521154884F87E
:205720008A31FCF723FB062184F88B01BDE810401048FCF703BBBDE810400420BAE700298D
:2057400014BF0020042094F8D1301A0748BF40F002005B0701D411B108B940F00100BDE8BB
:205760001040A7E7022BD3D10420ECE710BD00BFE40400206A060020F8B5224C04F5C6770E
:20578000030A84F8910105460621384684F89031FCF7ECFA94F8D13084F89201DB072AD46C
:2057A000B4F8D220AA4226D1174DD4F88C31C5F8DB39C3B285F8E13941F26F714FF6FF73D4
:2057C0008A4218BF0123134405F6DB16C3F307220621304685F8DF2985F8E039FCF7C6FA75
:2057E000072185F8E1093046FCF7A8FA052104F29310FCF7A3FABDE8F84004480721FCF77C
:205800009DBA00BFE404002070B900207006002008B5FCF743FA48B1A1F59C53083BB3F535
:205820007A7F03D2BDE808400846A5E708BD2DE9F0476B4E3368002B3AD06A4D6A4C05F1D5
:20584000CE07306838F04AFE002833D1674B198809291D4609D95F8864227A43B2FBF1F2BB
:20586000452A40F3A1811880588094F8193A012B00F0C581022B00F0E08133B95C4805217F
:20588000FCF75CFA012384F8193A5A4B1D685A4B1B78002B00F0DB81584B1B68EB1A782B25
:2058A00040F2D581D4F83406F9F730F9C4F81C5ABDE8F087306838F009FE94F8E2398046BF
:2058C000052BBED8DFE803F00309171D3745AA28B7D1012384F8E239B3E7552803D1022367
:2058E00084F8E239ADE7414A938801339380002384F8E239A5E7032384F8E30984F8E23925
:205900009FE7132884F8E409C4F8FC0907DD374AD3880133D380002384F8E23991E718B952
:20592000052384F8E2398CE70023C4F8003A042384F8E23985E7D4F8003AE218013382F844
:20594000E509D4F8FC29C4F8003A93427FF479AFE6E7D4F8FC392A4803F1020A4FFA8AF1FE
:20596000FCF704FA804594F8E39940F01481262022F0B4FD204B48B100221A701B4A53884B
:2059800001335380002384F8E2395AE71A784A4519D100221A7009F1FF33102B00F2F6807F
:2059A000DFE813F030008E008E00DE008E00F400F400F4003000F400F400F400F400F40095
:2059C000F400F4003000B9F1090F02D0B9F1110F01D1012ADDD0054A538901335381DAE7B3
:2059E000B46D0020E404002070B90020E26D002077060020C42F0020F06D0020F46D0020F8
:205A000053C30020BAF1060F5ADDB9F1010F06D0B9F1090F0CBF4FF002094FF0030994F81B
:205A2000E80994F8E91994F8E72994F9E5E994F9E7C994F8E63985F8CE9041EA002109B226
:205A4000900785F8CFE085F8D1C0A5F8D21006D512F00C0F14BF0122002285F8D620B9F1C9
:205A6000030F13D1BAF1090F2ADD94F9EB29082AA8BF082222EAE27285F80421002043B2EB
:205A80009A4200F1010059DC94F8EA39D4F828A0002002469BB25245904657DB7C4B85F828
:205AA000D0001B78232B0BD109EB8903794A03EB83030CEB83031380A2F802E09180D080B5
:205AC000754976480A225EF046FD10B1002384F80E3A714B3A681A607A685A603A891A8113
:205AE00094F80E3A2BBB95F8D6306D4A002B14BF0223012384F80E3A95F8D130117884F804
:205B0000101A13F001031CBFB1FA81F35B09517884F8111AD8B29188927884F80F0AA4F8A8
:205B2000121A84F8142A13B109B1A4F8161A84F8180A0EF079FF0EF077FF1FE704EB43086D
:205B4000234493F8ED39A8F8223698E704EB48080132B8F82C8052B2984508BF10469AE769
:205B6000BAF1040FACDD94F8E52994F8E63943EA022359041AB204D5C3F30D03A5F8D430DE
:205B80009EE7002AF8DBA5F8D23099E7454A938901339381F2E619F0010F7FF4F3AE414AE1
:205BA000138901331381EDE63F4BD3F89821B3F89C11012A1AD141F25632914203D14FF091
:205BC000FF32C3F89821D3F89821306802EB820202EB820201EB420189B2A3F89C11036805
:205BE0001B69984700232B806B803EE60132EAD1B1F5965F04BF0122C3F89821E3E72A4D41
:205C000095F9CE60002E3FF440AE022E11D14FF48040FFF7B1FD84F8196A95F9CE30012B09
:205C20007FF733AE95F8D130C3F3400385F8D6302BE6032384F8193AEFE71B4BB3F8D43012
:205C4000002B3FF422AE032384F8193A1DE694F8402094F841309A4204D0FCF7C5FEC4F813
:205C60001C5A25E6D4F81C3AEB1AB3F57A7FBFF41FAE0E4B1B68ED1A952D7FF619AE0C4826
:205C80000521FCF75BF8BDE8F047FCF7ADBE00BFE4590020E859002074C30020B2050020B3
:205CA000B86D0020E26D0020E4040020F46D002077060020104BD3F81C0610B5D8B10F4C19
:205CC000217841B162780DF071FDA38883421ABFA08001210021E2885AB141F28833934290
:205CE000B8BF13469A4204D0E380BDE810404BF00BB90029F9D110BD70B90020B86D00207F
:205D000010B401440446002014F8013B08225840430010F0800F08BF400083F0070314BFDD
:205D2000D8B2C0B2013AF3D18C42EDD15DF8044B704700BF30B54FF4806085B030F048FB22
:205D400048B3164C90F9040094F8203A144A002B18BF08234FF4E1310125CDE901530091D2
:205D600000234FF4806130F090FBFF23C4F88000003818BF012084F8FC3484F80C3584F8BE
:205D80001C3584F82C3584F83C3584F84C3584F85C3584F86C3505B030BD00BF70B9002017
:205DA0006D200108374B1B6813F000635CD02DE9F04F354B1F78B84251D3FF2856D1334B60
:205DC00093F8DE30002B47D0DFF8D4A00022CAF8242ACAF8282ACAF82C2AAAF8302A002F14
:205DE0004CD00AF2FC431046144611461546164603EB071BB946B3F802C09F8993F80080DF
:205E000093F901E061443A444645D3E901C738BF464610337545B8BF75469B4509B212B2D2
:205E200064443844E7D191FBF9F192FBF9F28AF8246A8AF8255ACAF8284ACAF82C0A144BFC
:205E4000AAF8261A1B781149AAF8302A092B4FF0000281F8DE200CD00E48BDE8F08F0E4ADD
:205E600002EB0010BDE8F08F184670470020BDE8F08F0A4B9AF8242ADA80EDE73A46394646
:205E8000DDE700BF146C002080060010E4040020E459002094C300206CBE0020E8590020C2
:205EA00070B900200268F8B53A4E3B4CB6F9343A511C01607E2111700168054603EBC30300
:205EC00084FB0302481CDC17002328600B70FF20C4EB6204FFF766FF2034304BA4B20028E5
:205EE0004DD01B78B0F90C1023BB2D4BA1F57A729A4246D82B48B0FBF1F189B228464AF078
:205F0000C7F996F897357BB12AF06CFD014628464AF0BEF9214628464AF0BAF928460821B9
:205F2000F7F7DEFF0120F8BDB6F84C1628464AF0AFF9EFE71C4B1F78002FD6D01B48002331
:205F400000EB830201339289BB421144F8DB184B9FED186A93F8223007EE103A07EE901A31
:205F6000B8EEC77AF8EE676AC6EE077A67EEA67AFCEEE77A17EE901AB1FBF7F1B5E71B781C
:205F800013B94EF69C21B9E7074B1F78002FF8D00146D3E770B90020676666662813001086
:205FA0001783930300879303800600105C2F00106C300020000048432DE9F8434A4C42787B
:205FC00094F8363A02F00F05C3B9EDB92B46002184F8381AEB1AD9B20E290BD8234493F8A1
:205FE000981539B102F0F002802A4AD0902A5FD0A02A0DD000273846BDE8F8830021AB42FF
:020000040801F1
:2060000084F8381AF6D8E5E784F8365A2B46DEE7412966D081F08003042B62D90846FCF797
:206020003FF8031D0246DBB2304884F8383A65F05F0584F8395AFCF7EBFE94F8387A002FBD
:20604000D8D0BE1E16F0FF0024D1FF25A946022756B1DFF89C80464418F8011BD4F85C0AA4
:2060600038F040FA4645F7D1D4F85C0A494638F039FAD4F85C0A294638F034FA3846BDE835
:20608000F88365F07F050427022684F8395A84F8387A3046164A4FF6FF71104412F8015BD7
:2060A000491B904289B2F9D15FFA81F90D0ACFE7412914D081F08003042B10D90846FBF76B
:2060C000EFFF65F06F050627042684F83B0A84F8395A84F83A1A84F8387A3046DAE7042089
:2060E000EFE7082304229FE770B90020AAC30020A8C300200B4B93F86E2612B1B3F8A825E2
:206100004AB9B3F99436084AD81782FB0323C0EBA30000B27047D3F8880690FBF2F000B2F3
:20612000704700BF70B9002067666666F8B5184CC6B205463146D4F8600A38F0D3F994F806
:20614000641AD4F8600AC5F307274E40394684F8646A38F0C7F994F8641AD4F8600AC5F36E
:2061600007464F40314684F8647A38F0BBF994F8641AD4F8600A2D0E4E40294684F8646AD4
:2061800038F0B0F994F8641A4D4084F8645AF8BD70B9002070B50C4DC6B231460446D5F8DB
:2061A000600A38F09FF995F8641AD5F8600A240A4E40214685F8646A38F094F995F8641A45
:2061C0004C4085F8644A70BD70B9002038B50B4C002305462421D4F8600A84F8643A38F023
:2061E00081F9D4F8600A542138F07CF9D4F8600A2946BDE8384038F075B900BF70B90020BD
:206200002DE9F043DFF894932DED028B99F8654A83B00E461546002C00F03982013C89F8D9
:20622000654A9FEDD88AD84FDFF874833378002B62D099F8654A002C5ED135B137F052FAD0
:206240002B68C01A002880F2028499F8664A002C40F0A68399F8670A062840F2D781CB4A1C
:2062600092F8A53192F8A411994200F00082D2F8A01199F868CA31F813406444013001336B
:2062800002F5D072A4B2C0B2DBB2B4F5E06F89F8670A537100F0D18100F2AA80B4F5806FCC
:2062A00000F0F88264D9B4F5A06F00F0CC823CD9B4F5A16F25D8601EC0B2FFF773FDC8B1A7
:2062C000B0F90C30B24AADF8014092F82210D9F8842503EB830303EB830349089B0093FB5F
:2062E000F1F31021CDF803308DF800106846904700233370002D99D103B0BDEC028BBDE88C
:20630000F083B4F5C06FF5D1B9F87036002B00F054832AF07FFB10220024CDF80300062348
:206320008DF800208DF801401FE2B4F5826F00F05082B4F5846F40F0358199F848369A0763
:20634000D8D5B9F84A36CDF803301021202204238DF800108DF801208DF80230D9F8843551
:206360006846002498473470002D7FF45FAFC3E7B4F5067FBED8B4F5007FC0F02C81A4F58E
:206380000073182BB6D801A252F823F009670108F7660108F7660108F7660108F7660108A8
:2063A000F7660108F7660108F7660108F7660108F5620108F5620108F5620108F5620108C5
:2063C000F5620108F5620108F5620108D3660108BD660108BD660108BD660108BD660108AB
:2063E000BD660108BD660108BD660108BD660108B4F5116F00F0E0815BD8B4F5026F00F036
:20640000BF8121D9B4F5036F00F07282B4F5046F7FF470AFB9F99436D9F8842503EB83032B
:206420005B001020CDF80330402108238DF800008DF801108DF8023068460024904734702E
:20644000002D7FF4F3AE57E7B4F5E46F00F07881B4F5006F76D199F8482691077FF54AAF75
:2064600013F0010F4B4B00F005835A6882EAE273A3EBE27303EB5303A7FB0313DB08002A8C
:20648000ACBF43F0004343F04043102100240822CDF803308DF800108DF80140D9F8843509
:2064A0008DF80220684698473470002D7FF4BEAE22E745F230239C4200F0B1811DD945F238
:2064C00040239C4200F0298245F250239C427FF411AFD9F88836CDF8033010215022522386
:2064E0008DF802308DF80010D9F884358DF80120684600249847347036E7B4F5376F00F06F
:2065000031826FF437616318072B3FF6F3AEA4F17100C0B2FFF746FC00283FF4EBAE90F91D
:206520000130CDF8033010238DF80030ADF80140D9F884356846984700233370002D7FF4E7
:2065400075AED9E6B4F5E26F7FF4D4AE124B93ED140AD3ED017A20EE270A002420EE080AB1
:206560005CF01CFD10230722CDF803008DF800308DF801308DF80220D9F884356846984769
:20658000347092E70000C8421F85EB51E40400206C300020A46C0020002F001070B9002078
:2065A000C5B3A29140F201439C427FF4A3AEB9F9343ACDF803301021012204238DF80230CE
:2065C0008DF80010D9F884358DF801206846002498473470C8E6B4F5807F00F01481B4F51D
:2065E000887F7FF487AEB9F99636CDF80330012210238DF800308DF801308DF80220D9F83D
:2066000084356846002498473470ADE60130CD4AC0B292F8AD1192F8AC318B4222D04B1C4A
:20662000DBB24900D2F8A841C74A645A89F8670AB4F5E06F53717FF42FAEC44B93ED130A58
:20664000D3ED017A20EE270A002420EE080A5CF0A5FC10220723CDF803008DF800208DF841
:20666000014082E0002182F8AD110123DAE7B84999F8683A097882F8A5410133DBB2013131
:206680008B4289F8683A00F087810120C1E700283FF4C7AD0378303B012B3FF6C2AD013093
:2066A00009F665220621FCF7F3FE99F8653A89F8660A002B3FF4B5AD3470B2E5A4F1110087
:2066C000C0B2FFF76FFB00283FF414AEB0F9023027E799F89735002B40F0B081B9F84C06F6
:2066E000CDF80300102302228DF800308DF801308DF8022083E7601EC0B2FFF753FB0028A3
:206700003FF4F8AD43680CE7D9F880369149D9F8842581FB0301DB17C3EBA103002410210F
:20672000CDF8033002238DF800108DF801408DF80230684690473470002D7FF477ADDBE57D
:20674000824B93ED150AD3ED017A20EE270A002420EE080A5CF022FC102320228DF800307B
:20676000CDF8030007238DF801208DF802306846D9F8843598473470002D7FF457ADBBE5CB
:2067800099F848369B077FF5B5AD734AD9F884359268CDF80320102220218DF80020082207
:2067A0008DF801108DF802206846002498473470002D7FF43BAD9FE52AF014F910230922B6
:2067C000CDF803008DF800308DF801308DF8022015E7D9F8803513F0200440F0F1805F4BEB
:2067E0001B681B0640F13981102304228DF803408DF804408DF805408DF806408DF80030D6
:206800008DF801304AE6D9F86C3ACDF803301022002401238DF800208DF80140A5E7B9F900
:206820009236CDF803301021302252238DF802308DF80010D9F884358DF801206846002452
:206840009847347090E5FF20FFF7ACFA00283FF451ADB0F90C304249D9F8842591F8221087
:2068600003EB830303EB83031020490800249B0093FBF1F305218DF80000CDF803308DF856
:2068800001408DF80210684690473470002D7FF4CDAC31E599F8703A0133DAB2042A00F0AF
:2068A000D08042F2107389F8702A03FB02F3D9F8742A002A00F0C080023399F8B825D2077E
:2068C000B9F88C2648BF0433D40748BF0A33900748BF1433D10548BF2833540748BF6433E2
:2068E000500648BF03F57A63102100240422CFE599F8483698077FF5FDAC174BD9F8842590
:20690000D9894FF4F36303FB01F3A7FB03135B091020CDF80330302187E5B9F99036CDF84C
:2069200003301021402252238DF802308DF80010D9F884358DF8012068460024984734704B
:2069400012E500BFE40400208C060020002F00108006001067666666A46C0020146C002089
:206960006C300020FF20FFF71DFA00283FF4C2AC90F90130CDF80330102170220B238DF83E
:2069800002308DF80010D9F884358DF801206846002498473470E7E489F8684A012038E66E
:2069A0005C490620FCF7C4FC002389F8660A337003B0BDEC028BBDE8F083D9F88806AAE4B4
:2069C000554A99F84816538A643BC3EB4370C3EBC00388FB03401844DB17C3EB202309339A
:2069E000092BA8BF092323EAE37303EB830311F0020F03EB830314BF4FF47A7000209B00B8
:206A0000C90748BF00F5FA60117DD9F884259BB203440B44042010218DF80200CDF8033091
:206A20008DF800108DF801106846002490473470002D7FF4FBAB5FE401333EE729F0D2FF12
:206A40004EE6012389F8703A42F210732FE7347003B0BDEC028BBDE8F08399F89635002BBA
:206A60003FF448AC99F8783A032B4ED8DFE803F043392A111A6882EAE273A3EBE27303EBD3
:206A80005303A7FB0313DB08002AB8BF43F08043FBE4D9F8802A537A907AD17A03F140734B
:206AA00003EB0023002203EB014389F8782A10220421CDF803308DF800208DF801208DF82F
:206AC00002104BE4D9F87C1A8A7D087C897A120402EB00220A44591C89F8781A02EB036332
:206AE000E5E7D9F87C1A4A7DC87B497A120402EB00220A44EFE7D9F87C1A0A7D887B097AD9
:206B0000120402EB00220A44E5E75A1C89F8782A1B06CCE759210108A46C002030B5A0F1A0
:206B20007D03012B044683B00D46104608D9214637F0D8FC15B1288804442C8003B030BD36
:206B40007D21019237F0CEFC019884F0200137F0C9FCEFE730B50F4B85B0D3F8B4250023E8
:206B60000446C51DADF80E3014F8010B01920DF10E01FFF7D3FFA542019AF5D10DF10E0032
:206B800018F058F8019A9DF80E000021FFF7C6FF05B030BD70B900207E28F8B50F4652D0CE
:206BA000324E96F8B04164B9314D95F88C1A51B11B2885F88C4A3DD00D2837D0012386F885
:206BC000B0310020F8BD7D284AD095F8902A1AB180F0200085F8901A95F88B2A062A14D819
:206BE000B5F88E4A511C2A440444C9B2A5F88E4A85F88B1A82F8840A002BE2D10729E0D114
:206C000001231C4886F8B031F8BDB5F88E3A1844C0F3072353FA80F0FF284FF00103A5F866
:206C20008E0A86F8B031CCD11248F8BDA5F88E4A2046F8BD90470028C0D0012320463B705D
:206C400086F8B031F8BD0A4B084A0024012183F88B4A83F88C1A3C7082F8B0412046F8BD90
:206C60000123084685F8903AF8BD00BFE404002070B90020F4C30020044AD2F8943A43F4A2
:206C8000DF2343F48063C2F8943A704770B90020013070B5094EC4B203E04AF035FD0134A9
:206CA00048B9E5B2152D21463046F6D9162D04BF034B93F8985A284670BD00BF04C400203B
:206CC00070B9002000B1D7E7044AD2F8943A23F4DF2323F48063C2F8943A704770B900207B
:206CE00070B5114C84B00546D4F89C0A0E462FF02DFB94F8902594F89135003A18BF0122BF
:206D00000BB142F00802CDE9016200234FF4964195F9000000911A4608212FF0B6FBC4F8F1
:206D20009C0A04B070BD00BF70B9002010B5064C03E0D4F89C0A37F0C9FBD4F89C0A37F0D4
:206D4000CDFB0028F5D110BD70B9002010B50D4CD4F8A03A1B791E3B012B0DD9D4F89C0A32
:206D600001213830FFF7BCFF0023C4F8A43A84F8A83ABDE81040D9E7D4F89C0A012137F04D
:206D80009DFBF1E770B900200B2814D810B401EB4103094C01EB83032344184490F8A83637
:206DA000934205D02144002380F8A82681F89C365DF8044B7047704770B90020F0B5444C80
:206DC00094F8A93A012B83B005464FD994F8AA1A4048DFF810C194F8AB7A4A1CA0FB0260DE
:206DE00000F4FE7606EB90001944121A5CF8216084F8AA2A2FB1D4F8AC1A04F52B62914231
:206E00000DD06EB9344A0133A2FB031222F0010101EB52029B1A84F8A93A03B0F0BD2F4EC5
:206E200094F8C43A93B92E4B019348F2A501123B15226F46A4F8C81A009384F8CA2A294666
:206E40003846B04758B994F8A93ADBE76F46384616F0B0FC29463846B0470028F3D094F83B
:206E6000C41A49B1384616F01FFCECE71D4A52F82360002EC6D0D3E7009E1B4A964214D94E
:206E8000013A013E41F2210512F8013F81EA0321082311F4004F85EA41000ABF490081B2D2
:206EA00089B2013BF5D19642EED1384649F016FA0E49009D6D1A152DA8BF15252A4601F177
:206EC00018005DF00FFB94F8A93A84F8F55A99E770B90020CDCCCCCCABAAAAAA9D3201088E
:206EE0004DC40020144807083BC4002038C4002070B50C4E054606F6FA21D52249F08AFE22
:206F00002C686C6006F6F821641A182CA8BF18242960224606F531605DF0E4FA86F8284BFE
:206F200070BD00BF70B90020F0B58BB004461F4B1F4A2049009302A81F4B4AF023FB266829
:206F40000025731C2360357023682922591C21601A702368EA22591C21601A702368C82273
:206F6000591C216002A81A705AF0DCF8471C02A93A4620685DF0B6FA236829461F440C232A
:206F800000E027687A1C013B22603970F9D12268511C2160137023680122991821601A7056
:206FA00023689B1B33700BB0F0BD00BFA3C400203CE007083CE1070834E1070870B5056832
:206FC0002C4E00236A1C02602B7003682122591C01601A7096F8B835DB0704461ED5B6F83B
:206FE0008C36590510D52449204649F0F9F896F8B835DB071DD523680022591C21601A7013
:2070000023685B1B2B7070BD1A0524D4D80524D4D90724D49A0724D51849E5E7D6F8743AA0
:207020006BB11749204649F0DBF896F8B835DB07E1D423682A22591C21601A70DBE7114BDB
:207040001B681806CBD596F8483603F00303032BC5D00D49C8E70D49C6E70D49C4E70D49C8
:20706000C2E796F83C2B0C490C4B002A18BF1946BAE700BF70B9002064E1070848E1070831
:2070800054E10708146C00205CE107086CE1070870E1070878E107084CE1070880E10708F0
:2070A00038B50368394D591C082201601A7003681E22591C01601A70B5F99236B3F5E16FEF
:2070C000044650DDA3F561631BB2B3F5E16FF9DC07EE903A9FED2E7AF8EEE77A204667EE4E
:2070E000877AFDEEE77A17EE903A99B249F0D0F8B5F99036B3F5E16F3CDDA3F561631BB27A
:20710000B3F5E16FF9DC07EE903A9FED217AF8EEE77A204667EE877AFDEEE77A17EE903A9E
:2071200099B249F0B5F8B5F99436B3F5E16F28DDA3F561631BB2B3F5E16FF9DC07EE903AF4
:207140009FED137AF8EEE77A204667EE877AFDEEE77A17EE903A99B2BDE8384049F098B807
:2071600003F561631BB213F5E16FF9DBB0E703F561631BB213F5E16FF9DBC4E703F56163A7
:207180001BB213F5E16FF9DBD8E700BF70B9002058A08B41026810B40421541C04601170C3
:2071A00002680B24511C016014705DF8044BC82149F06EB838B50368214D591C0A22016030
:2071C0001A7003680822591C01601A7095F8973504466BB329F006FC1A490530A1FB0031EF
:2071E000C1F3CF01204649F053F8D5F88036164AD91782FB0323C1EBA30189B2204649F081
:2072000047F829F007FCD5F8885623682A0C591C21601A7023682A0A591C21601A7023685D
:207220005A1C22601D7023685A1C2260187038BD29F0E4FB0146204649F02AF8D5E700BF4E
:2072400070B90020CDCCCCCC6766666603681122591C70B501601A7003681D4D1D4E5A1C42
:20726000026002221A700446296848F0F9FF6968204648F0F5FFE98901EBC1018900323184
:20728000A6FB0131C1F34F11204649F001F8298A01EB8101490089B2204648F0F9FF0E4ADC
:2072A0000E4BD2F86C1A9942A8BF194621EAE171A6FB0131490901F57A7189B2204648F048
:2072C000E7FF23682A7D591C21601A7070BD00BFA46C00201F85EB5170B9002020A1070009
:2072E000F8B50B4D0B4F06462946D52249F092FC34687460A91E641A402CA8BF4024316039
:20730000224607F534605DF0EDF887F8804BF8BDE25A002070B9002070B5104E104B0A4671
:20732000151D014696F8810B03F83F5C82B003F83D0C7B25C82003F83C0CA3F13B0403F815
:20734000400C03F83E5C68460193009448F05AFF6846FFF7C5FF02B070BD00BF70B9002096
:20736000205B0020F0B5434C94F8843BD90785B0054637D594F8853B0F2B56D900210F465C
:207380003D4B94F8842B3D4843F8400CA3F1400640F6C82CC2F38202712003F8381CA6F863
:2073A00004C0B11C0393B071373B02A8F271BA22029349F02FFC029A731CD21A727016F032
:2073C0001BFA02A8FFF78CFF16F016FA94F8843BC4F8885B23F0030343EA470384F8843BA2
:2073E00005B0F0BD9A0728D5D4F8880B2D1AB5F57A6FF5DB94F8853BD4F88C0B0F2B97BF45
:207400001F4A204902EB8303D969036801911B69984701990620FDF7F3FE94F8843B6FF333
:20742000410384F8843B05B0F0BD174B93F834301F1E18BF01273946A2E7144B1B685B0594
:20744000CED4114B93F83430002BC9D00A4B0393C821A3F13F0202A803F8401C0292FFF747
:2074600099FE16F0C9F902A8FFF73AFF16F0C4F9B6E700BF70B90020205B0020C80032ECEB
:2074800014480708A0680600C4650020146C00202DE9F843254E96F8904B804634BBD6F8DA
:2074A000F43B6BB306F694374FF001090DE001352C44EFF31183502282F31288D6F8F42BF8
:2074C000944220DADBB283F311883319601C93F8945B384429460022FBF7DAFF0028E6D048
:2074E00096F8803BD3B186F8909BE0E796F8803B33B901463A20FBF71BFF044686F8900B0A
:207500002046BDE8F8830022DBB2C6F8F42B96F8904B83F311882046BDE8F88341463A207A
:20752000FBF706FF86F8900BC1E700BF70B90020044BD3F8AC3530EA030314BF012000205C
:20754000704700BF70B90020AB4A38B50820002382F8AD31FFF7ECFF002800F08C80D2F818
:20756000A8314FF4806102204FF48264198082F8AD0101465C804FF40020FFF7D9FF50B1AD
:207580004B1CD2F8A801DBB240F2014482F8AD3120F811401946994C94F86D36002B6CD171
:2075A00094F86E36002B40F088804FF40070FFF7BFFF50B14B1CD2F8A801DBB24FF40465BD
:2075C00082F8AD3120F811501946D4F88045A50700F11881600700F1EB80894B1B681B0679
:2075E00000F1A38000234FF4803082F8AC1182F8AD3182F8A531FFF79BFFD0B3D2F8A031D4
:2076000001214FF4047082F8A51118804FF40040FFF78EFF50B14B1CD2F8A001DBB24FF420
:20762000007482F8A53120F8114019464FF40030FFF77EFF50B14B1CD2F8A001DBB24FF435
:20764000A06482F8A53120F8114019464FF48020FFF76EFF38B1D2F8A0014FF437644B1C2F
:2076600020F81140D9B2002382F8A41182F8A53138BD0146CAE701467DE70120FFF758FF6E
:2076800000288DD04FF48030FFF752FFD2F8A85128B94FF4047325F811300131C9B20BB205
:2076A000481CC1B24FF4116082F8AD1125F8130094F86E36002B3FF478AF0220FFF738FFD3
:2076C00000283FF472AF4FF40040FFF731FF50B94B1CD2F8A801DBB24FF4007582F8AD3105
:2076E00020F8115019460420FFF722FF50B14B1CD2F8A801DBB24FF4C06582F8AD3120F837
:20770000115019464FF48010FFF712FF00283FF44CAF4B1CD2F8A801DBB245F2502582F8EC
:20772000AD3120F8115019463FE74FF40050FFF7FFFE50B14B1CD2F8A801DBB24FF40364D5
:2077400082F8AD3120F8114019464FF48050FFF7EFFE68B1D2F8A8014B1C4FF40064DBB2EC
:207760008D1C20F81140E9B282F8AD1120F813404FF48040FFF7DCFE50B14B1CD2F8A8010B
:20778000DBB24FF4846482F8AD3120F8114019464FF48060FFF7CCFE00283FF423AFD2F837
:2077A000A8014FF402644B1C20F81140D9B219E74FF48060FFF7BCFE50B14B1CD2F8A8016E
:2077C000DBB24FF4807482F8AD3120F8114019464FF40060FFF7ACFE00283FF4FEAE4B1C14
:2077E000D2F8A801DBB24FF4887482F8AD3120F811401946F1E600BFE404002070B9002043
:20780000146C00208020FFF793FE50B14B1CD2F8A801DBB245F2302582F8AD3120F81150DC
:2078200019464FF48070FFF783FE50B14B1CD2F8A801DBB245F2402582F8AD3120F811506A
:2078400019461020FFF774FE50B14B1CD2F8A801DBB24FF4E06582F8AD3120F81150194611
:207860002020FFF765FE50B14B1CD2F8A801DBB24FF4E26582F8AD3120F8115019464020ED
:20788000FFF756FE00283FF4A5AE4B1CD2F8A801DBB24FF4E46582F8AD3120F811501946CD
:2078A00098E600BFF0B5C94C94F8FC3BD4F88015C4F8F80B0133880785B084F8FC3B12D45D
:2078C00011F0340F34D1090794F8FC2B41D412F007055AD0282A00F0DA80D4F888355E20AC
:2078E000984705B0F0BD7020FFF722FE0028E7D0B74E2425A6F14C07F6EC017A97ED017A2E
:2079000067EE877A2846FDEEE77A013517EE901AC1EB411301EB8301C90009B2EDB2FAF7EE
:2079200057FC272DE8D1D4F8801511F0340FCAD04FF40060FFF7FCFD002840F0278194F88A
:20794000FC2B12F0030100F0FD80D4F880150907BDD54FF40070FFF7EBFD0028B7D012F048
:207960000305B4D19B4AB4F99436D91782FB0323C1EBA30109B21420FAF72AFC29461C208A
:20798000FAF726FC94F8FC2BA1E7FF20FEF70AFA002800F001810378FF2B00F09A8090F9AF
:2079A00001100220FAF714FCFF20FEF7FBF9002800F091800378FF2B00F08D80B0F90C20EB
:2079C000854B844893F8221002EB820202EB82029300490893FBF1F3D91780FB0320C1EBDC
:2079E000A00001B20320FAF7F3FB94F86D36002B79D1D4F880359A0640F198804FF4005091
:207A0000FFF796FD002840F0CB80744D4FF48060FFF78EFD002840F04D816B8A94F8FC2B07
:207A2000297DB3F5967F02D9100740F1128194F89335002B40F0B280A1F1200307EE903AD8
:207A40009FED677AF8EEE77AF6EE006A67EE877ABEEE007AF5EEC07AF1EE10FA58BFB0EEED
:207A6000667A77EE877AFDEEE77A17EE903A19B20520FAF7ADFB4FF48050FFF759FD002895
:207A800040F0BE8094F8FC2B282A7FF426AF554A554B15685549A3FB0535AD09A1FB05366C
:207AA0007609A1FB06314909C1EB0111A6EB81010902C6EB0616002309B21720A5EB860648
:207AC00084F8FC3BFAF784FB31B21820FAF780FB03E7294665E700210320FAF779FB94F822
:207AE0006D36002B85D00120FFF722FD002840F0F38094F86E36002B3FF47BAF0220FFF792
:207B000017FD002840F041810420FFF711FD00283FF46FAFB4F87036002B00F0438128F04D
:207B200079FF01B20420FAF753FB62E71B07A9D52F4B93E8030002AB83E803001846FAF76C
:207B40005DFB9FE74FF48060FFF7F2FC00283FF4FCAE284BD4F8F82BD4F86C5A9A4240F239
:207B6000F180254BE91783FB0523C1EB6313642101FB13510DB219B21020FAF729FB294639
:207B80002120FAF725FB94F8FC2BDEE6B4F996163020FAF71DFBD2E6014602E709B267E779
:207BA00094F848369F075AD44FF48060FFF7C0FC0A4D00283FF431AF002631460120FAF7D1
:207BC00007FB31460920FAF703FB26E770B900204C2F0010676666666C300020A46C0020AE
:207BE000E4380E3FC42F0020D34D621089888888704807083F4B4C001F85EB510050C3477F
:207C000094F8482600239207CDE9003347D494F8003C012B43D0B4F98C355FED086A07EE82
:207C2000103AB4F98E3507EE903AB8EEC77AF8EEE77A27EE267A67EEA67ABDEEC77AFDEE9C
:207C4000E77A02A88DED027ACDED037AFAF7D6FA18E742F20F719942A8BF1946E7E6544D69
:207C6000544BE9894FF4F36606FB01F14909A3FB0131C9091120FAF7ABFAE9894E4B06FB9D
:207C800001F1A3FB01214909A3FB01235B09642202FB131109B21920FAF79AFAB6E6D5E940
:207CA000002301216846CDE9002384F8001CFAF7A5FAE7E694F848369E077FF57DAFAB68A1
:207CC0003D4AD91782FB0302C1EB6211642606FB113636B209B271E794F8FD1B00293DD1E4
:207CE0000B460620A4F8FE3BFAF772FAB4F8FE3B0133A4F8FE3B28F081FE94F8943594F875
:207D0000FD2B012B94F897351ED000EB800086B213B10AB1B6FBF2F6274BA3FB062343F39F
:207D20004F113A205D09FAF753FA642101FB1561224B89B20531A3FB0131C9083B20FAF723
:207D400047FAD6E60D4617E71BB112B1B0FBF2F080B201B23920FAF73BFACAE6B4F8FE0BF0
:207D6000B4F84C26B0FBF1F301FB1303642000FB02129BB24900B2FBF1F2110241EA031139
:207D8000C2F30322114309B2ABE7D4F880360C49DA1781FB0313C2EBA30319B22820FAF7B7
:207DA00017FAB1E6D4F8883683F3100319B2B9E6A46C0020C55A7C0A1F85EB51CDCCCCCCB8
:207DC0006766666603685A0607D513F4057F04D007298CBF00200120704703F48253B3F51D
:207DE000825F03BFC81FB0FA80F040090020704770B5BC4C94F8013C012B84B000F04D81AB
:207E000094F80D0CFCF778F894F80E3C834205461FD0002800F0D680D4F8A03ACBB194F869
:207E2000912593F90400002A18BF08224FF4964100230325CDE9015200911A4608212EF02B
:207E400024FBC4F89C0A20B1FEF780FF012384F80E3C94F80F3C012B00F0C180D4F8186CEE
:207E60003EB1A14B30465978FFF7ACFF002840F0F28094F81D0CFCF73FF894F81C3C8342ED
:207E8000054621D0002800F0F680EEB1337A002B00F01881954A02EB8303DB6994F8902541
:207EA00096F904000093003A18BF012202210023CDE901121A4610212EF0E7FAC4F8600AA3
:207EC00010B1012384F81C3CD4F8206C3EB1864B30465978FFF776FF002840F0AC8094F80F
:207EE0002C0CFCF709F894F8243C8342054622D0002800F0C980F6B1337A002B00F0E58033
:207F00007A4A02EB8303DB6994F8902596F904000093003A18BF012202210023CDE901123C
:207F20001A464FF400712EF0B0FAC4F8280C10B1012384F8243C94F82D0CFBF7DDFF94F895
:207F40002E3C8342054631D090B3694BD4F8306CD3F800354FF47A721A613EB34FF4805297
:207F6000402130462EF020FA0546F8B994F8903596F90400002B14BF0921082103224FF459
:207F8000E133CDE9012100932A462B464FF480512EF07BFAC4F8340C40B10123C4F85C0AA7
:207FA00084F8365A84F8385C84F82E3C04B070BDD4F8340C2EF0CAF9C4F8345C84F82E5C9F
:207FC00004B070BDD4F89C0A2EF0C0F994F80F3CC4F89C5A012B84F80E5C7FF43FAF94F8EF
:207FE000100CFBF789FF0546002871D0D4F8B435002B7FF433AFD4F8142C002A3FF42EAFBC
:020000040801F1
:2080000094F8915594F8901592F90400002D14BF08220022002908BF42F0010203254FF452
:208020006141CDE9015200911A4620212EF02DFAC4F8B40512E794F8243C002B7FF47BAFFC
:20804000D4F8083C002B3FF476AF0122C4F8283C84F8242C6FE794F81C3C002B7FF434AFC3
:20806000D4F8083C002B3FF42FAF0122C4F8603A84F81C2C28E7D4F8600A2EF067F9C4F8F8
:20808000605A84F81C5C1FE7D4F8280C2EF05EF9C4F8285C84F8245C4DE7D4F8045C124BBE
:2080A00028465978FFF78EFE20B3D4F84436002B7FF4A6AED4F8083C002B3FF4A1AEC4F87B
:2080C00044369DE64FF49643E8E64FF461431BE7D4F8B40500283FF4C1AE2EF037F9C4F877
:2080E000B455BBE670B90020A065002014480708D84C002094F80C0CFBF7FEFE0646D8B152
:20810000D4F84436002B7FF47BAE002D3FF478AE94F8902595F90400B2FA82F252094FF43B
:2081200016510225CDE9015200911A4604212EF0ACF9C4F8440663E6D4F8440600283FF40F
:208140005FAE2EF003F9C4F8446659E670B5C94C94F8013C002B00F0BF8108202EF038F97E
:20816000C4F8A00A00283CD008212EF027F900260346C149C14884F80D3C0522C4F8406C28
:208180003AF0D6FF41F208530122BC48A4F8443C84F8482C0DF008FD31462B22B8485CF00D
:2081A00002FA48F67C607D25E02331462B22A4F8500CB44884F8533C84F87B5C5CF0F3F9B6
:2081C00048F67C21A0224EF27B0384F8A75C84F8AA6C84F8535DA4F87C1C84F87F2CA4F810
:2081E000A83C94F80F3C002B00F0608110202EF0EFF81021C4F8180C2EF0E0F8A24B84F823
:208200001D0C3A2140F23B1094F86D2618809F254AF21E40197100219D7198601973002AE1
:2082200040F00E8194F86E36002B72D1D4F88035580700F1FE80990700F1F2801A0700F17D
:20824000E880924D2868C0F3C010FEF73BFD0020FEF71EFD03464FF4007084F8983A2EF0FF
:20826000B7F84FF40071C4F8200C2EF0A7F8D4F8543D84F82C0C002B14BF0123002384F824
:20828000583D40F09280D4F88C3B002B14BF0123002384F8613D43D1D4F8A42E0023C4F884
:2082A000F43B002A00F0DC80012284F8C43A84F8A82E002376487749C4F8B43A06223AF08D
:2082C00037FF40F609437248A4F8B83A0DF06CFC4FF480502EF07CF84FF48051C4F8300C88
:2082E0002EF06CF8D4F8B03E6B4A6C4D84F82D0CC4F8202702F5A070591C0022C4F8240797
:20830000C5F81031C4F8B01E84F82E2CBDE870406EE5D4F8943A43F00403C4F8943A85E78D
:20832000D4F88005002310F0020084F8623D84F8633D40F0EA80024694F86D362BB1012082
:20834000FFF7F6F8002840F0F28094F86E36002B40F0E7800820FFF7EBF820B1A3180421CB
:2083600083F8641D01322B681B0600F101814C4B10219818053300F8011B8342FBD105212C
:20838000092042F2090384F8691D84F88D0E45494548A4F8983E2025042284F88E5E3AF0D1
:2083A000C7FE41480DF000FC76E794F86D362BB10120FFF7BDF8002840F0BF8094F86E268B
:2083C000002A40F0E2802B681B0600F1BA80D4F880154E070CD54FF48060FFF7A9F838B1C8
:2083E000A318082183F85C1D013284F8602D4AE7080705D54FF40070FFF79AF80028EFD12C
:208400000905F2D54FF40060FFF792F80028ECD0E6E7D4F8943A43F48073C4F8943A10E76E
:20842000D4F8942A42F4601242F0C002C4F8942A04E7D4F8942A42F40272C4F8942AFAE623
:20844000D4F8943A94F86E2643F00201C4F8941A002A3FF4EBAE43F03603C4F8943AE5E60B
:20846000D4F8AC3E002B4BD0012384F8A83E84F8C43A1EE770B9002078480708ACC5002052
:20848000C0C50020ECC50020BC6C0020146C002020C4002020490708A0C00020E40400207A
:2084A000D4C60020CC48070800C8002020202DF08FFFC4F8140C00283FF498AE20212DF031
:2084C0007DFF354BC4F8843584F8100CFFF73CF8012384F80F3C89E604202DF079FFC4F89A
:2084E000040C00283FF439AE04212DF067FF2B4A84F80C0C0123C4F8882584F8013C2CE621
:2085000084F8A83E84F8C43AE2E64FF46070FFF70FF800283FF40FAF012084F8640D024638
:208520000AE70620FFF704F800283FF413AFA318022183F8641D01320CE7012284F85C2DED
:2085400041E74FF4A050FEF7F3FF20B1A318022183F85C1D01324FF40850FEF7E9FF002863
:208560003FF435AFA318042183F85C1D01322EE74FF45850FEF7DCFF00283FF4F8AEA31851
:20858000082183F8641D0132F1E60620FEF7D0FF0028D2D1024616E7556B0108012E0108B1
:2085A00030B40023022515244FF4167140F2D93205808471018130BC4281438083808381D8
:2085C0007047084B5A881B88801A9B1AC00090FBF3F00628A8BF062020EAE070C0F1960033
:2085E000C0B27047D4BF0020074B084A33F81010127802EAD122520705D0DA6F511CD96723
:20860000134483F880007047BCC800209806002010B5164B42681B7803F00303032B21D173
:20862000134B1B88DBB1134B1349B3F9BE30B1F904100A2491FBF4F15B1A1B0103F5B95367
:2086400014334FF4B471B3FBF1F3C3F1080303F00F0360331370436800225A7010BD052373
:208660001370F8E72D231370F5E700BFB8BF0020BABF0020BCC8002000C000204368722237
:208680001A70436873225A70436874229A7043680022DA7070470F4B4268B3F904300A211E
:2086A00093FBF1F31B0110B503F5B9530A4C4FF4B4711433B3FBF1F303F00F031919E3585A
:2086C00013604B6853600B7A1372436800225A7210BD00BF00C00020FCE80708044B93F8E5
:2086E000C53013F0FD0F14BF9E209D20704700BFBCC80020094B93F8C53013F0FD0F06D154
:2087000042F210735843064B90FBF3F07047242358434FF47A7390FBF3F07047BCC80020B6
:2087200040D20600064B07EE900A93F8C530B8EEE70A1BB9DFED037A20EE270A704700BF58
:20874000BCC8002048F9514010B5104B93F82C21012A10D1D3F83021811A00290BDD0221B4
:20876000B3F8264183F82C110949B1FBF4F142B10A44C3F8302193F82C01013818BF012016
:2087800010BD0844C3F83001F5E700BFBCC8002040420F00831E00F17A02EA2123F8021FAF
:2087A0009342FBD14E2243F64913C280CE2243850281CD2323228380A0F87220A0F87830F4
:2087C000704700BF08BB1F48B0F8343103F001036BBB30B490F83841ACB11B4A02F1F00540
:2087E00002E00133A3420ED052F8041B4904F8D590F8241200EB8101D1F8BC1145F82310EC
:208800000133A342F0D130BC70470E48B0F83421032A4FEA52030BD90A68A0F8343102F583
:20882000C332A03203F001030A60002BD1D070470B6803F5C333A03348F205020B60A0F815
:2088400034217047BCC80020F8C900202DE9F04100283AD12D4A92F8380180B32C4A2D4BB2
:2088600092F804E092F905C092F90680CEF1FF07AEF17F06FFB2F6B203EB800003F1F00293
:20888000002403E0834202F1040218D053F8041B8904F7D5E1B2A1EB0C0181EAE175A5EBEB
:2088A000E175012D0DDC71B1414514BF394631468342D17004F1010402F10402E6D1BDE885
:2088C000F0810821F4E77146F2E7114B1A79F02A09D802F10F000D4A18710B6803F5824397
:2088E0001A330B60B7E7094A93F9054092F83A017F2584421D71987905DB4042C0B2987153
:2089000020445871E9E7002CFADAF6E7BCC8002098060020F8C90020F0B5384E78B196F858
:20892000AC32002B46D0364A013BDBB286F8AC321378DC0741D4334B0A681A440A6096F8AA
:2089400038414CB3304B2E4F03EB840403F1F001002503E09C4201F104011DD053F8042B08
:20896000C2F303200628F5D13878C00715D596F8AC0296F83BE100EB050CBCFBFEF00EFB3A
:2089800010C00128CCBF0020012058B99C4205F1010501F10401E1D1F0BDE84300F00100B5
:2089A0000028F3D0C2F3834206EB8202D2F8BC210A60EBE796F83B31B5E7144A144BD2EDE8
:2089C000037A144CFDEEE77A642017EE902AA2F57A7200FB02F283FB0230D317C3EBA013BE
:2089E00003EB4303C3EB031384FB0302DB17C3EB62130533084A92FBF3F39DE7BCC80020C1
:208A000028BF0020400D0300F8C90020686D0020D34D62101F85EB5140420F00F0B4524CE4
:208A2000002868D194F8AD02002856D04F4BD3ED007AB3EE097AF4EEC77AF1EE10FA4EDC1E
:208A4000BBEE097AF4EEC77AF1EE10FA4CBF08270027D3ED017AB3EE097AF4EEC77AF1EE1C
:208A600010FA3EDD47F0010794F83851ADB3404ADFF808C102EB850502F1F00014E094F918
:208A8000B062B142ACBF0221002194F9B162B3421CDB41F004010F421CBFDCF80C300360C1
:208AA000954200F1040018D052F8043BD903F7D594F9AF6203F00F01B142C3F30313DEDCB7
:208AC00094F9B162B3424FF00101E2DA94F9B262B342D8BF41F00801DDE7F0BC704704274B
:208AE000B7E7BBEE097AF4EEC77AF1EE10FA48BF47F00207B8E794F8AE3263B31B4B1D4D68
:208B0000D3ED007A93ED017A0A6894F8AD02F0EEE77AB0EEC77AF4EEC77AF1EE10FAB8BFD2
:208B2000F0EE477AFDEEE77A80F0010017EE903A193B03EB4303C3EB031385FB0365DB17E4
:208B4000C3EBE51305330C4DB5FBF3F31A440A6084F8AD0268E70B6894F8AD0203F54333EA
:208B600003F5A0730B605FE7BCC80020C4BF0020F8C90020353AFC4440420F00A8490708D1
:208B8000F0B40B4F97F8386186B107F59E72054607F50B77002352F8044B35EA040004BF01
:208BA000086847F823000133B342F4D1F0BC7047BCC8002030B42A4B60B92A48027DCAB908
:208BC00093F825322849203301EB830130BC4FF4A060D5E793F8B322F2B1013A214883F872
:208BE000B3220A6802F5C32202F520720A60027D002AE5D01D4A12689106E1D51C4A93F8E2
:208C0000B312127892071AD511BB93F827321649203301EB8301D9E7124893F8B442057D8E
:208C2000A54205D8042483F8B42283F8B342D8E70134012283F8B44283F8B322D1E70029CE
:208C4000BED193F826320849203301EB8301BDE793F823320449203301EB8301B6E700BF9E
:208C6000BCC80020A46C0020F8C90020F0BE0020B8BF002010B41E4A48B91E4C92F8B50202
:208C80000B6823440B6098B15DF8044B704792F8B63203B3012B16D092F8B5020B68164C9B
:208CA00080F00100234482F8B5020B600028EBD192F8233211495DF8044B203301EB8301BC
:208CC0004FF440705CE792F8B5020D4C80F0010082F8B502D4E70B685DF8044B03F57423C1
:208CE00003F5107301200B6082F8B502704700BFBCC8002040420F0048E80100F8C900207F
:208D000020A107003C4AA0B992F8B7326BB192F8B8128A081341DB070AD501F00101032A02
:208D200006D8DFE802F05048403892F8BA3253BB704792F8B832013303F00F0382F8B83240
:208D40003BB192F8B732086800F5C330A0300860DCE72A4882F8B732437A002B44D128481F
:208D6000C07818B143F0040382F8B73225480078C00730D592F8B9020028E4D043F0080345
:208D800082F8B732DFE792F8C6321F4901EB83014FF40030F4E61C4B03F13002002914BF7A
:208DA00019461146F4E7194B03F1180200290CBF19461146ECE7144B03F10802002914BFDA
:208DC00019461146E4E7104B03F11802002914BF19461146DCE70E4800680028CAD043F081
:208DE000010382F8B732C5E792F8B632002BB6D0022382F8B732B2E7BCC80020D4BF0020C5
:208E00002CBF002028BF0020A8490708B8490708E4C3002030B4022340F203154FF4FA7465
:208E2000322146F20142C37000238580C480018130BC42810380704770B40B4C0B490C4B34
:208E400022680E680D6883F8E002002122F0200283F8E412C3F8D062C3F8DC522260C3F867
:208E6000D81270BC704700BFF0BE0020C42F0020BCC8002090F8603043B9426901210720D9
:208E800082F84430A2F8460082F848107047044B0449B3F908304068012248F073BB00BF0B
:208EA0009806002026E10708064B07491A88074B40681B68534342F2107293FBF2F248F028
:208EC00061BB00BFBCBF0020D2E10708F0BF0020044A05495378127840680133013248F053
:208EE00051BB00BF9CC40020D7E107080B4B4068B3F904300A2293FBF2F31A0102F5B952C6
:208F00004FF4B4711432B2FBF1F2C2F1080202F00F020349603248F035BB00BF00C00020AE
:208F2000DDE10708034A044992684068072348F029BB00BFF0BF0020E4E1070807B5144A66
:208F4000406892F8E812B2F8EA32012909D1009392F8EC320F497B2248F014FB03B05DF89C
:208F600004FB022906D10C497B2203B05DF804EB48F008BB0A22534340F2FF32B3FBF2F354
:208F80009BB2092B054928BF09237B22EDE700BFBCC80020EAE10708F9E20708F4E1070873
:208FA00013B54468FFF79AFB0F4B1B789B07024612D50E4B93F8F7120D4B59B19889FFF78E
:208FC00099FB0C49009203467022204648F0DAFA02B010BDD889F2E7009007492D2370224E
:208FE000204648F0CFFAF3E7B8BF0020BCC80020A46C0020D3E20708FAE10708034B04497C
:20900000D3F8FC22406848F0BDBA00BFBCC8002001E20708044B1B78DB0703D4034940682C
:2090200048F0B0BA704700BF28BF002005E2070807B5094A0949B2F906300193B2F9043066
:209040000093B2F902304068B2F9002048F09AFA03B05DF804FB00BFE85900200EE207083B
:20906000084BD3F80C23002A0ADD074B03EB82035A6B2AB1054B0649DB68406848F082BA2F
:20908000704700BFBCC80020A84907089806002022E207081FB593880293937801935378F7
:2090A000009313780A46034948F06CFA05B05DF804FB00BF2AE20708024B03491A684068B2
:2090C0001432E7E7ECC300203DE20708024B03491A6840680832DDE7ECC3002041E20708BD
:2090E000024B03491A6840680E32D3E7ECC3002045E20708044B93F829310BB127F072BC79
:20910000024B1888704700BFBCC80020BCBF002010B5184CA379CBB194F82230DFED166AC2
:2091200007EE903AF8EEE77A144B86EEA77AC0B203EB8000838907EE903AF8EEE77A67EEEE
:20914000277AFDEEE77A17EE900A10BD0C4B1B6813F000630CD0C0B2FCF724FE8089642383
:2091600010FB03F094F822305B0890FBF3F0ECE71846EAE76C300020000048435C2F00105E
:20918000146C002008B5FFF7C3FF3C2390FBF3F008BD074B93ED6E7AD3ED6B7AB4EEE77AC6
:2091A000F1EE10FA03DD034940685BF020BA7047C01400109EEA070810B50C4698B9174AD2
:2091C000174892F8101323680344236001B110BD92F8233213492033BDE8104001EB8301BC
:2091E0004FF48060CCE414F04BFD32280ADD23680A4A03F5742303F510730121236082F807
:20920000101310BD054A92F81013142881F00101CCBF0548054882F81013D4E7BCC8002092
:2092200040420F00F8C9002020A1070048E8010010B5044624F0C4FD03490346042260685C
:20924000BDE8104048F09EB926E10708224B1B885A0510B5446805D520462049BDE81040F6
:209260005BF0C5B9180505D520461D49BDE810405BF0BDB9590605D520461A49BDE81040B5
:209280005BF0B5B9DA0705D520461749BDE810405BF0ADB99B0705D520461449BDE81040BA
:2092A0005BF0A5B925201FF019F928B120461049BDE810405BF09BB90E4B1B782BB1204645
:2092C0000D49BDE810405BF092B920460B49BDE810405BF08CB900BFFCBF002049E207089A
:2092E0004EE2070853E2070858E207085DE2070862E20708ACC4002067E207086CE20708BC
:20930000032811D8DFE800F00A0C0206074BD3F818037047064B1B78DB0701D434F0E2B91B
:20932000024BD3F81403704700207047BCC8002028BF002037B504462A4800EB4303B3F841
:20934000C65005F00F0049B1022804F101011DD8002814BF9C239B2323700C460AB3C5F311
:209360000315FFF7CDFF3C21012D1F4BB0FBF3F3B3FBF1F201FB123315D0022D23D01B4950
:20938000204603B0BDE8304048F0FCB8032806D1174B1B7803F00103653BDBB2DCE7202392
:2093A000DAE71546DDE7642542F21071B0FBF1F1B1FBF5F005FB101000900E49204648F0CC
:2093C000E1F803B030BD0A250B49B0FBF1F1B1FBF5F005FB101000900849204648F0D2F80A
:2093E000EFE700BFBCC8002040420F0071E2070828BF00207BE20708A08601008AE207082C
:20940000037840680122053B114693E7F0B52B4B2B4E1C68317887B0074620460AF02EFA28
:209420007178054620460AF015FA00220592B2788DF8132003466CB1039005A920460AF0E7
:209440002FFA327A039B2AB10DF1130120460AF02DFA039B9DF81310ECB1E1B1194A1268C3
:20946000914218DC184A02EB8102D2F84043039326201FF033F80599039B70B911F0010F7A
:2094800014BF502200228907786808D50F4948F079F807B0F0BD0E4CE9E74422F3E732B166
:2094A000CDE900420B492A4648F06CF8F1E70A4900942A4648F066F8EBE700BF8CBF002093
:2094C000B86D002098B90020BCC8002099E207086EEC0708A1E20708ADE20708F8B5044618
:2094E0002D4B4178827893F8E10023780138302B2A4B4FEA8000034429480BBF93F8BC505F
:2095000093F8BE5093F8BD6093F8BF6000EB8505D5ED007AFDEEE77A00EB860017EE903A23
:20952000D0ED007A40F2CF75FDEEE77AAB4217EE900AA8BF2B46B3F57A7FB8BF4FF47A7386
:20954000A8424FF47A77A8BF2846A3F57A73B842C3EB0313B3FBF7F3C3F10E03B8BF384683
:20956000DBB24FF0030CB3FBFCFC0CEB4C0EA3EB0E03A0F57A706244C0EBC0000833B0FB04
:20958000F7F73944DBB2D2B2C9B22046F5F7B2FA00232373F8BD00BFBCC80020A849070805
:2095A000686D00202DE9F04790F8029090F8018009F1020704460026FFB2002508EB060AFA
:2095C000032E1BD108F10301022DC9B20ED10B233A462046F5F78EFA0135052DF0D1013600
:2095E000072EEAD100232373BDE8F08709EB05021623D2B22046F5F77DFAEDE7022DEBD166
:2096000017233A465FFA8AF12046F5F773FAE3E770B504466FF00205A278617852FA85F2A8
:2096200007391323D2B2C9B22046F5F763FAA2786178EEB2324407311323D2B2C9B220462A
:209640000135F5F757FA042DE6D16178A27806390323C9B22046F5F74DFA6178A278063119
:209660000223C9B22046F5F745FA0023237370BD2DE9F8432B49054691F8D03091F8D120C0
:20968000294891F8DF10B0F90040002902EB820214BF4FF0FF31012152004C43C2F100085E
:2096A00003EB830344454FEA430303DB9442A8BF1446A046B0F902205C424A43A24203DB1B
:2096C0009A42A8BF1A4614461BB11922544394FBF3F4293C4FEA88066FF003074FF0090993
:2096E000002E3346B8BF06F13F03C4EBA313512B0FD893FBF9F101EBC1029B1AAA780A44FF
:209700006978803B3944DBB2D2B2C9B22846F5F7F1F90137052FA6EB0806E1D100232B73E2
:20972000BDE8F883BCC8002000C0002010B5044614F0E2FA642202FB00F3C3F38F23632B2A
:2097400060680449BDE8104028BF6323012247F019BF00BFF9E207081D4B1E499A68B1F83D
:20976000C0309FED1D7A406807EE902AF8EEE76A07EE903AF8EEE77A67EE877AF4EEE76AB9
:20978000F1EE10FA02D8154947F0FCBE934202DA134947F0F7BE9B1A07EE903AB8EEE77A43
:2097A000D1EDC57A0F4AF8EE677A3C2167EE277A87EEA67AFDEEC77A17EE903AB3FBF2F316
:2097C000B3FBF1F201FB1233074947F0DBBE00BFF0BF0020BCC80020CDCCCC3DB6E207081C
:2097E000BCE2070840420F0071E20708244A00234361D2F8D41041F45C5130B541F02C01C1
:209800000124C2F8D4104471D2F8CC1004FA03F50133112B41EA0501F8D121F4F0314FF451
:209820002063C2F8CC10C38040F601230381154B0360142303718023037642F614035022A3
:20984000114903824FF6FF734383A0F8562003F58C036FF07E42C0E91612C3610B4A40F27C
:20986000012303844FF0A0640023C0E9184280F8223080F8333080F84430A0F8683030BD26
:20988000BCC8002098086400C4FF00FF180B0C002DE9F84305461CF0E5FB1D4EDFF8749061
:2098A000074600244FF0880833786968A342214403DC00230B70BDE8F88337B3D6ED427A9C
:2098C000FDEEE77A09EB840317EE900AD3ED007AFDEEE77A17EE902AD6ED437AFDEEE77A11
:2098E000121A17EE903AD2001B1A92FBF3F3C3F188030B702046FFF70BFCB0F57A7F02DA5C
:209900006B6853221A550134CEE781F80080FAE780060010E02F001013B5374BC1789A6892
:20992000364B02299B89044641D0032945D0012905D19A1A9A42A8BF1A4622EAE272D3B180
:209940009A1A9A42A8BF1A4622EAE27207EE902A0B20B3FBF0F307EE103AF8EEE77AB8EEB9
:20996000C70A87EE800A59F08BFAFCEEC07ACDED017A9DF8043062688A2111700122616845
:209980009342ACBF8B208D20885401320C2AF6D162688F2111735A1E092A03D8626813447E
:2099A0008E225A70636800225A7302B010BD9A1A9A42A8BF1A4622EAE272ABB107EE902A32
:2099C000B8EEE70ADFED0E7A20EE270A07EE903AF8EEE77A80EE270A59F0E0FA64280346C0
:2099E000A8BF642323EAE37306496068072202B0BDE8104047F0C6BDF0BF0020D4BF0020F3
:209A00000000C842C2E20708084B93F8C53007EE900A4BB9F8EEE77A9FED057A9FED050A36
:209A2000A7EE870A59F0BABA704700BFBCC800206766E63F000000420D4B1B681B0137B512
:209A400014D50C4C4568D4F8643393F90100FFF7DBFF94F8C5200849002A0CBF0D220E2242
:209A60000346009228467A2247F08CFD03B030BD146C0020BCC80020C9E207080B4B13B585
:209A80004468B3F90000FFF7BFFF094A094992F8C520002A0CBF0D220E2203460092204611
:209AA0007A2247F06FFD02B010BD00BFA4C30020BCC80020D2E207082DE9F0472DED028B47
:209AC00082B092469DF834809DF8302007460C469946002B52D0022B14BF0A25642507EED6
:209AE000905AF8EEE77A27EE808A002A48D0B0EE480A59F053FA07EE900AF8EEE77AF0EE9A
:209B0000E77AFDEEE77A17EE906AB6FBF5F205FB12660CB13C700124B5EEC08AF1EE10FA25
:209B200005D552EA060302D02D233B5501349AF80010154B3819002914BF5146194647F0A3
:209B400021FD2518B9F1000F0AD010494A46684647F018FD78193246694647F013FD0544EC
:209B6000B8F1000F02D007F805800135002328467B5502B0BDEC028BBDE8F0870125AEE781
:209B8000F0EE487ABBE700BFDBE20708E0E207081A4B1A6812F0200F13B502F004034468A2
:209BA00025D0174A1278920721D5164BB3F90000FEF7B8FDDFED147A144B154A93F8C530E7
:209BC00020EE270A2046B5EEC00AF1EE10FA4CBF76217521002B0CBF99239F230193012326
:209BE0000093B0EEC00AFFF767FF02B010BD002BDBD12D22227042685370F6E7F0BE0020BF
:209C0000B8BF002006C000200AD7233CBCC80020C43208081FB5184B9FED187A1B88184A83
:209C20009FED180A92F8B622446807EE903AF8EEE77AF4EEC77AF1EE10FAACBF01230223A2
:209C4000022A27EE800A14D08DED030A029326F0C9FEFEF7B6FC029B9DED030A0146012217
:209C60000620CDE90020084A2046FFF725FF04B010BD9721F3E700BFBCBF002000007A44EB
:209C8000BCC800200AD7233CC4320808114BB3F86833B3F57A7F07B5406806D20E490122E1
:209CA00003B05DF804EB47F06DBC07EE903A5722F8EEE77A00239FED090ACDE90032012300
:209CC000074A27EE800A1946FFF7F6FE03B05DF804FB00BFBCC80020E8E207086F12833ACA
:209CE000C432080873B5194E96F8E032052B0546406807D016491F231E2202B0BDE870404D
:209D000047F040BC134C1449237D00931E221F2347F038FC96F81A31ABB16B68DFED0F7AD7
:209D200020221A54638A0E4A00EE103A441CB8EEC00A686801230021CDE9003120EE270AEB
:209D40002044FFF7B9FE02B070BD00BFBCC80020F0E20708A46C0020F7E207080AD7233C77
:209D6000C432080807B501234722CDE900320549054A91EDDB0A40680021FFF79DFE03B09F
:209D80005DF804FBBCC80020C432080807B50B4BDFED0B7A93ED000A0A4A00219A23B8EE00
:209DA000C00ACDE9001320EE270A0223B0EEC00A4068FFF781FE03B05DF804FBF0BF002051
:209DC0000AD7233CFFE2070813B5044626F00AFE0E4B646893F8B632022B00EE100A13D073
:209DE000FEF7EFFB0146DFED0A7AB8EEC00A00230622CDE9003220EE270A064A0223204630
:209E0000FFF75AFE02B010BD9721ECE7BCC800200AD7233CC432080813B50378134ADFED94
:209E2000147A144C1A2B0CBFB2F90220B2F9002000EE102AB8EEC00A1A2B20EE270A4FF031
:209E400001034FF00002CDE90032B5EEC00A0CBF15211421F1EE10FA074A406848BF2246E1
:209E6000B0EEC00AFFF728FE02B010BD00C00020CDCCCC3D03E3070809E30708194B1A6887
:209E800012F0200F13B502F00403446820D0164A127892071CD5154BC27893F8C530002B7B
:209EA000134B18680CBF0F210C21FEF73BFC0123DFED107A0093D31A01910F4A20EE270A4C
:209EC00018BF01237F212046FFF7F6FD02B010BD002BE0D17F22227042682D2151704268A7
:209EE0009370F3E7F0BE0020B8BF0020BCC80020DCC300200AD7233CC432080813B5044665
:209F000008461146FEF70EFC174B93F8C530002B0CBF4FF4A5534FF47A7307EE903AF8EEB5
:209F2000E77A08BF7E22F4EEC07A16BF7D220F230C23F1EE10FA13DC80EE270AF2EE047A93
:209F4000B4EEE70AF1EE10FAACBF012302230192002200922046054AFFF7AEFD02B010BDB5
:209F60001A460023F3E700BFBCC80020C432080810B40C4B44681B7803F00303032B06D1C3
:209F8000094B204619885DF8044B1122B6E71123237043682D225A70436800229A705DF83B
:209FA000044B7047B8BF0020BABF0020094B40681B7803F00303032B07D1074B7122D3F82D
:209FC00070136423B1FBF3F198E704492D23712247F0D8BAB8BF0020BCC80020FCE1070848
:209FE00010B5044613201EF079FA48B30BF062FE30B960681349BDE81040102247F0C2BA61
:020000040801F1
:20A000000BF0C8FE034660682BB1BDE810400E49102247F0B7BA0D4B93F87523022A4FF086
:20A02000100208D1D3F89033002B04DBBDE81040074947F0A7BABDE81040064947F0A2BAE9
:20A0400010BD00BF0FE3070813E30708BCC8002017E307080B270808244B1A6812F020026A
:20A0600013B5044624D0224B1A7812F001021FD0204B1A7812F002021AD01F4BD8896328A4
:20A080002AD9FEF737FB1D4BD3ED007A07EE100AF8EEE77AB2EE040A67EE807AB8EEC70A2A
:20A0A000174887EE800A41F0EDFA58F077FF0246144B606893F8C530541E002B42F20E712D
:20A0C0000CBF7E237D238C4208D800930E49072347F058FA02B010BD0022E9E70B4907223B
:20A0E00002B0BDE8104047F04DBA00BFF0BE002028BF0020B8BF0020A46C0020F0BF002051
:20A1000054CC0020BCC800201CE3070825E3070838B5802200F18004002105465AF043FA3F
:20A120000021204638225AF03EFA0C49002351F8232044F8232001330E2BF8D108491E2272
:20A1400005F1C0005AF0CEF906490B2205F1E4005AF0C8F9032385F8EF3038BDA849070820
:20A16000744A0708944A07082DE9F04FCC4907780E784468C578172F91B00CBF4FF0980E96
:20A180004FF0890E16F00406099004D0C54B172F0CBF5E681E68DFF834C386EAE673A3EBDA
:20A1A000E673022DB3FBFCF20CFB123300F09C81032D15D0012D03D14FF47A71B3FBF1F34B
:20A1C000002EBBBF2D216170601CA01C84F800E0B549B64C002D08BF214647F0D3F916E1CF
:20A1E00022461E2302F8023B1F2363700B7813F0040300F06F81AB4D686857F0EDF89CA3CA
:20A20000D3E9002357F052F9824628688B4657F0E3F897A3D3E9002357F048F9A44B0022D0
:20A2200006460F4657F0C8FB08B9A14F0026A14B00223046394657F0B5FB08B99D4F0026CF
:20A240009C4B00223046394657F0A2FB40B93046394689A3D3E9002356F070FF06460F46CD
:20A26000DFF86C924FF00008934B00225046594657F08EFB002840F0E580DFF854924FF004
:20A2800000088E4B00225046594657F095FB002840F0E1808A4B0BAA03F1100C186859681B
:20A2A000154603C5083363452A46F7D11B882B80304673A3D3E90023394657F0F7F872A3DD
:20A2C000D3E9002356F03CFF57F0EEFB70A3D3E90023074688465046594657F0E7F86EA375
:20A2E000D3E9002356F02CFF57F0DEFB4FF00F0905460E460DF12C0A4FF0FF3B0522002301
:20A300003846414657F06CFB05F00303069306F000430793DDE90601002871F100030BDAE4
:20A32000069B13F1FF330693069B63F0030101314BF1000306910793624B03EB8202069B53
:20A340001A443846137809F80A3005220023414657F046FB002D884676F1000107462A46E2
:20A36000334602DAEA1C46F1000309F1FF399508B9F10A0F45EA83754FEAA306BED14FF0DF
:20A38000000A284631461422002357F029FB4D4B9B5C10AA4A44069202F8143C384641464C
:20A3A0001422002357F01CFB464B9B5C069A384602F8153C41461422002357F011FB14228C
:20A3C0000746884628463146002357F009FBA9F1020B05460E46BAF1000F45D110AB5B449F
:20A3E0004FF02B02A9F1030903F8142C0AF1010ABAF1050FC5D10BAA631C04F10D0112F874
:20A40000010B03F8010F9942F9D10023A373099B2D491B785A0901EB820103F01F03012290
:20A4200002FA03F31E4AD1F8A003127802F00602042A0CBF034320EA0303C1F8A03311B036
:20A44000BDE8F08F5046594642464B4656F078FE82468B4608E75046594642464B4656F0B2
:20A460006DFE82468B460CE7D946BFE7AFF3008048AFBC9AF2D77A3E2D431CEBE236EA3E79
:20A480000000000084D77741000000D088C3E0410000000000405F410000000000F9D5417E
:20A4A000B8BF0020A46C002037E307082FE30708008056C000805640008066C00080664013
:20A4C00055E3070818E90708BCC8002080969800008076404FF02D31C4F802105160916090
:20A4E0002B22A272A37392E73C2101FB03F52046B5FBFCF40CFB14535943172FB1FBFCF528
:20A5000000F801EB0CFB15130C49B3FBF1F310D1002EB4BF5721452105912221CDE903311E
:20A520002723CDE9004306490295082347F02AF86DE7002EB4BF53214E21EDE740420F0031
:20A540003FE30708F8B52D4F0A24B7F9002092FBF4F484EAE473A3EBE4739BB25A2B054667
:20A5600005D90A32CCBFB4236FF0B3031C1B244E96F8B92232B9234B1B78DB0729D41BF062
:20A580007FFE30BB96F8AC33B32B02D81BF078FEF8B9B7F902100A2391FBF3F304B9C3B16A
:20A5A000002BB8BF5B4284EAE4709BB2A0EBE470B3EB400F6A6813DAB0EB430F10DA0929B9
:20A5C00008DD002CCCBF6E23622313706B6800225A70F8BD002CCCBF6A2366231370F5E7A6
:20A5E000834205DD0929CCBF602368231370EDE7002CCCBF6C2364231370E7E700C0002094
:20A60000BCC8002028BF002030B585B0054601A846F094FA044618B92870204605B030BD02
:20A62000044A0123B2F9002001A9284646F0C0FFF3E700BF706E00204068E5E773B50D4D43
:20A64000009104461646002302460221286838F0A1FD094B0093224628680023142138F080
:20A6600099FD2868009600232246162138F092FD02B070BDB06D0020E73408082DE9F04315
:20A68000B54C94F8AE338BB0DBB1B44FB449DFF820E3B44EB44A4FF0010C94F8AF33D4F825
:20A6A000D480FD18172B33D984F8AF3394F8AE3394F8B023002A40F0AE8284F8B0330120AF
:20A6C00023E094F8B053002DDFD0A84A1068027A95422946A8BF1146954238BF0131A2EB95
:20A6E000010202EBD27238BF0123C2F3470213B984F8AE23C9E7531C84F8AE339C4B0093FE
:20A700000221002338F046FD00200BB0BDE8F08315F8010B0CFA00F9013319EA080FDBB2A2
:20A72000C0D094F8AE5384F8AF331728B5D8DFE810F0180036004F0079008F00B200D300E1
:20A74000F3004101500161015D007201BA01CD01E301F80103029F00130236024102540251
:20A760002A0202AE3046FFF74FFF18B98149304646F008FF7D480096006800232A4602217C
:20A7800038F008FD794A94F8AE3312680133127ADBB29A4284F8AE338AD90020B5E7B4F891
:20A7A000C620002312F00F02194618BF012202A8FEF7C0FDB4F8C63003F00F026E4B03EB7B
:20A7C00082032846D3F8F81002AAFFF737FFD9E7B4F8C820012312F00F0218BF1A460021F8
:20A7E00002A8FEF7A7FDB4F8C830E5E7D4F82803FDF798FF94F8C530DFED607A604A002B28
:20A800000CBF0F230C230193012320EE270A0093002102A8FFF750F95A4902AA2846FFF7C5
:20A820000DFFAFE713681B067FF537AFB4F91C03FDF760FF0246FDF751FF5349034602A846
:20A8400046F0A0FE514902AA2846FFF7F7FE99E7136818067FF521AFB4F92C1302A8002270
:20A86000FFF74CFB4A4902AA2846FFF7E7FE89E713681B067FF511AFD4F87013642302A853
:20A88000B1FBF3F10022FFF739FB424902AA2846FFF7D4FE76E7B4F91E33DFED387A384A14
:20A8A00000EE103AB8EEC00A4FF0060C0123CDE9003C20EE270A0223002102A8FFF7FCF870
:20A8C00094F82901344B354902AA002808BF19462846FFF7B3FE55E7B4F82033DFED277A0E
:20A8E000274A00EE103AB8EEC00A01230627CDE9003720EE270A0223002102A8FFF7DCF808
:20A9000094F82901264B274902AA002808BF19462846FFF793FE35E7FEF7ECFB07EE900A2A
:20A92000B8EEE70ADFED157A154A01230626CDE9003620EE270A0223002102A8FFF7BCF8B1
:20A9400094F82901184B194902AA002808BF19462846FFF773FE15E7BCC80020B04A070804
:20A96000D4070010D4BF0020146C0020B06D0020A7E30708B7E30708A84907080AD7233CDA
:20A98000C4320808BEE30708CBE30708D0E30708DAE30708E7E3070874E3070867E307081E
:20A9A0008DE3070880E3070891E3070899E30708F0BE002002A994F82403F3F707F99749A2
:20A9C00002A859F0F8FD964902AA2846FFF736FED8E6B37A002B3FF460AEB4F92223914949
:20A9E0009A2302A846F0CEFD8F4902AA2846FFF725FEC7E6B37A002B3FF44FAE8B4A894908
:20AA00009268072302A846F0BDFD894902AA2846FFF714FEB6E694F87533002B3FF43DAE6B
:20AA2000032B3FF43AAE0BF045F994F87533012B21D0022B30D188B3F9F7B0FA4FF4FA62A1
:20AA40000668B6FBF2F641F2A8737A4AD0584FF47A22B0FBF2F0301A642250437649B0FB7C
:20AA6000F6F202A892B246F08DFD744902AA2846FFF7E4FD86E688B1F1F7FCFB074647F08A
:20AA80000BFBBE887A88B21A466802FB066647F011F8B60A800ADFE700B1FFDE684902A84C
:20AAA00046F070FDE1E794F87533022B7FF4F5ADD4F890030028FFF6F0AD02A9F3F786F889
:20AAC000604902AA2846FFF7B9FD5BE6DEF8003098077FF5E2AD01234722CDE9003294ED28
:20AAE000CC0A594A002102A8FEF7E6FF574902AA2846FFF7A3FD45E6B4F93403FEF784FF61
:20AB000094F8C5304749002B02460CBF0D230E2302A846F037FD4E4902AA2846FFF78EFD3F
:20AB200030E602A9D4F83803F3F750F8494902AA2846FFF783FD25E6B4F83C23464902A8AA
:20AB400046F020FD354902A859F035FD434902AA2846FFF773FD15E6CB68002B7FF79DADDA
:20AB60000A69002A09DD3E4902A846F00BFD3D4902AA2846FFF762FD04E63B4A394928468F
:20AB8000FFF75CFDFEE5B4F93E23384902A846F0F9FC374902AA2846FFF750FDF2E502A9C0
:20ABA000D4F8FC02F3F712F8324902AA2846FFF745FDE7E53C21D4F80033B3FBF1F302A8A6
:20ABC000B3FBF1F201FB12332B4946F0DBFC2B4902AA2846FFF732FDD4E594F8C530D4F869
:20ABE000042373B940F249617E23B2FBF1F202A80C4946F0C7FC224902AA2846FFF71EFD67
:20AC0000C0E54FF47A717D23B2FBF1F202A8054946F0B8FCEFE7012077E500BFC7E2070885
:20AC2000F7E30708CBE3070800E40708F0BF00200CE407081CA10020C4E207081BE407080D
:20AC400015E4070824E40708C43208082FE407083BE4070848E407087630080854E4070847
:20AC60005DE4070862E407086BE4070826E2070874E4070881E407088FE4070898E40708D2
:20AC8000AAE407082DE9F043744B1F6883B0002F56D0FF238DF803308DF80230002877D1FF
:20ACA0006F4B93F8B123002A4DD093F83851002D46D06C4A93F8B6136B48536992F810804A
:20ACC00000294FF0000103F0010C14BF4FF00F0E8E4600F1F0020B460F4612E0984554D389
:20ACE000BCF1000F51D174461E260133DBB216809770D4700131A94222D0062B02F104029D
:20AD00001ED050F8044B2404F4D5002BE6D174467826EAE7012203EB82027169D2F8BC219C
:20AD20000192CA077CD593F8B633002B14BF0F23002301A94FF400408DF80730FDF720FF9B
:20AD400003B0BDE8F083474EB3F8B22341F228618A42DFD941F24F618A4263D941F27661DE
:20AD60008A4261D941F29D618A4262D941F2C5618A426FD941F2EB618A426DD941F21271E1
:20AD80008A4294BF0B220D22C5E700242646ACE7344E0DF102020C4638460DF1030108F01B
:20ADA00088FD06F11001384608F080FD06F11401384608F075FD9DF803909DF80280494651
:20ADC0004246384608F0F2FC7569317C244B05F0010505EB410505EB091593F8B123A3F854
:20ADE000B20305EB0825ADB202BBB3F8B423AA4221D0A3F8B4530F22206893F8B65300F522
:20AE00004331013AD2B201F5A07185F0010083F8B123216083F8B603002A7FF446AF92E773
:20AE2000FF2386E7022276E7032274E7A3F8B453E2E704226FE7216893F8B603A3F8B4235C
:20AE400001F5433202F5A07280F00101226083F8B61379E706225EE70A225CE78CBF00209F
:20AE6000BCC8002098060020F8C90020F0B55A4C5A4DD4F8B8232B68DFED596A594E29689C
:20AE8000C4F8B8139B1A07EE903AF8EE677AB7EE007A67EEA67A3378F4EEC77AF1EE10FAA5
:20AEA00088BFF0EE477A13F0010383B0C4EDEF7A0CD14D4A4D491278A4F8BE30D2070B80D6
:20AEC0002FD4012384F8DC3303B0F0BD01AB6A4604F5717104F57070F3F710FB4248444944
:20AEE000019B009A0078414FA1FB02C281FB03C1DB17C3EB61135209C1073A80A4F8BE30F9
:20AF0000DFD533782D68DB075FD594F8F732394E7BBBF3890F2B2ED8B068D4F8C833C11A3F
:20AF200005E0344ED4F8C833B0682D68C11AD4F8D823C4F8C8034FF47A73AA1A03FB01F327
:20AF400040F2DC5193FBF2F31BB28B422A4AC4F8D853A8BF0B469342B8BF1346D6E90021ED
:20AF6000A4F8D4330123C4E9F32184F8DC3303B0F0BDB389CEE7214901AB081F6A46F3F796
:20AF8000BDFA94F8F732B0684BB9D4F8C833009AC11AD4F870331344C4F87033C7E7D4F84E
:20AFA000C833DDED007AC11AF8EE677A07EE101A67EEA77AB8EEC77AE7EE077AB1EEE77ADE
:20AFC000FCEEC77A17EE902AE3E70A4ED4F8C833B068C11AABE700BFBCC80020C42F0020A3
:20AFE0006F12833AB8BF002028BF0020BABF00201F85EB51A46C002024FAFFFF8CCC002038
:20B0000090F8602062B910B50378032B29D0042B12D0022B1C4C08D0002384F8DD3310BDAC
:20B02000194B002283F8DD237047012384F8DE33002384F8DD3310BD4368017E5B78124CD0
:20B040000120814203F00F0384F8DE0310D00229E2D1002BE0D0162084F8DF232BF0ECFA5C
:20B06000DAE7094C002384F8DE2384F8DD3310BD2BB1152084F8DF132BF0DEFACCE7162066
:20B080002BF0DAFAC8E700BFBCC800202DE9F84306461D4C0D46D4F8E003317833F022FABF
:20B0A0007178D4F8E00333F01DFA022D29D0EB1EDBB20333002506F1020906EB03082F4632
:20B0C00019F8011BD4F8E0030D44EDB233F00AFA2F44C845FFB2F3D1D4F8E003294633F047
:20B0E00001FAD4F8E003394633F0FCF9F37884F8E2320022012384F8E32284F8E432BDE816
:20B10000F88300252F46E7E7BCC8002070B5002892B014BF082103214FF6FF7000238DF89D
:20B120000C10ADF80A00032413488DF80D4042F210724FF0FA11ADF80E30ADF81030ADF883
:20B1400014300A93ADF82C30ADF8122024230B4A0691079005264FF470554FF448042A215F
:20B1600001A8CDE90854ADF816600192ADF80830FFF78CFF12B070BD64002C01B562062447
:20B1800070B330B583B040F25514AA230022ADF800408DF803308DF802108DF804200DF10F
:20B1A000010401AD55235A400821530012F0800F08BF520083F0310314BFDAB2D2B20139E0
:20B1C000F3D1AC4202D014F8013BECE7AA2369468DF803208DF80430F1F7F6FD03B030BD78
:20B1E000704700BFF0B590F860309BB004467BB9416843694A7883F84420C8788A780121F9
:20B2000042EA0022A3F8462083F848101BB0F0BD466902E0306833F059F9306833F05EF9E4
:20B2200005460028F6D12946642201A859F0BBF91549164B164E1868D1F8E833039391F893
:20B24000E4138DF85B5003441791049311496369B578114F029740F2FF50CDE90513ADF801
:20B2600004005DB97078642202FB006001A9043059F038F9012263697570B2701868FF21FB
:20B280001BB0BDE8F0407BE7BCC80020C42F002034650020758E0108F46400202DE9F04F63
:20B2A000AA4C89B005460F46164694F8B69232F019FA8246002028703070D4F8CC8038707A
:20B2C00018F0010F49D01DF009F9002842D0A04B1A68002A3ED0910104D5B2F1007F18BFEB
:20B2E00002F17E42D4F8F4139FED9A7AAAEB010307EE903AF8EE677AF4EEC77AF1EE10FAFD
:20B3000005DCD4F8F80301238340134212D111B91923C4F8F833D4F8F833C4F8F4A301200E
:20B3200001331A2B28BF002300FA03F11142F7D0C4F8F833D4F8F823874B884903EB82039E
:20B340002846D3F8202146F01DF90223337009B0BDE8F08F0023C4F8F433D4F8FC338BB343
:20B360007F4B1B78DB072DD4D4F800349FED7D7A03F5921303F57863A3EB0A0307EE903A40
:20B38000F8EE677A67EE877AFDEEE77AB8EEE77A17EE903AF1EE0C7AB4EEE77AF1EE10FA1D
:20B3A00006DB7149284646F0EDF801233370CEE70A212846B3FBF1F201FB12336B4946F098
:20B3C000E1F8F2E718F4007F0BD0694BDB7843B16849284646F0D6F80323337001233B709F
:20B3E000B5E718F0200F16D01B201DF077F890B194F8B93223B16049284646F0C3F8D4E78E
:20B40000574B1B78D80706D45C49284646F0BAF8012333709BE718F4806F34D094F8043437
:20B42000012B30D1564B1B68990727D5554BB3F90220B4F91434D21A6FF463739A4218DBC8
:20B4400040F28D339A4217DC0A2392FBF3F24E49284646F097F822F0B3FC4C4B1B6893F85C
:20B4600063300A3B23EAE37398429EDB01233B709BE76FF05902EAE75A22E8E7444928461C
:20B4800046F080F8E7E718F4005F0ED012F0F8FB94F8C430834208D93E49284646F072F837
:20B4A0000223337001233B7051E718F4004F08D0394BB4F91821B3F908309A4201DD374902
:20B4C000EBE718F4804F07D012F0C2FBB4F81631834201D93249E0E718F0080F04D0B9F1B8
:20B4E000020F01D12F4974E718F4006F0FD01C4B1B78DA070BD51CF089FF40B12A4B1B78F4
:20B50000DB0704D594F851340BB92849C5E718F4805F14D0124B1B78D80710D51CF076FF7A
